:020000040800F2
:1000000000060020E1010008E3010008E301000808
:10001000E3010008E3010008E3010008E301000830
:10002000E3010008E3010008E3010008752F000860
:10003000E3010008E3010008E3010008E301000810
:10004000E3010008E3010008E3010008E301000800
:10005000E3010008E30100081D32000845320008F2
:100060006D32000895320008BD320008E301000837
:10007000E3010008E3010008E3010008E3010008D0
:10008000E3010008E3010008E3010008E3010008C0
:10009000E3010008E3010008E3010008E53200087D
:1000A000E3010008E3010008E3010008E3010008A0
:1000B000B9330008E3010008E3010008E301000888
:1000C000E3010008E3010008E3010008E301000880
:1000D000E3010008E3010008E3010008E301000870
:1000E00049330008E3010008E3010008E3010008C8
:1000F000E3010008E3010008E3010008E301000850
:10010000E3010008E3010008E3010008E30100083F
:10011000E3010008E3010008E3010008E30100082F
:10012000E3010008E3010008E3010008E30100081F
:10013000E3010008E3010008E3010008E30100080F
:10014000E3010008E3010008E30100082927000893
:10015000E3010008E3010008E3010008E3010008EF
:10016000E3010008E3010008E3010008E3010008DF
:10017000E3010008E3010008E3010008E3010008CF
:10018000E3010008E3010008E3010008E3010008BF
:10019000E3010008E3010008E3010008E3010008AF
:1001A000E3010008E3010008E3010008E30100089F
:1001B000E3010008E3010008E3010008E30100088F
:1001C000E3010008E3010008E3010008E30100087F
:1001D000E3010008E3010008E3010008E30100086F
:1001E00002E000F000F8FEE772B6374880F30888B6
:1001F000364880F3098836483649086040F20000E6
:10020000CCF200004EF63471CEF200010860BFF36C
:100210004F8FBFF36F8F40F20000C0F2F0004EF638
:100220008851CEF200010860BFF34F8FBFF36F8F8C
:100230004FF00000E1EE100A4EF63C71CEF20001E4
:100240000860062080F31488BFF36F8F01F034FF3D
:1002500002F02EFE4FF055301F491B4A91423CBF21
:1002600041F8040BFAE71D49184A91423CBF41F896
:10027000040BFAE71A491B4A1B4B9A423EBF51F83E
:10028000040B42F8040BF8E700201849184A914281
:100290003CBF41F8040BFAE701F012FF02F05CFEEC
:1002A000144C154DAC4203DA54F8041B8847F9E7A7
:1002B00000F042F8114C124DAC4203DA54F8041B22
:1002C0008847F9E701F0FABE00060020002200206E
:1002D0000000000808ED00E00000002000060020FB
:1002E0008037000800220020402200204022002009
:1002F000602E0020E0010008E0010008E001000895
:10030000E00100082DE9F04F2DED108AC1F80CD066
:10031000C3689D46BDEC108ABDE8F08F002383F3CF
:1003200011882846A047002001F076FAFEE701F088
:1003300005FA00DFFEE7000038B500F069FB01F0C8
:100340008BFE054601F0AEFE0446D8B90F4B9D4228
:100350001AD001339D4218BF044641F2883504BFCC
:1003600001240025002001F081FE0CB100F076F898
:1003700000F004FD00F0B2FB284600F0BFF800F0EA
:100380006DF8F9E70025EDE70546EBE7010007B05A
:1003900008B500F075FBA0F120035842584108BD94
:1003A00007B541F21203022101A8ADF8043000F0B4
:1003B00085FB03B05DF804FB38B5302383F3118867
:1003C000174803680BB101F0F3FA164A14480023EA
:1003D0004FF47A7101F0E2FA002383F31188124C92
:1003E000236813B12368013B2360636813B163681A
:1003F000013B63600D4D2B7833B963687BB90220F4
:1004000000F036FC322363602B78032B07D163683E
:100410002BB9022000F02CFC4FF47A73636038BDD6
:1004200040220020B9030008602300205822002049
:10043000084B187003280CD8DFE800F00805020804
:10044000022000F00BBC022000F0FEBB024B002299
:100450005A6070475822002060230020234B244A12
:1004600010B51C46196801313FD004339342F9D1CD
:100470006268A24239D31F4B9B6803F1006303F506
:1004800040439A4231D2002000F042FB0220FFF7A5
:10049000CFFF194B1A6C00221A64196E1A66196E76
:1004A000596C5A64596E5A665A6E5A6942F0800203
:1004B0005A615A6922F080025A615A691A6942F0F7
:1004C00000521A611A6922F000521A611B6972B651
:1004D0004FF0E0233021C3F8084DD4E9003281F316
:1004E00011889D4683F30888104710BD00C000089E
:1004F00020C0000800220020003802402DE9F04F03
:1005000093B0AA4B00902022FF210AA89D6800F01A
:10051000DFFBA74A1378A3B9A64801210360117035
:10052000302383F3118803680BB101F041FAA24A2A
:10053000A04800234FF47A7101F030FA002383F3CE
:100540001188009B13B19D4B009A1A609C4A009C35
:100550001378032B1EBF00231370984A4FF0000A34
:1005600018BF5360D3465646D146012000F076FBB3
:1005700024B1924B1B68002B00F01182002000F088
:100580007FFA0390039B002BF2DB012000F05CFB61
:10059000039B213B162BE8D801A252F823F000BFA1
:1005A000FD05000825060008B90600086B050008CF
:1005B0006B0500086B0500084307000813090008D5
:1005C0002D0800088F080008B7080008DD0800089B
:1005D0006B050008EF0800086B05000861090008BA
:1005E0009D0600086B050008A5090008090600081B
:1005F0009D0600086B0500088F0800080220FFF721
:10060000C7FE002840F0F581009B0221BAF1000FDF
:1006100008BF1C4605A841F21233ADF8143000F0B3
:100620004DFAA2E74FF47A7000F02AFA071EEBDBCE
:100630000220FFF7ADFE0028E6D0013F052F00F2B3
:10064000DA81DFE807F0030A0D101336052305935E
:10065000042105A800F032FA17E054480421F9E714
:1006600058480421F6E758480421F3E74FF01C08E6
:10067000404600F04FFA08F104080590042105A84F
:1006800000F01CFAB8F12C0FF2D1012000FA07F7A4
:1006900047EA0B0B5FFA8BFB4FF0000900F064FB9D
:1006A00026B10BF00B030B2B08BF0024FFF778FEDD
:1006B0005BE746480421CDE7002EA5D00BF00B03E5
:1006C0000B2BA1D10220FFF763FE074600289BD029
:1006D000012000F01DFA0220FFF7AAFE00261FFAF3
:1006E00086F8404600F024FA044690B100214046C6
:1006F00000F02EFA01360028F1D1BA46044641F244
:100700001213022105A8ADF814303E4600F0D6F9C8
:100710002BE70120FFF78CFE2546244B9B68AB425C
:1007200007D9284600F0F6F9013040F0678104351A
:10073000F3E7234B00251D70204BBA465D603E4613
:10074000ACE7002E3FF460AF0BF00B030B2B7FF4F4
:100750005BAF0220FFF76CFE322000F091F9B0F1A0
:100760000008FFF651AF18F003077FF44DAF0F4AB2
:10077000926808EB050393423FF646AFB8F5807FD9
:100780003FF742AF124B0193B84523DD4FF47A7027
:1007900000F076F90390039A002AFFF635AF019B2B
:1007A000039A03F8012B0137EDE700BF0022002078
:1007B0005C23002040220020B903000860230020B1
:1007C0005822002004220020082200200C220020B1
:1007D0005C220020C820FFF7DBFD074600283FF41D
:1007E00013AF1F2D11D8C5F1200242450AAB25F0E9
:1007F000030028BF424683490192184400F042FAA0
:10080000019A8048FF2100F063FA4FEAA8037D496E
:100810000193C8F38702284600F062FA06460028D2
:100820003FF46DAF019B05EB830537E70220FFF72F
:10083000AFFD00283FF4E8AE00F0B6F900283FF421
:10084000E3AE0027B846704B9B68BB4218D91F2FF8
:1008500011D80A9B01330ED027F0030312AA1344C8
:1008600053F8203C05934046042205A900F0B0FA55
:1008700004378046E7E7384600F04CF90590F2E788
:10088000CDF81480042105A800F018F906E700232C
:10089000642104A8049300F007F900287FF4B4AEA3
:1008A0000220FFF775FD00283FF4AEAE049800F07B
:1008B00063F90590E6E70023642104A8049300F09F
:1008C000F3F800287FF4A0AE0220FFF761FD0028B6
:1008D0003FF49AAE049800F05FF9EAE70220FFF7D0
:1008E00057FD00283FF490AE00F06EF9E1E70220DA
:1008F000FFF74EFD00283FF487AE05A9142000F055
:1009000069F904210746049004A800F0D7F8394695
:10091000B9E7322000F0B4F8071EFFF675AEBB074A
:100920007FF472AE384A926807EB090393423FF6B0
:100930006BAE0220FFF72CFD00283FF465AE27F0D8
:1009400003074F44B9453FF4A9AE484600F0E2F82A
:100950000421059005A800F0B1F809F10409F1E7B8
:100960004FF47A70FFF714FD00283FF44DAE00F00D
:100970001BF9002844D00A9B01330BD008220AA996
:10098000002000F0ADF900283AD02022FF210AA86B
:1009900000F09EF9FFF704FD1C4800F043FF13B080
:1009A000BDE8F08F002E3FF42FAE0BF00B030B2BA6
:1009B0007FF42AAE0023642105A8059300F074F8A3
:1009C000074600287FF420AE0220FFF7E1FC8046B6
:1009D00000283FF419AEFFF7E3FC41F2883000F045
:1009E00021FF059800F0F2F9464600F0BDF93C46BB
:1009F000BBE5064652E64FF0000905E6BA467EE63C
:100A000037467CE65C22002000220020A086010000
:100A10007047000070B50F4B1B780133DBB2012B20
:100A20000C4611D80C4D29684FF47A730E6AA2FB5C
:100A30000332014622462846B047844204D1074B80
:100A400000221A70012070BD4FF4FA7000F0EAFE27
:100A50000020F8E710220020082600209423002020
:100A600070B504464FF47A76412C254628BF4125BF
:100A700006FB05F000F0D6FE641BF5D170BD00004A
:100A800007B50023024601210DF107008DF807305C
:100A9000FFF7C0FF20B19DF8070003B05DF804FB2D
:100AA0004FF0FF30F9E700000A4608B50421FFF7D0
:100AB000B1FF80F00100C0B2404208BD30B4054C27
:100AC0002368DD69044B0A46AC460146204630BC2B
:100AD000604700BF08260020A086010070B501F025
:100AE000C1F9094E094D30800024286833888342BB
:100AF00008D901F0B1F92B6804440133B4F5404F33
:100B00002B60F2D370BD00BF962300206823002025
:100B100001F056BA00F1006000F5404000687047EF
:100B200000F10060920000F5404001F0E1B90000E2
:100B3000054B1A68054B1B889B1A834202D9104447
:100B400001F08AB900207047682300209623002016
:100B500038B5084D044629B128682044BDE838401E
:100B600001F09AB92868204401F07EF90028F3D0FA
:100B700038BD00BF6823002010F003030AD1B0F590
:100B8000047F05D200F10050A0F51040D0F80038E5
:100B9000184670470023FBE700F10050A0F5104015
:100BA000D0F8100A70470000064991F8243033B19C
:100BB0000023086A81F824300822FFF7B1BF012022
:100BC000704700BF6C230020014B1868704700BFBE
:100BD000002004E070B5194B1D68194B0138C5F3AE
:100BE0000B0408442D0C04221E88A6420BD15C681D
:100BF0000A46013C824213460FD214F9016F4EB1EE
:100C000002F8016BF6E7013A03F10803ECD18142E7
:100C10000B4602D22C2203F8012B0A4A052416881F
:100C2000AE4204D1984284BF967803F8016B013C30
:100C300002F10402F3D1581A70BD00BF002004E095
:100C40009C34000888340008022802BF024B4FF091
:100C500080729A61704700BF00000240022802BF04
:100C6000024B4FF480729A61704700BF000002404F
:100C7000022801BF024A536983F4807353617047AD
:100C80000000024010B50023934203D0CC5CC45452
:100C90000133F9E710BD000010B5013810F9013F2C
:100CA0003BB191F900409C4203D11AB10131013AA4
:100CB000F4E71AB191F90020981A10BD1046FCE72C
:100CC00003460246D01A12F9011B0029FAD17047D7
:100CD00002440346934202D003F8011BFAE770472F
:100CE0002DE9F8431F4D144695F824200746884601
:100CF00052BBDFF870909CB395F824302BB92022BA
:100D0000FF2148462F62FFF7E3FF95F82400C0F16A
:100D10000802A24228BF2246D6B24146920005EB05
:100D20008000FFF7AFFF95F82430A41B1E44F6B2F5
:100D3000082E17449044E4B285F82460DBD1FFF715
:100D400033FF0028D7D108E02B6A03EB82038342EC
:100D5000CFD0FFF729FF0028CBD10020BDE8F883D2
:100D60000120FBE76C230020024B1A78024B1A701B
:100D7000704700BF942300201022002010B5104CB3
:100D8000104800F0B5F821460E4800F0DDF8246860
:100D9000626DD2F8043843F00203C2F804384FF40D
:100DA0007A70FFF75DFE0849204600F0D3F9626DC6
:100DB000D2F8043823F00203C2F8043810BD00BF93
:100DC00068350008082600207035000870470000CC
:100DD00030B5094D0A4491420DD011F8013B5840FD
:100DE000082340F30004013B2C4013F0FF0384EA86
:100DF0005000F6D1EFE730BD2083B8ED02684368BC
:100E00001143016003B118477047000013B5446BEC
:100E1000D4F894341A681178042915D1217C022958
:100E200012D11979128901238B4013420CD101A9E7
:100E300004F14C0001F0F8FED4F89444019B2179B0
:100E40000246206800F0D0F902B010BD143001F065
:100E50007BBE00004FF0FF33143001F075BE000080
:100E60004C3001F04DBF00004FF0FF334C3001F02B
:100E700047BF0000143001F049BE00004FF0FF31C1
:100E8000143001F043BE00004C3001F019BF0000E7
:100E90004FF0FF324C3001F013BF000000207047CC
:100EA00010B5D0F894341A6811780429044617D183
:100EB000017C022914D15979528901238B401342B4
:100EC0000ED1143001F0DCFD024648B1D4F8944450
:100ED0004FF4807361792068BDE8104000F072B96A
:100EE00010BD0000406BFFF7DBBF00007047000043
:100EF0007FB5124B036000234360C0E90233012534
:100F000002260F4B057404460290019300F18402FF
:100F1000294600964FF48073143001F08DFD094B83
:100F20000294CDE9006304F523724FF480732946DF
:100F300004F14C0001F054FE04B070BDBC34000854
:100F4000E50E00080D0E00080B68302282F31188B0
:100F50000A7903EB820290614A79093243F8220050
:100F60008A7912B103EB820398610223C0F89414CA
:100F70000374002080F311887047000038B5037FA8
:100F8000044613B190F85430ABB9201D012502215D
:100F9000FFF734FF04F1140025776FF0010100F032
:100FA00069FC84F8545004F14C006FF00101BDE875
:100FB000384000F05FBC38BD10B501210446043054
:100FC000FFF71CFF0023237784F8543010BD000086
:100FD00038B504460025143001F046FD04F14C00FC
:100FE000257701F015FE201D84F854500121FFF7EC
:100FF00005FF2046BDE83840FFF752BF90F8443067
:1010000003F06003202B07D190F84520212A4FF0F0
:10101000000303D81F2A06D800207047222AFBD1DC
:10102000C0E90E3303E0034A82630722C26303640C
:10103000012070471122002037B5D0F894341A6887
:101040001178042904461AD1017C022917D1197993
:10105000128901238B40134211D100F14C0528461F
:1010600001F096FE58B101A9284601F0DDFDD4F843
:101070009444019B21790246206800F0B5F803B042
:1010800030BD0000F0B500EB810385B09E690446D9
:101090000D46FEB1302383F3118804EB8507301D24
:1010A0000821FFF7ABFEFB685B691B6806F14C008B
:1010B0001BB1019001F0C6FD019803A901F0B4FD38
:1010C000024648B1039B2946204600F08DF80023D4
:1010D00083F3118805B0F0BDFB685A691268002AD5
:1010E000F5D01B8A013B1340F1D104F14402EAE739
:1010F000093138B550F82140DCB1302383F3118831
:10110000D4F894241368527903EB8203DB689B695B
:101110005D6845B104216018FFF770FE294604F1AF
:10112000140001F0B7FC2046FFF7BAFE002383F35A
:10113000118838BD7047000001F016B80123037014
:101140000023C0E90133C36183620362C362436267
:101150000363704738B50446302383F311880025B4
:10116000C0E90355C0E90555416001F00DF80223BF
:10117000237085F31188284638BD000070B500EB58
:10118000810305465069DA600E46144618B11022F4
:101190000021FFF79DFDA06918B110220021FFF783
:1011A00097FD31462846BDE8704001F0B7B8000011
:1011B000826802F0011282600022C0E9042282618A
:1011C00001F038B9F0B400EB81044789E4680125E7
:1011D000A4698D403D43458123600023A260636084
:1011E000F0BC01F053B90000F0B400EB81040789B2
:1011F000E468012564698D403D4305812360002337
:10120000A2606360F0BC01F0CDB9000070B50223AC
:10121000002504460370C0E90255C0E90455C564C1
:10122000856180F8345001F015F863681B6823B1BC
:1012300029462046BDE87040184770BD0378052B4D
:1012400010B504460AD080F8503005230370436877
:101250001B680BB1042198470023A36010BD000058
:101260000178052906D190F85020436802701B6868
:1012700003B118477047000070B590F83430044649
:1012800013B1002380F8343004F14402204601F009
:10129000F3F863689B68B3B994F8443013F06005C1
:1012A00035D00021204601F093FB0021204601F0BB
:1012B00085FB63681B6813B1062120469847062307
:1012C00084F8343070BD204698470028E4D0B4F844
:1012D0004A30E26B9A4288BFE36394F94430E56B8D
:1012E000002B4FF0300380F20381002D00F0F280DC
:1012F000092284F8342083F311880021D4E90E23D5
:101300002046FFF771FF002383F31188DAE794F892
:10131000452003F07F0343EA022340F20232934266
:1013200000F0C58021D8B3F5807F48D00DD8012BBF
:101330003FD0022B00F09380002BB2D104F14C027D
:10134000A2630222E2632364C1E7B3F5817F00F068
:101350009B80B3F5407FA4D194F84630012BA0D1F7
:10136000B4F84C3043F0020332E0B3F5006F4DD0D7
:1013700017D8B3F5A06F31D0A3F5C063012B90D877
:10138000636894F846205E6894F84710B4F84830D3
:101390002046B047002884D04368A3630368E36312
:1013A0001AE0B3F5106F36D040F6024293427FF454
:1013B00078AF5C4BA3630223E3630023C3E794F895
:1013C0004630012B7FF46DAFB4F84C3023F00203AC
:1013D000C4E90E55A4F84C30256478E7B4F84430DD
:1013E000B3F5A06F0ED194F8463084F84E30204605
:1013F00000F088FF63681B6813B1012120469847FD
:10140000032323700023C4E90E339CE704F14F0348
:10141000A3630123C3E72378042B10D1302383F384
:1014200011882046FFF7C4FE85F311880321636805
:1014300084F84F5021701B680BB12046984794F8F0
:101440004630002BDED084F84F30042323706368CD
:101450001B68002BD6D0022120469847D2E794F88B
:1014600048301D0603F00F0120460AD500F0F6FFB4
:10147000012804D002287FF414AF2B4B9AE72B4BA2
:1014800098E700F0DDFFF3E794F84630002B7FF497
:1014900008AF94F8483013F00F01B3D01A06204675
:1014A00002D501F0A9FAADE701F09CFAAAE794F899
:1014B0004630002B7FF4F5AE94F8483013F00F015E
:1014C000A0D01B06204602D501F082FA9AE701F06F
:1014D00075FA97E7142284F8342083F311882B4699
:1014E0002A4629462046FFF76DFE85F31188E9E676
:1014F0005DB1152284F8342083F311880021D4E9EA
:101500000E232046FFF75EFEFDE60B2284F8342012
:1015100083F311882B462A4629462046FFF764FEAE
:10152000E3E700BFEC340008E4340008E8340008C6
:1015300038B590F834300446002B3ED0063BDAB282
:101540000F2A34D80F2B32D8DFE803F037313108B7
:10155000223231313131313131313737C56BB0F869
:101560004A309D4214D2C3681B8AB5FBF3F203FBD9
:1015700012556DB9302383F311882B462A4629462C
:10158000FFF732FE85F311880A2384F834300EE029
:10159000142384F83430302383F3118800231A464F
:1015A00019462046FFF70EFE002383F3118838BD4D
:1015B000036C03B198470023E7E70021204601F0C0
:1015C00007FA0021204601F0F9F963681B6813B19E
:1015D0000621204698470623D7E7000010B590F86B
:1015E0003430142B044629D017D8062B05D001D847
:1015F0001BB110BD093B022BFBD80021204601F096
:10160000E7F90021204601F0D9F963681B6813B19E
:10161000062120469847062319E0152BE9D10B2314
:1016200080F83430302383F3118800231A4619469A
:10163000FFF7DAFD002383F31188DAE7C3689B69BB
:101640005B68002BD5D1036C03B19847002384F865
:101650003430CEE700230375826803691B689968FC
:101660009142FBD25A680360426010605860704734
:1016700000230375826803691B6899689142FBD84F
:101680005A680360426010605860704708B50846A9
:10169000302383F311880B7D032B05D0042B0DD051
:1016A0002BB983F3118808BD8B6900221A604FF0B3
:1016B000FF338361FFF7CEFF0023F2E7D1E9003269
:1016C00013605A60F3E70000FFF7C4BF054BD96809
:1016D0000875186802681A60536001220275D860A4
:1016E000FEF710BE9823002030B50C4BDD684B1C74
:1016F00087B004460FD02B46094A684600F04EF9E1
:101700002046FFF7E3FF009B13B1684600F050F955
:10171000A86907B030BDFFF7D9FFF9E7982300208B
:101720008D160008044B1A68DB6890689B68984225
:1017300094BF00200120704798230020084B10B56B
:101740001C68D86822681A60536001222275DC6028
:10175000FFF78EFF01462046BDE81040FEF7D2BDE0
:101760009823002038B5074C074908480123002575
:101770002370656001F044FB0223237085F3118818
:1017800038BD00BF00260020F43400089823002054
:1017900000F044B9034A516853685B1A9842FBD879
:1017A000704700BF001000E08B60022308618B824D
:1017B000084670478368A3F1840243F8142C026939
:1017C00043F8442C426943F8402C094A43F8242C3E
:1017D000C26843F8182C022203F80C2C002203F8EC
:1017E0000B2C044A43F8102CA3F12000704700BFD3
:1017F0001D0300089823002008B5FFF7DBFFBDE8B4
:101800000840FFF761BF0000024BDB6898610F20C2
:10181000FFF75CBF98230020302383F31188FFF784
:10182000F3BF000008B50146302383F31188082078
:10183000FFF75AFF002383F3118808BD064BDB68CE
:1018400039B1426818605A60136043600420FFF7A2
:101850004BBF4FF0FF307047982300200368984239
:1018600006D01A680260506099611846FFF72CBFD5
:101870007047000038B504460D462068844200D108
:1018800038BD036823605C608561FFF71DFFF4E7E6
:1018900010B503689C68A2420CD85C688A600B6033
:1018A0004C602160596099688A1A9A604FF0FF3342
:1018B000836010BD1B68121BECE700000A2938BFCB
:1018C0000A2170B504460D460A26601901F092FA05
:1018D00001F07EFA041BA54203D8751C2E4604466F
:1018E000F3E70A2E04D9BDE87040012001F0C8BA20
:1018F00070BD0000F8B5144B0D46D96103F110011D
:1019000041600A2A1969826038BF0A220160486072
:101910001861A818144601F05FFA0A2701F058FA76
:10192000431BA342064606D37C1C281901F062FA29
:1019300027463546F2E70A2F04D9BDE8F8400120D2
:1019400001F09EBAF8BD00BF98230020F8B5064606
:101950000D4601F03DFA0F4A134653F8107F9F429F
:1019600006D12A4601463046BDE8F840FFF7C2BF1F
:10197000D169BB68441A2C1928BF2C46A34202D94E
:101980002946FFF79BFF224631460348BDE8F84051
:10199000FFF77EBF98230020A823002010B4C0E9E1
:1019A000032300235DF8044B4361FFF7CFBF000022
:1019B00010B5194C236998420DD0D0E900328168E6
:1019C00013605A609A680A449A60002303604FF0DB
:1019D000FF33A36110BD2346026843F8102F536004
:1019E0000022026022699A4203D1BDE8104001F052
:1019F000FBB9936881680B44936001F0E9F92269AF
:101A0000E1699268441AA242E4D91144BDE8104049
:101A1000091AFFF753BF00BF982300202DE9F047B4
:101A2000DFF8BC8008F110072C4ED8F8105001F0F8
:101A3000CFF9D8F81C40AA68031B9A423ED8144438
:101A4000D5E900324FF00009C8F81C4013605A6015
:101A5000C5F80090D8F81030B34201D101F0C4F9B4
:101A600089F31188D5E9033128469847302383F359
:101A700011886B69002BD8D001F0AAF96A69A0EB34
:101A800004094A4582460DD2022001F0F9F90022EC
:101A9000D8F81030B34208D151462846BDE8F04787
:101AA000FFF728BF121A2244F2E712EB090938BFE8
:101AB0004A4629463846FFF7EBFEB5E7D8F810301E
:101AC000B34208D01444211AC8F81C00A960BDE82C
:101AD000F047FFF7F3BEBDE8F08700BFA823002062
:101AE0009823002000207047FEE7000070470000A8
:101AF0004FF0FF307047000002290CD0032904D0BA
:101B00000129074818BF00207047032A05D8054857
:101B100000EBC2007047044870470020704700BFC8
:101B2000CC350008202200208035000870B59AB01E
:101B30000546084601A9144600F0C2F801A8FFF7BF
:101B4000BFF8431C5B00C5E9003400222370032367
:101B50006370C6B201AB02341046D1B28E4204F1BA
:101B6000020401D81AB070BD13F8011B04F8021C5E
:101B700004F8010C0132F0E708B5302383F3118833
:101B80000348FFF759FA002383F3118808BD00BF0B
:101B90000826002090F8443003F01F02012A07D1E4
:101BA00090F845200B2A03D10023C0E90E3315E03D
:101BB00003F06003202B08D1B0F848302BB990F81F
:101BC0004520212A03D81F2A04D8FFF717BA222A52
:101BD000EBD0FAE7034A82630722C2630364012061
:101BE000704700BF1822002007B5052917D8DFE885
:101BF00001F0191603191920302383F31188104AB4
:101C000001900121FFF7BAFA01980E4A0221FFF76D
:101C1000B5FA0D48FFF7DCF9002383F3118803B010
:101C20005DF804FB302383F311880748FFF7A6F91A
:101C3000F2E7302383F311880348FFF7BDF9EBE7A0
:101C400020350008443500080826002038B50C4D22
:101C50000C4C0D492A4604F10800FFF767FF05F117
:101C6000CA0204F110000949FFF760FF05F5CA72C6
:101C700004F118000649BDE83840FFF757BF00BF20
:101C8000D02A002020220020003500080A35000854
:101C90001535000870B5044608460D46FFF710F8E4
:101CA000C6B22046013403780BB9184670BD3246DF
:101CB0002946FEF7F1FF0028F3D10120F6E70000E6
:101CC0002DE9F04705460C46FEF7FAFF2B49C6B250
:101CD0002846FFF7DFFF08B10636F6B22849284646
:101CE000FFF7D8FF08B11036F6B2632E0BD8DFF835
:101CF0008C80DFF88C90234FDFF894A02E7846B9C3
:101D00002670BDE8F08729462046BDE8F04701F07F
:101D10009DBB252E2ED1072241462846FEF7BCFF4B
:101D200070B9194B224603F10C0153F8040B42F829
:101D3000040B8B42F9D11B78137007350D34DDE7A6
:101D4000082249462846FEF7A7FF98B90F4BA21C68
:101D5000197809090232C95D02F8041C13F8011B45
:101D600001F00F015345C95D02F8031CF0D118348E
:101D70000835C3E704F8016B0135BFE7EC3500080F
:101D80001535000802360008F4350008107AFF1FE8
:101D90001C7AFF1FBFF34F8F024AD368DB03FCD4CA
:101DA000704700BF003C024008B5094B1B7873B96F
:101DB000FFF7F0FF074B1A69002ABFBF064A5A60B7
:101DC00002F188325A601A6822F480621A6008BDF3
:101DD0002E2D0020003C02402301674508B50B4B27
:101DE0001B7893B9FFF7D6FF094B1A6942F00042FE
:101DF0001A611A6842F480521A601A6822F48052FA
:101E00001A601A6842F480621A6008BD2E2D002004
:101E1000003C02400B28F0B516D80C4C0C49237836
:101E20007BB90C4D0E460C234FF0006255F8047B35
:101E300046F8042B013B13F0FF033A44F6D101238B
:101E4000237051F82000F0BD0020FCE7602D002039
:101E5000302D002014360008014B53F82000704745
:101E6000143600080C2070470B2810B5044601D921
:101E7000002010BDFFF7CEFF064B53F82430184466
:101E8000C21A0BB90120F4E712680132F0D1043B09
:101E9000F6E700BF143600080B2810B5044621D819
:101EA000FFF778FFFFF780FF0F4AF323D360C300EB
:101EB000DBB243F4007343F002031361136943F48C
:101EC00080331361FFF766FFFFF7A4FF074B53F85A
:101ED000241000F0D9F8FFF781FF2046BDE810403C
:101EE000FFF7C2BF002010BD003C024014360008BE
:101EF000F8B512F00103144642D18218B2F1016F15
:101F000057D82D4B1B6813F0010352D02B4DFFF710
:101F10004BFFF323EB60FFF73DFF40F20127032C5B
:101F200015D824F001046618244C401A40F2011719
:101F3000B142236900EB010524D123F001032361A1
:101F4000FFF74CFF0120F8BD043C0430E7E78307AE
:101F5000E7D12B6923F440732B612B693B432B6141
:101F600051F8046B0660BFF34F8FFFF713FF036850
:101F70009E42E9D02B6923F001032B61FFF72EFF6E
:101F80000020E0E723F44073236123693B4323618E
:101F90000B882B80BFF34F8FFFF7FCFE2D8831F8A5
:101FA000023BADB2AB42C3D0236923F001032361EE
:101FB000E4E71846C7E700BF00380240003C024093
:101FC000084908B50B7828B11BB9FFF7EDFE0123CE
:101FD0000B7008BD002BFCD0BDE808400870FFF76F
:101FE000FDBE00BF2E2D002010B50244064BD2B21C
:101FF000904200D110BD441C00B253F8200041F8BB
:10200000040BE0B2F4E700BF502800400F4B30B59E
:102010001C6F240407D41C6F44F400741C671C6FED
:1020200044F400441C670A4C236843F48073236023
:102030000244084BD2B2904200D130BD441C00B2E1
:1020400051F8045B43F82050E0B2F4E70038024056
:10205000007000405028004007B5012201A900206F
:10206000FFF7C2FF019803B05DF804FB13B5044607
:10207000FFF7F2FFA04205D0012201A90020019440
:10208000FFF7C4FF02B010BD70470000034B1A6891
:102090001AB9034AD2F874281A607047642D0020D8
:1020A0000030024008B5FFF7F1FF024B1868C0F39B
:1020B000407008BD642D002070470000FEE700005E
:1020C0000A4B0B480B4A90420BD30B4BDA1C121AEB
:1020D000C11E22F003028B4238BF00220021FEF70E
:1020E000F7BD53F8041B40F8041BECE7C0370008A9
:1020F000602E0020602E0020602E002070B5D0E9F8
:1021000015439E6800224FF0FF3504EB4213510146
:10211000D3F800090028BEBFD3F8000940F0804082
:10212000C3F80009D3F8000B0028BEBFD3F8000B9A
:1021300040F08040C3F8000B013263189642C3F8A8
:102140000859C3F8085BE0D24FF00113C4F81C38FB
:1021500070BD0000890141F02001016103699B0607
:10216000FCD41220FFF716BB10B5054C2046FEF735
:10217000E5FF4FF0A0436365024BA36510BD00BFB0
:10218000682D00206836000870B50378012B0546DD
:1021900050D12A4B446D98421BD1294B5A6B42F0C7
:1021A00080025A635A6D42F080025A655A6D5A692C
:1021B00042F080025A615A6922F080025A610E216F
:1021C00043205B6900F022FC1E4BE3601E4BC4F809
:1021D00000380023C4F8003EC02323606E6D4FF426
:1021E0000413A3633369002BFCDA012333610C2051
:1021F000FFF7D0FA3369DB07FCD41220FFF7CAFAE5
:102200003369002BFCDA0026A6602846FFF776FF2C
:102210006B68C4F81068DB68C4F81468C4F81C68FC
:102220004BB90A4BA3614FF0FF336361A36843F0DE
:102230000103A36070BD064BF4E700BF682D0020CA
:10224000003802404014004003002002003C30C02F
:10225000083C30C0F8B5446D054600212046FFF724
:1022600079FFA96D00234FF001128F68C4F834384C
:102270004FF00066C4F81C284FF0FF3004EB431207
:1022800001339F42C2F80069C2F8006BC2F8080926
:10229000C2F8080BF2D20B686A6DEB65636210231B
:1022A0001361166916F01006FBD11220FFF772FABF
:1022B000D4F8003823F4FE63C4F80038A36943F46B
:1022C000402343F01003A3610923C4F81038C4F875
:1022D00014380A4BEB604FF0C043C4F8103B084B76
:1022E000C4F8003BC4F81069C4F80039EB6D03F181
:1022F000100243F48013EA65A362F8BD4436000877
:1023000040800010426D90F84E10D2F8003823F44F
:10231000FE6343EA0113C2F8003870472DE9F84321
:1023200000EB8103456DDA68166806F00306731E3C
:10233000022B05EB41130C4680460FFA81F94FEA58
:1023400041104FF00001C3F8101B4FF0010104F1E0
:10235000100398BFB60401FA03F391698EBF334EA0
:1023600006F1805606F5004600293AD0578A04F156
:102370005801490137436F50D5F81C180B43C5F875
:102380001C382B180021C3F8101953690127611E4E
:10239000A7409BB3138A928B9B08012A88BF5343A3
:1023A000D8F85C20981842EA034301F1400205EB9B
:1023B0008202C8F85C00214653602846FFF7CAFE37
:1023C00008EB8900C3681B8A43EA845348346401DC
:1023D0001E432E51D5F81C381F43C5F81C78BDE8A4
:1023E000F88305EB4917D7F8001B21F40041C7F823
:1023F000001BD5F81C1821EA0303C0E704F13F03D2
:1024000005EB83030A4A5A6028462146FFF7A2FEDD
:1024100005EB4910D0F8003923F40043C0F8003927
:10242000D5F81C3823EA0707D7E700BF0080001063
:1024300000040002826D1268C265FFF75FBE0000F3
:102440005831436D49015B5813F4004004D013F434
:10245000001F0CBF02200120704700004831436D6F
:1024600049015B5813F4004004D013F4001F0CBF63
:10247000022001207047000000EB8101CB68196A3F
:102480000B6813604B6853607047000000EB8103DA
:1024900030B5DD68AA691368D36019B9402B84BFD1
:1024A000402313606B8A1468426D1C44013CB4FBEA
:1024B000F3F46343033323F0030302EB411043EAD5
:1024C000C44343F0C043C0F8103B2B6803F0030340
:1024D000012B09B20ED1D2F8083802EB411013F4E7
:1024E000807FD0F8003B14BF43F0805343F000538B
:1024F000C0F8003B02EB4112D2F8003B43F004432A
:10250000C2F8003B30BD00002DE9F041244D6E6D56
:1025100006EB40130446D3F8087BC3F8087B380762
:102520000AD5D6F81438190706D505EB84032146D9
:10253000DB6828465B689847FA071FD5D6F8143839
:10254000DB071BD505EB8403D968CCB98B69488AB6
:102550005A68B2FBF0F600FB16228AB91868DA68EE
:1025600090420DD2121AC3E90024302383F311885C
:102570000B482146FFF78AFF84F31188BDE8F081FC
:10258000012303FA04F26B8923EA02036B81CB680F
:10259000002BF3D021460248BDE8F041184700BFA8
:1025A000682D002000EB810370B5DD68436D6C6918
:1025B0002668E6604A0156BB1A444FF40020C2F870
:1025C00010092A6802F00302012A0AB20ED1D3F8D8
:1025D000080803EB421410F4807FD4F8000914BFFC
:1025E00040F0805040F00050C4F8000903EB421264
:1025F000D2F8000940F00440C2F80009D3F83408CA
:10260000012202FA01F10143C3F8341870BD19B96F
:10261000402E84BF4020206020682E8A8419013C0F
:10262000B4FBF6F440EAC44040F000501A44C6E758
:102630002DE9F8433B4D6E6D06EB40130446D3F88D
:102640000889C3F8088918F0010F4FEA40171AD01B
:10265000D6F81038DB0716D505EB8003D9684B692F
:102660001868DA68904230D2121A4FF000091A60E6
:10267000C3F80490302383F3118821462846FFF7DE
:1026800091FF89F3118818F0800F1CD0D6F83438E8
:102690000126A640334216D005EB84036D6DD3F8B6
:1026A0000CC0DCF814200134E4B2D2F800E005EBF1
:1026B00004342F445168714515D3D5F8343823EAD2
:1026C0000606C5F83468BDE8F883012303FA04F26E
:1026D0002B8923EA02032B818B68002BD3D0214660
:1026E00028469847CFE7BCF81000AEEB01038342C1
:1026F00028BF0346D7F8180980B2B3EB800FE2D8A1
:102700009068A0F1040959F8048FC4F80080A0EB88
:1027100009089844B8F1040FF5D818440B449060A8
:102720005360C7E7682D00202DE9F74FA24C656D77
:102730006E69AB691E4016F480586E6107D0204662
:10274000FEF764FD03B0BDE8F04F00F047BC002E7B
:1027500012DAD5F8003E98489B071EBFD5F8003E18
:1027600023F00303C5F8003ED5F8043823F0010335
:10277000C5F80438FEF774FD370505D58E48FFF718
:10278000BDFC8D48FEF75AFDB0040CD5D5F80838CD
:1027900013F0060FEB6823F470530CBF43F410538F
:1027A00043F4A053EB6031071BD56368DB681BB9AA
:1027B000AB6923F00803AB612378052B0CD1D5F866
:1027C000003E7D489A071EBFD5F8003E23F0030364
:1027D000C5F8003EFEF744FD6368DB680BB1764840
:1027E0009847F30274D4B70227D5D4F85490DFF891
:1027F000C8B100274FF0010A09EB4712D2F8003B9D
:1028000003F44023B3F5802F11D1D2F8003B002B05
:102810000DDA62890AFA07F322EA0303638104EB03
:102820008703DB68DB6813B1394658469847A36DC8
:1028300001379B68FFB29F42DED9F00617D5676D5E
:102840003A6AC2F30A1002F00F0302F4F012B2F572
:10285000802F00F08580B2F5402F08D104EB830370
:102860000022DB681B6A07F5805790426AD130036B
:10287000D5F8184813D5E10302D50020FFF744FE30
:10288000A20302D50120FFF73FFE630302D5022019
:10289000FFF73AFE270302D50320FFF735FE750345
:1028A0007FF550AFE00702D50020FFF7C1FEA1077A
:1028B00002D50120FFF7BCFE620702D50220FFF718
:1028C000B7FE23077FF53EAF0320FFF7B1FE39E7E0
:1028D000636DDFF8E4A0019300274FF00109A36DB9
:1028E0009B685FFA87FB9B453FF67DAF019B03EB3F
:1028F0004B13D3F8001901F44021B1F5802F1FD1FB
:10290000D3F8001900291BDAD3F8001941F09041DF
:10291000C3F80019D3F800190029FBDB5946606D94
:10292000FFF718FC218909FA0BF321EA030323813D
:1029300004EB8B03DB689B6813B1594650469847FC
:102940000137CCE7910708BFD7F80080072A98BF66
:1029500003F8018B02F1010298BF4FEA182884E7BF
:10296000023304EB830207F580575268D2F818C08F
:10297000DCF80820DCE9001CA1EB0C0C00218842EB
:102980000AD104EB830463689B699A6802449A60E5
:102990005A6802445A606AE711F0030F08BFD7F87B
:1029A00000808C4588BF02F8018B01F1010188BFCE
:1029B0004FEA1828E3E700BF682D0020436D03EBC2
:1029C0004111D1F8003B43F40013C1F8003B7047BC
:1029D000436D03EB4111D1F8003943F40013C1F802
:1029E00000397047436D03EB4111D1F8003B23F4EC
:1029F0000013C1F8003B7047436D03EB4111D1F860
:102A0000003923F40013C1F80039704700F1604326
:102A100003F561430901C9B283F80013012200F0F4
:102A20001F039A4043099B0003F1604303F5614390
:102A3000C3F880211A60704730B5039C01720433DB
:102A400004FB0325C0E90653049B03630021059B97
:102A5000C160C0E90000C0E90422C0E90842C0E941
:102A60000A11436330BD0000416A0022C0E904112D
:102A7000C0E90A22C2606FF00101FEF7FBBE000050
:102A8000D0E90432934201D1C2680AB9181D7047D7
:102A90000020704703691960C2680132C260C269D0
:102AA000134482690361934224BF436A0361002196
:102AB000FEF7D4BE38B504460D46E3683BB1626903
:102AC000131D1268A3621344E362002007E0237A17
:102AD00033B929462046FEF7B1FE0028EDDA38BDAD
:102AE0006FF00100FBE70000C368C269013BC360EF
:102AF0004369134482694361934224BF436A43613B
:102B000000238362036B03B11847704770B530230D
:102B1000044683F31188866A3EB9FFF7CBFF05466A
:102B200018B186F31188284670BDA36AE26A13F8CB
:102B3000015BA362934202D32046FFF7D5FF002337
:102B400083F31188EFE700002DE9F84F04460E46A5
:102B5000174698464FF0300989F311880025AA4698
:102B6000D4F828B0BBF1000F09D141462046FFF749
:102B7000A1FF20B18BF311882846BDE8F88FD4E976
:102B80000A12A7EB050B521A934528BF9346BBF1D7
:102B9000400F1BD9334601F1400251F8040B43F8B2
:102BA000040B9142F9D1A36A40334036A362403509
:102BB000D4E90A239A4202D32046FFF795FF8AF30D
:102BC0001188BD42D8D289F31188C9E730465A46E8
:102BD000FEF758F8A36A5B445E44A3625D44E7E7EE
:102BE00010B5029C0172043303FB0421C0E90613F3
:102BF0000023C0E90A33039B0363049BC460C0E95C
:102C00000000C0E90422C0E90842436310BD00008F
:102C1000026AC260426AC0E904220022C0E90A22B4
:102C20006FF00101FEF726BED0E904239A4201D1DC
:102C3000C26822B9184650F8043B0B607047002365
:102C40001846FAE7C368C2690133C3604369134495
:102C500082694361934224BF436A43610021FEF7C6
:102C6000FDBD000038B504460D46E3683BB123695D
:102C70001A1DA262E2691344E362002007E0237A8E
:102C800033B929462046FEF7D9FD0028EDDA38BDD4
:102C90006FF00100FBE7000003691960C268013AA8
:102CA000C260C269134482690361934224BF436ACC
:102CB000036100238362036B03B118477047000070
:102CC00070B530230D460446114683F31188866A99
:102CD0002EB9FFF7C7FF10B186F3118870BDA36A44
:102CE0001D70A36AE26A01339342A36204D3E169CF
:102CF00020460439FFF7D0FF002080F31188EDE76C
:102D00002DE9F84F04460D46904699464FF0300A9B
:102D10008AF311880026B346A76A4FB94946204670
:102D2000FFF7A0FF20B187F311883046BDE8F88F88
:102D3000D4E90A073A1AA8EB0607974228BF1746B4
:102D4000402F1BD905F1400355F8042B40F8042B04
:102D50009D42F9D1A36A4033A3624036D4E90A23E5
:102D60009A4204D3E16920460439FFF795FF8BF3BB
:102D700011884645D9D28AF31188CDE729463A46CB
:102D8000FDF780FFA36A3B443D44A3623E44E5E770
:102D9000D0E904239A4217D1C3689BB1836A8BB1EF
:102DA000043B9B1A0ED01360C368013BC360C36928
:102DB0001A44836902619A4224BF436A0361002373
:102DC00083620123184670470023FBE700F030B907
:102DD0004FF08043586A70474FF080430022586399
:102DE0001A610222DA6070474FF080430022DA60F5
:102DF000704700004FF0804358637047FEE70000C3
:102E000070B51B4B01630025044686B0586085628F
:102E10000E4600F0BFF804F11003C4E904334FF08C
:102E2000FF33C4E90635C4E90044A560E562FFF755
:102E3000CFFF2B460246C4E9082304F134010D4AB2
:102E4000256580232046FEF7AFFC0123E0600A4A97
:102E50000375009272680192B268CDE90223074BB4
:102E60006846CDE90435FEF7C7FC06B070BD00BF6B
:102E7000002600207436000879360008FD2D000871
:102E8000024AD36A1843D062704700BF98230020DB
:102E90004B6843608B688360CB68C3600B69436198
:102EA0004B6903628B6943620B68036070470000E3
:102EB00008B5264B26481A6940F2FF110A431A61E9
:102EC0001A6922F4FF7222F001021A611A691A6B60
:102ED0000A431A631A6D0A431A651E4A1B6D11468E
:102EE000FFF7D6FF02F11C0100F58060FFF7D0FF6D
:102EF00002F1380100F58060FFF7CAFF02F15401CA
:102F000000F58060FFF7C4FF02F1700100F58060FA
:102F1000FFF7BEFF02F18C0100F58060FFF7B8FFFC
:102F200002F1A80100F58060FFF7B2FF02F1C401D1
:102F300000F58060FFF7ACFF02F1E00100F5806072
:102F4000FFF7A6FFBDE8084000F0EEB800380240E9
:102F5000000002408036000808B500F059FAFEF77C
:102F600001FCFFF793F8BDE80840FEF76FBE0000D4
:102F700070470000EFF3098305494A6B22F0010214
:102F80004A63683383F30988002383F31188704709
:102F900000EF00E0302080F3118862B60C4B0D4A40
:102FA000D96821F4E0610904090C0A43DA60D3F816
:102FB000FC20094942F08072C3F8FC200A6842F004
:102FC00001020A602022DA7783F82200704700BFEE
:102FD00000ED00E00003FA05001000E010B530231A
:102FE00083F311880E4B5B6813F4006314D0F1EE89
:102FF000103AEFF30984683C4FF08073E361094BAA
:10300000DB6B236684F30988FEF78CFB10B1064B5B
:10301000A36110BD054BFBE783F31188F9E700BFFF
:1030200000ED00E000EF00E02F030008320300088D
:103030000F4B1A6C42F001021A641A6E42F0010240
:103040001A660C4A1B6E936843F0010393604FF0BD
:10305000804353229A624FF0FF32DA6200229A6173
:103060005A63DA605A6001225A611A60704700BFE1
:1030700000380240002004E04FF0804208B511699A
:10308000D3680B40D9B2C9439B07116107D53023E0
:1030900083F31188FEF77CFB002383F3118808BDBE
:1030A0001F4B1A696FEAC2526FEAD2521A611A694B
:1030B000C2F308021A614FF0FF301A695A69586169
:1030C00000215A6959615A691A6A62F080521A627B
:1030D0001A6A02F080521A621A6A5A6A58625A6A66
:1030E00059625A6A1A6C42F080521A641A6E42F09F
:1030F00080521A661A6E0B4A106840F48070106095
:10310000186F00F44070B0F5007F1EBF4FF48030A0
:1031100018671967536823F40073536000F054B9BB
:103120000038024000700040334B4FF080521A6468
:10313000324A4FF4404111601A6842F001021A60AD
:103140001A689107FCD59A6822F003029A602A4B0C
:103150009A6812F00C02FBD1196801F0F9011960AC
:103160009A601A6842F480321A601A689203FCD599
:103170005A6F42F001025A671F4B5A6F9007FCD5F5
:103180001F4A5A601A6842F080721A601B4A5368DC
:103190005904FCD5184B1A689201FCD5194A9A605B
:1031A000194B1A68194B9A42194B21D1194A1168C7
:1031B000194A91421CD140F205121A60144A136850
:1031C00003F00F03052BFAD10B4B9A6842F0020271
:1031D0009A609A6802F00C02082AFAD15A6C42F4FA
:1031E00080425A645A6E42F480425A665B6E70475F
:1031F00040F20572E1E700BF003802400070004075
:103200000854400700948838002004E0116400202E
:10321000003C024000ED00E041C20F41074A08B502
:10322000536903F00103536123B1054A13680BB1DD
:1032300050689847BDE80840FFF7D0BE003C014009
:10324000E02D0020074A08B5536903F002035361DB
:1032500023B1054A93680BB1D0689847BDE8084090
:10326000FFF7BCBE003C0140E02D0020074A08B536
:10327000536903F00403536123B1054A13690BB189
:1032800050699847BDE80840FFF7A8BE003C0140E0
:10329000E02D0020074A08B5536903F00803536185
:1032A00023B1054A93690BB1D0699847BDE808403E
:1032B000FFF794BE003C0140E02D0020074A08B50E
:1032C000536903F01003536123B1054A136A0BB12C
:1032D000506A9847BDE80840FFF780BE003C0140B7
:1032E000E02D0020164B10B55C6904F478725A6129
:1032F000A30604D5134A936A0BB1D06A98476006B7
:1033000004D5104A136B0BB1506B9847210604D5B6
:103310000C4A936B0BB1D06B9847E20504D5094A70
:10332000136C0BB1506C9847A30504D5054A936CF8
:103330000BB1D06C9847BDE81040FFF74FBE00BFFF
:10334000003C0140E02D0020194B10B55C6904F4ED
:103350007C425A61620504D5164A136D0BB1506D5B
:103360009847230504D5134A936D0BB1D06D984748
:10337000E00404D50F4A136E0BB1506E9847A104B8
:1033800004D50C4A936E0BB1D06E9847620404D5F5
:10339000084A136F0BB1506F9847230404D5054AB0
:1033A000936F0BB1D06F9847BDE81040FFF716BE82
:1033B000003C0140E02D002008B5FFF75DFEBDE8B0
:1033C0000840FFF70BBE0000062108B50846FFF7CE
:1033D0001DFB06210720FFF719FB06210820FFF738
:1033E00015FB06210920FFF711FB06210A20FFF734
:1033F0000DFB06211720FFF709FB06212820FFF708
:1034000005FBBDE8084007211C20FFF7FFBA0000BC
:1034100008B5FFF745FE00F00BF8FDF78DFEFDF750
:1034200065FDFFF7A5FDBDE80840FFF7CFBC000034
:103430000023054A19460133102BC2E9001102F19D
:103440000802F8D1704700BFE02D0020034611F8B4
:10345000012B03F8012B002AF9D1704753544D3347
:1034600032463F3F3F0053544D33324634307800AC
:1034700053544D3332463432780053544D33324630
:103480003434365858000000012033000010410049
:1034900001105A000310590007103100000000000D
:1034A0005C340008130400006634000819040000AE
:1034B00070340008210400007A3400080000000085
:1034C000690E0008550E0008910E00087D0E0008D8
:1034D000890E0008750E0008610E00084D0E0008E8
:1034E0009D0E000800000000010000000000000028
:1034F00063300000F0340008F02300200026002094
:103500004172647550696C6F740025424F4152449A
:10351000252D424C002553455249414C25000000C1
:10352000020000000000000085100008F1100008F3
:1035300040004000A02A0020B02A00200200000025
:10354000000000000300000000000000351100082A
:103550000000000010000000C02A00200000000051
:103560000100000000000000682D002001010200A1
:10357000E91B0008F91A0008951B0008791B0008D0
:10358000430000008835000809024300020100C022
:1035900032090400000102020100052400100105A7
:1035A000240100010424020205240600010705820B
:1035B000030800FF09040100020A000000070501DA
:1035C00002400000070581024000000012000000D8
:1035D000D4350008120110010200004009124157C1
:1035E00000020102030100000403090425424F41C7
:1035F000524425007370656564796265656634764A
:10360000340030313233343536373839414243446F
:10361000454600000040000000400000004000005F
:103620000040000000000100000002000000020055
:103630000000020000000200000002000000020082
:103640000000020000000000791200083115000897
:10365000DD15000840004000C82D0020C82D0020C6
:1036600001000000D82D0020800000004001000073
:10367000030000006D61696E0069646C6500000004
:103680000001812A00000000AAAAAAAA00010024C1
:10369000FFFE00000000000000A00A000000000182
:1036A00000000000AAAAAAAA00000001FFFF000073
:1036B00000000000000000000000001000000000FA
:1036C000AAAAAAAA00000010FFFF00000000000044
:1036D000000000000000000000000000AAAAAAAA42
:1036E00000000000FFFF00000000000000000000DC
:1036F0000000000000000000AAAAAAAA0000000022
:10370000FFFF0000000000000000000000000000BB
:1037100000000000AAAAAAAA00000000FFFF000003
:103720000000000000000000000000000000000099
:10373000AAAAAAAA00000000FFFF000000000000E3
:103740000000000000000000000000000A0000006F
:103750000000000003000000000000000000000066
:103760000000000000000000000000000000000059
:103770000000000000000000000000000000000049
:10378000700400000000000000400F000000000076
:10379000FF009600000000080096000000000800EE
:1037A00004000000E83500080000000000000000F0
:1037B0000000000000000000000000000000000009
:1037C000FFFFFFFFFFFFFFFFFFFFFFFFFFFFFFFF09
:1037D000FFFFFFFFFFFFFFFFFFFFFFFFFFFFFFFFF9
:1037E000FFFFFFFFFFFFFFFFFFFFFFFFFFFFFFFFE9
:10C0000000060020B5D20008B91109081511090869
:10C0100081110908151109084D110908B7D2000846
:10C02000B7D20008B7D20008B7D2000871350B08A4
:10C03000B7D20008B7D20008B7D20008B7D20008BC
:10C04000B7D20008B7D20008B7D20008B7D20008AC
:10C05000B7D20008B7D2000809410B0831410B08DC
:10C0600059410B0881410B08A9410B08B9E80A089E
:10C07000E1E80A080DE90A0839E90A0865E90A0849
:10C080008DE90A08B9E90A083DE80A08B7D20008AC
:10C09000B7D20008B7D20008B7D20008D1410B08C8
:10C0A0001D430B0821430B0835430B0839430B088C
:10C0B0003D430B0851430B0865430B0845EF0A0845
:10C0C000EDF00A08B7D20008B7D20008B7D20008CE
:10C0D000B7D20008A5420B08B9420B08CD420B08A5
:10C0E00035420B08B7D20008B7D2000889430B08C5
:10C0F0008D430B08A1430B08A5430B08E5E90A088B
:10C10000B7D20008B7D2000879430B08B7D20008AD
:10C11000E1420B08F5420B08B7D20008B7D200087D
:10C1200011EA0A0839EA0A0865EA0A0891EA0A08DF
:10C13000BDEA0A08B7D20008B7D20008B7D2000893
:10C14000B7D20008B7D20008B7D200089D3C0B0850
:10C15000E5EA0A0811EB0A083DEB0A0809430B0857
:10C16000B7D20008B7D20008B7D20008B7D200088B
:10C17000B7D20008B7D20008B7D20008B7D200087B
:10C18000B7D20008B7D20008B7D20008B7D200086B
:10C19000B7D20008B7D20008B7D20008B7D200085B
:10C1A000B7D20008B7D20008B7D20008B7D200084B
:10C1B000B7D20008B7D20008B7D20008B7D200083B
:10C1C000B7D20008B7D20008B7D20008B7D200082B
:10C1D000B7D20008B7D20008B7D20008B7D200081B
:10C1E000551801081143020839B10308896C050884
:10C1F000AD72050861D10508E5340608A93C0608BA
:10C20000E13F060841A506085DCC0608CDA1070858
:10C21000BDFC0708150A0808B10209083508090815
:10C2200039C20908A11D0A0879440A08015B0A08F5
:10C23000AD880A08758E0A080000000000000000A2
:10C2400081F0004102E000BF83F0004330B54FEAC7
:10C2500041044FEA430594EA050F08BF90EA020F34
:10C260001FBF54EA000C55EA020C7FEA645C7FEAC7
:10C27000655C00F0E2804FEA5454D4EB5555B8BFEA
:10C280006D420CDD2C4480EA020281EA030382EA5B
:10C29000000083EA010180EA020281EA0303362DED
:10C2A00088BF30BD11F0004F4FEA01314FF4801CC0
:10C2B0004CEA113102D0404261EB410113F0004FD2
:10C2C0004FEA03334CEA133302D0524263EB430389
:10C2D00094EA050F00F0A780A4F10104D5F1200E27
:10C2E0000DDB02FA0EFC22FA05F2801841F1000182
:10C2F00003FA0EF2801843FA05F359410EE0A5F156
:10C3000020050EF1200E012A03FA0EFC28BF4CF086
:10C31000020C43FA05F3C01851EBE37101F000453C
:10C3200007D54FF0000EDCF1000C7EEB00006EEB49
:10C330000101B1F5801F1BD3B1F5001F0CD34908D3
:10C340005FEA30004FEA3C0C04F101044FEA44522A
:10C3500012F5800F80F09A80BCF1004F08BF5FEAB1
:10C36000500C50F1000041EB045141EA050130BD91
:10C370005FEA4C0C404141EB0101013C28BFB1F5A3
:10C38000801FE9D291F0000F04BF01460020B1FAEE
:10C3900081F308BF2033A3F10B03B3F120020CDAC1
:10C3A0000C3208DD02F1140CC2F10C0201FA0CF09F
:10C3B00021FA02F10CE002F11402D8BFC2F1200C04
:10C3C00001FA02F120FA0CFCDCBF41EA0C019040BA
:10C3D000E41AA2BF01EB0451294330BD6FEA040403
:10C3E0001F3C1CDA0C340EDC04F11404C4F12002EE
:10C3F00020FA04F001FA02F340EA030021FA04F300
:10C4000045EA030130BDC4F10C04C4F1200220FA56
:10C4100002F001FA04F340EA0300294630BD21FA94
:10C4200004F0294630BD94F0000F83F4801306BF5A
:10C4300081F480110134013D4EE77FEA645C18BF4E
:10C440007FEA655C29D094EA050F08BF90EA020FE5
:10C4500005D054EA000C04BF1946104630BD91EADD
:10C46000030F1EBF0021002030BD5FEA545C05D1E0
:10C470004000494128BF41F0004130BD14F580041F
:10C480003CBF01F5801130BD01F0004545F0FE4193
:10C4900041F470014FF0000030BD7FEA645C1ABFC8
:10C4A000194610467FEA655C1CBF0B46024650EAFF
:10C4B000013406BF52EA033591EA030F41F400212B
:10C4C00030BD00BF90F0000F04BF0021704730B5B1
:10C4D0004FF4806404F132044FF000054FF0000186
:10C4E00050E700BF90F0000F04BF0021704730B547
:10C4F0004FF4806404F1320410F0004548BF40421C
:10C500004FF000013EE700BF42004FEAE2014FEA70
:10C5100031014FEA02701FBF12F07F4393F07F4F4B
:10C5200081F06051704732F07F4208BF704793F04E
:10C530007F4F04BF41F40021704730B54FF4607461
:10C5400001F0004521F000411CE700BF50EA010264
:10C5500008BF704730B54FF000050AE050EA01020D
:10C5600008BF704730B511F0004502D5404261EB7D
:10C5700041014FF4806404F132045FEA915C3FF4BE
:10C58000D8AE4FF003025FEADC0C18BF03325FEA5B
:10C59000DC0C18BF033202EBDC02C2F1200300FA0C
:10C5A00003FC20FA02F001FA03FE40EA0E0021FA31
:10C5B00002F11444BDE600BF70B54FF0FF0C4CF41F
:10C5C000E06C1CEA11541DBF1CEA135594EA0C0FD1
:10C5D00095EA0C0F00F0DEF82C4481EA030621EA0C
:10C5E0004C5123EA4C5350EA013518BF52EA033547
:10C5F00041F4801143F4801338D0A0FB02CE4FF0F9
:10C600000005E1FB02E506F00042E0FB03E54FF028
:10C610000006E1FB03569CF0000F18BF4EF0010E20
:10C62000A4F1FF04B6F5007F64F5407404D25FEA1C
:10C630004E0E6D4146EB060642EAC62141EA5551CF
:10C640004FEAC52040EA5E504FEACE2EB4F1FD0C11
:10C6500088BFBCF5E06F1ED8BEF1004F08BF5FEA8F
:10C66000500E50F1000041EB045170BD06F0004641
:10C6700046EA010140EA020081EA0301B4EB5C04EE
:10C68000C2BFD4EB0C0541EA045170BD41F48011E6
:10C690004FF0000E013C00F3AB8014F1360FDEBF0B
:10C6A000002001F0004170BDC4F10004203C35DAE7
:10C6B0000C341BDC04F11404C4F1200500FA05F36A
:10C6C00020FA04F001FA05F240EA020001F000420B
:10C6D00021F0004110EBD37021FA04F642EB060181
:10C6E0005EEA430E08BF20EAD37070BDC4F10C04AB
:10C6F000C4F1200500FA04F320FA05F001FA04F26F
:10C7000040EA020001F0004110EBD37041F100015A
:10C710005EEA430E08BF20EAD37070BDC4F1200565
:10C7200000FA05F24EEA020E20FA04F301FA05F2CD
:10C7300043EA020321FA04F001F0004121FA04F275
:10C7400020EA020000EBD3705EEA430E08BF20EA45
:10C75000D37070BD94F0000F0FD101F0004640007F
:10C7600041EB010111F4801F08BF013CF7D041EA01
:10C77000060195F0000F18BF704703F00046520005
:10C7800043EB030313F4801F08BF013DF7D043EAD6
:10C790000603704794EA0C0F0CEA135518BF95EA8C
:10C7A0000C0F0CD050EA410618BF52EA4306D1D113
:10C7B00081EA030101F000414FF0000070BD50EA32
:10C7C000410606BF1046194652EA430619D094EABC
:10C7D0000C0F02D150EA013613D195EA0C0F05D1A6
:10C7E00052EA03361CBF104619460AD181EA0301FA
:10C7F00001F0004141F0FE4141F470014FF00000B2
:10C8000070BD41F0FE4141F4780170BD70B54FF04C
:10C81000FF0C4CF4E06C1CEA11541DBF1CEA1355CC
:10C8200094EA0C0F95EA0C0F00F0A7F8A4EB0504AE
:10C8300081EA030E52EA03354FEA013100F08880A5
:10C840004FEA03334FF0805545EA131343EA12636E
:10C850004FEA022245EA111545EA10654FEA002623
:10C860000EF000419D4208BF964244F1FD0404F5DC
:10C87000407402D25B084FEA3202B61A65EB030538
:10C880005B084FEA32024FF480104FF4002CB6EBF5
:10C89000020E75EB030E22BFB61A754640EA0C0075
:10C8A0005B084FEA3202B6EB020E75EB030E22BFB5
:10C8B000B61A754640EA5C005B084FEA3202B6EBF6
:10C8C000020E75EB030E22BFB61A754640EA9C00B5
:10C8D0005B084FEA3202B6EB020E75EB030E22BF85
:10C8E000B61A754640EADC0055EA060E18D04FEA43
:10C8F000051545EA16754FEA06164FEAC30343EAE3
:10C9000052734FEAC2025FEA1C1CC0D111F4801FAF
:10C910000BD141EA00014FF000004FF0004CB6E7A8
:10C9200011F4801F04BF01430020B4F1FD0C88BF47
:10C93000BCF5E06F3FF6AFAEB5EB030C04BFB6EB52
:10C94000020C5FEA500C50F1000041EB045170BD45
:10C950000EF0004E4EEA113114EB5C04C2BFD4EB72
:10C960000C0541EA045170BD41F480114FF0000EF6
:10C97000013C90E645EA060E8DE60CEA135594EA72
:10C980000C0F08BF95EA0C0F3FF43BAF94EA0C0F75
:10C990000AD150EA01347FF434AF95EA0C0F7FF4EA
:10C9A00025AF104619462CE795EA0C0F06D152EA3E
:10C9B00003353FF4FDAE1046194622E750EA410622
:10C9C00018BF52EA43067FF4C5AE50EA41047FF433
:10C9D0000DAF52EA43057FF4EBAE12E74FF0FF3C98
:10C9E00006E000BF4FF0010C02E000BF4FF0010C69
:10C9F0004DF804CD4FEA410C7FEA6C5C4FEA430CE2
:10CA000018BF7FEA6C5C1BD001B050EA410C0CBF30
:10CA100052EA430C91EA030F02BF90EA020F002092
:10CA2000704710F1000F91EA030F58BF994208BFF9
:10CA300090422CBFD8176FEAE37040F001007047B6
:10CA40004FEA410C7FEA6C5C02D150EA013C07D10D
:10CA50004FEA430C7FEA6C5CD6D152EA033CD3D058
:10CA60005DF8040B704700BF8446104662468C4652
:10CA70001946634600E000BF01B5FFF7B7FF002885
:10CA800048BF10F1000F01BD4DF808EDFFF7F4FFAE
:10CA90000CBF012000205DF808FB00BF4DF808ED39
:10CAA000FFF7EAFF34BF012000205DF808FB00BF5C
:10CAB0004DF808EDFFF7E0FF94BF012000205DF87E
:10CAC00008FB00BF4DF808EDFFF7CEFF94BF012033
:10CAD00000205DF808FB00BF4DF808EDFFF7C4FF2C
:10CAE00034BF012000205DF808FB00BF4FEA410C75
:10CAF0007FEA6C5C02D150EA013C0AD14FEA430C58
:10CB00007FEA6C5C02D152EA033C02D14FF0000094
:10CB100070474FF0010070474FEA410212F50012D2
:10CB200015D211D56FF47873B3EB625212D94FEA74
:10CB3000C12343F0004343EA505311F0004F23FA5E
:10CB400002F018BF404270474FF00000704750EAB3
:10CB5000013005D111F0004008BF6FF00040704770
:10CB60004FF00000704700BF4A0011D212F50012CA
:10CB700011D20DD56FF47873B3EB62520ED44FEA35
:10CB8000C12343F0004343EA505323FA02F07047B5
:10CB90004FF00000704750EA013002D14FF0FF30F3
:10CBA00070474FF0000070474FEA4102B2F1E04396
:10CBB00024BFB3F5001CDCF1FE5C0DD901F0004C84
:10CBC0004FEAC0024CEA5070B2F1004F40EB8300D4
:10CBD00008BF20F00100704711F0804F21D113F100
:10CBE0003872BCBF01F00040704741F480114FEA39
:10CBF0005252C2F11802C2F1200C10FA0CF320FAC2
:10CC000002F018BF40F001004FEAC1234FEAD323DE
:10CC100003FA0CFC40EA0C0023FA02F34FEA430348
:10CC2000CCE77FEA625307D150EA01331EBF4FF0D1
:10CC3000FE4040F44000704701F0004040F0FE40EC
:10CC400040F40000704700BF80F0004002E000BFE9
:10CC500081F0004142001FBF5FEA410392EA030FE7
:10CC60007FEA226C7FEA236C6AD04FEA1262D2EB31
:10CC70001363C1BFD218414048404140B8BF5B4236
:10CC8000192B88BF704710F0004F40F4000020F0CF
:10CC90007F4018BF404211F0004F41F4000121F0E5
:10CCA0007F4118BF494292EA030F3FD0A2F101022F
:10CCB00041FA03FC10EB0C00C3F1200301FA03F16D
:10CCC00000F0004302D5494260EB4000B0F5000F90
:10CCD00013D3B0F1807F06D340084FEA310102F14F
:10CCE0000102FE2A51D2B1F1004F40EBC25008BF01
:10CCF00020F0010040EA03007047490040EB0000CB
:10CD0000013A28BFB0F5000FEDD2B0FA80FCACF1CB
:10CD1000080CB2EB0C0200FA0CF0AABF00EBC250F8
:10CD200052421843BCBFD0401843704792F0000FE6
:10CD300081F4000106BF80F400000132013BB5E739
:10CD40004FEA41037FEA226C18BF7FEA236C21D0AF
:10CD500092EA030F04D092F0000F08BF0846704714
:10CD600090EA010F1CBF0020704712F07F4F04D1E2
:10CD7000400028BF40F00040704712F100723CBFF5
:10CD800000F50000704700F0004343F0FE4040F41F
:10CD9000000070477FEA226216BF08467FEA2363DD
:10CDA0000146420206BF5FEA412390EA010F40F4C8
:10CDB000800070474FF0000304E000BF10F0004314
:10CDC00048BF40425FEA000C08BF704743F09643FB
:10CDD00001464FF000001CE050EA010208BF704716
:10CDE0004FF000030AE000BF50EA010208BF70479D
:10CDF00011F0004302D5404261EB41015FEA010CB2
:10CE000002BF84460146002043F0B64308BFA3F1A9
:10CE10008053A3F50003BCFA8CF2083AA3EBC2538B
:10CE200010DB01FA02FC634400FA02FCC2F12002AA
:10CE3000BCF1004F20FA02F243EB020008BF20F0E1
:10CE40000100704702F1200201FA02FCC2F1200247
:10CE500050EA4C0021FA02F243EB020008BF20EA3C
:10CE6000DC7070477BB972B90029BEBF00204FF05B
:10CE7000004106E008BF00281CBF6FF000414FF0E2
:10CE8000FF3000F015BAADF1080C6DE904CE0029B1
:10CE900009DB002B1ADB00F0A3F8DDF804E0DDE984
:10CEA000022304B07047404261EB4101002B1BDBC1
:10CEB00000F096F8DDF804E0DDE9022304B040421A
:10CEC00061EB4101524263EB43037047524263EB13
:10CED000430300F085F8DDF804E0DDE9022304B047
:10CEE000404261EB41017047524263EB430300F063
:10CEF00077F8DDF804E0DDE9022304B0524263EB89
:10CF00004303704753B94AB9002908BF00281CBF22
:10CF10004FF0FF314FF0FF3000F0CAB9ADF1080C0F
:10CF20006DE904CE00F05CF8DDF804E0DDE90223F1
:10CF300004B0704730B1012390FAA0F0B0FA80F04D
:10CF40001844704708460029FBD02123F4E700BFAE
:10CF5000430803F05533C01A830803F0333300F05D
:10CF60003330184400EB101000F00F3000EB0020BD
:10CF700000EB0040000E704707EE900AF5EEC07A15
:10CF8000F1EE10FA01D400F00BB8F1EE677A08B5B3
:10CF900017EE900A00F004F8404261EB410108BD31
:10CFA000D0B5FFF7B1FA0C4B002206460F46FFF74B
:10CFB00003FBFFF7D9FD0446FFF784FA074B002275
:10CFC000FFF7FAFA02460B4630463946FFF73CF9BE
:10CFD000FFF7CAFD2146D0BD0000F03D0000F04142
:10CFE0002DE9F047089D04468E46002B4DD18A421C
:10CFF000944669D9B2FA82F252B101FA02F3C2F14F
:10D00000200120FA01F10CFA02FC41EA030E9440DF
:10D010004FEA1C48210CBEFBF8F61FFA8CF708FB00
:10D0200016E341EA034306FB07F199420AD91CEBD8
:10D03000030306F1FF3080F01F81994240F21C810A
:10D04000023E63445B1AA4B2B3FBF8F008FB103352
:10D0500044EA034400FB07F7A7420AD91CEB040487
:10D0600000F1FF3380F00A81A74240F20781644457
:10D07000023840EA0640E41B00261DB1D4400023DC
:10D08000C5E900433146BDE8F0878B4209D9002D40
:10D0900000F0EF800026C5E9000130463146BDE8CA
:10D0A000F087B3FA83F6002E4AD18B4202D3824234
:10D0B00000F2F980841A61EB030301209E46002DE3
:10D0C000E0D0C5E9004EDDE702B9FFDEB2FA82F238
:10D0D000002A40F09280A1EB0C014FEA1C471FFA96
:10D0E0008CFE0126200CB1FBF7F307FB131140EA7D
:10D0F00001410EFB03F0884208D91CEB010103F14A
:10D10000FF3802D2884200F2CB804346091AA4B20B
:10D11000B1FBF7F007FB101144EA01440EFB00FEDF
:10D12000A64508D91CEB040400F1FF3102D2A64544
:10D1300000F2BB800846A4EB0E0440EA03409CE7E3
:10D14000C6F12007B34022FA07FC4CEA030C20FA90
:10D1500007F401FA06F31C43F9404FEA1C4900FAB0
:10D1600006F3B1FBF9F8200C1FFA8CFE09FB18112D
:10D1700040EA014108FB0EF0884202FA06F20BD9A0
:10D180001CEB010108F1FF3A80F08880884240F2F0
:10D190008580A8F102086144091AA4B2B1FBF9F034
:10D1A00009FB101144EA014100FB0EFE8E4508D92F
:10D1B0001CEB010100F1FF346CD28E456AD90238B4
:10D1C000614440EA0840A0FB0294A1EB0E01A14299
:10D1D000C846A64656D353D05DB1B3EB080261EB07
:10D1E0000E0101FA07F722FA06F3F1401F43C5E9E1
:10D1F000007100263146BDE8F087C2F12003D84017
:10D200000CFA02FC21FA03F3914001434FEA1C4758
:10D210001FFA8CFEB3FBF7F007FB10360B0C43EA4A
:10D22000064300FB0EF69E4204FA02F408D91CEBFA
:10D23000030300F1FF382FD29E422DD902386344F8
:10D240009B1B89B2B3FBF7F607FB163341EA034198
:10D2500006FB0EF38B4208D91CEB010106F1FF38E7
:10D2600016D28B4214D9023E6144C91A46EA0046DE
:10D2700038E72E46284605E70646E3E61846F8E670
:10D280004B45A9D2B9EB020864EB0C0E0138A3E7B9
:10D290004646EAE7204694E74046D1E7D0467BE79A
:10D2A000023B614432E7304609E76444023842E712
:10D2B000704700BF02E000F000F8FEE772B63748A2
:10D2C00080F30888364880F3098836483649086074
:10D2D00040F20000CCF200004EF63471CEF20001B4
:10D2E0000860BFF34F8FBFF36F8F40F20000C0F2B2
:10D2F000F0004EF68851CEF200010860BFF34F8F68
:10D30000BFF36F8F4FF00000E1EE100A4EF63C7154
:10D31000CEF200010860062080F31488BFF36F8FFF
:10D32000A6F084F9A5F05CFA4FF055301F491B4A6E
:10D3300091423CBF41F8040BFAE71D49184A91425B
:10D340003CBF41F8040BFAE71A491B4A1B4B9A42AF
:10D350003EBF51F8040B42F8040BF8E700201849CF
:10D36000184A91423CBF41F8040BFAE7A6F062F973
:10D37000A5F08AFA144C154DAC4203DA54F8041B9C
:10D380008847F9E701F000F9114C124DAC4203DA7D
:10D3900054F8041B8847F9E7A6F04AB900060020B4
:10D3A0000022002000C0000808ED00E0000000207E
:10D3B0000006002078F70D0800220020442C0020F1
:10D3C000482C0020C8660120E0C1000838C20008CF
:10D3D00038C2000838C200082DE9F04F2DED108A40
:10D3E000C1F80CD0C3689D46BDEC108ABDE8F08F33
:10D3F000002383F311882846A0470020A4F076FF7D
:10D40000FEE7A4F0E3FD00DFFEE7000001F0FF010E
:10D41000102A2BDB10F0070F08D010F8013B013A5F
:10D420008B422DD010F0070F42B3F6D1F0B441EA91
:10D43000012141EA014122F007047FF000070023A7
:10D44000F0E80256083C85EA010586EA010685FAFD
:10D4500047F5A3FA87F586FA47F6A5FA87F68EB957
:10D46000EED1F0BC01F0FF0102F0070232B110F87A
:10D47000013B013A83EA010313B1F8D10020704760
:10D4800001387047002D06BF35460338073815F0C0
:10D49000010F07D1013015F4807F02BF013015F470
:10D4A000C03F0130F0BC0138704700BF10F8012BBD
:10D4B00011F8013B012A28BF9A42F7D0D01A7047D1
:10D4C000034613F8012B002AFBD1181A01387047C4
:10D4D00038B50022002304460D46FFF7DFFA28B9CD
:10D4E00020462946BDE8384000F00AB8204605F13C
:10D4F000004100F005F8404261EB410138BD00BF3A
:10D50000D0B50C4B002206460F46FFF755F8FFF743
:10D510002BFB0446FEF7D6FF074B0022FFF74CF823
:10D5200002460B4630463946FEF78EFEFFF71CFBDF
:10D530002146D0BD0000F03D0000F041036800220C
:10D540001B68184710B503685B680446984708B124
:10D5500094F84D0010BD000038B504467BF0B0FED5
:10D560000E4B1D680146E86A02681268904751F048
:10D570009BFDEB6A93F89C1050F082FD94F83730D5
:10D580005BB183F04FFEEB6AD3F8A030C01AB0F560
:10D59000FA6F24BF002384F8373038BD542C0020A4
:10D5A00070B50E4605465DF0EBF95DF0ADF910B9CA
:10D5B0000124204670BD0A4B93F9B633012BF7D1F5
:10D5C0005DF0DEF9437A002BF2D15DF0D9F9847A6F
:10D5D000002CEDD1034A314628467CF0B7F8E8E745
:10D5E000584C0020A0B90B08034BD3F820340BB9DA
:10D5F0007BF01CBE01207047584C00202DE9F04301
:10D600002DED028BC47F91B006460F468CB990F980
:10D610000430002B00F0FE807F4B1D68A86A036871
:10D620005B6B9847044650B97C4A394630467CF0DB
:10D630008DF8204611B0BDEC028BBDE8F083B368D5
:10D640004BB933685B6B3946304611B0BDEC028B89
:10D65000BDE8F0431847E86AFFF774FF0446002866
:10D66000E7D1394630467CF04FFFDFF8E4810546CC
:10D67000394630467CF092F898EDF27AD8EDF17A9E
:10D68000B4EEE77A2840F1EE10FAC5B209D598F960
:10D69000C033032B05D0624A394630467CF056F839
:10D6A0002546D8EDDA7AB0EE088AF4EEC87AF1EEC3
:10D6B00010FA0BD517EE900AFEF726FF594ACDE96E
:10D6C0000001394630467CF041F80025D8EDDB7A80
:10D6D000F4EEC87AF1EE10FA0BD517EE900AFEF7C9
:10D6E00013FF514ACDE90001394630467CF02EF84F
:10D6F0000025D8EDDC7AB8EE087AF4EEC77AF1EEC0
:10D7000010FA0BDD17EE900AFEF7FEFE474ACDE950
:10D710000001394630467CF019F80025B8F9543339
:10D72000042B07DC052200923946414A30467CF042
:10D730000DF80025D8F8040C5DF07EF980B198F959
:10D74000B6336BB1D8F8043CB8F9B823B3F90E304E
:10D750009A4205DA374A394630467BF0F7FF002512
:10D76000DFF8F09039463046FFF71AFF99F8C93DC7
:10D77000002B48D100EA05042F484FF4806100F0E7
:10D78000F9FE78B1D8F8043CB3F90C30A3F2E242C8
:10D7900092B2B2F5FA7F05D9284A394630467BF075
:10D7A000D5FF0024264890F864345BB100F25C4059
:10D7B0002CF042FD054628B9224A394630467BF016
:10D7C000C5FF2C4600212E2204A80DF10C08039160
:10D7D000A9F0A8FED9F8B40D4246322108F05EF94E
:10D7E000054600287FF425AFD9F8B40D03689B687F
:10D7F0009847154ACDF800800346394630467BF0FD
:10D80000A5FF2C4615E7114A394630467BF09EFFAE
:10D810000024B1E701240CE7542C0020B0B90B0818
:10D82000C7B90B08EAB90B080ABA0B082CBA0B08DF
:10D830004EBA0B086DBA0B08582C0020A8BA0B087A
:10D84000587C0020D0BA0B08A06B0C0893BA0B08C8
:10D85000584C0020586C002070B505460E46FFF766
:10D860009FFE3146044628467CF0FAFC2040C0B2B8
:10D8700070BD0000F0B591B005460E467CF02EF864
:10D880000446D8B1102128467BF036FDB0B1002106
:10D890002E2204A803AF0391A9F044FE10F03AF938
:10D8A00032233A4601210FF043FC044630B9054BC0
:10D8B00000973246102128467BF026FD204611B005
:10D8C000F0BD00BFE4BA0B0870B505460E46B1B90D
:10D8D00090F910408CB116480BF050F8DFED157A36
:10D8E000B0EEC00AB4EEE70AF1EE10FA07D4124A1D
:10D8F000012128467BF02AFF3446204670BDAB68E4
:10D900009BB10E4B1B68D86AFFF71CFE044630B172
:10D910005BF044FB0A4A042154F074FCEDE7314605
:10D920002846BDE870407CF0A5BA0124E5E700BFB9
:10D93000582C002000000034F0BA0B08542C0020B2
:10D9400002BB0B0838B504467CF09EFE0546A8B124
:10D950000B4805F075FB38B10A490B480FF028FD5C
:10D9600010B1074800F0D8FD2046FFF7F5FD012370
:10D97000064984F8373020467CF096FD284638BDAD
:10D98000582C0020908B0020683F002024BB0B08FF
:10D99000F8B505460E461746C2B1232901D0012924
:10D9A00014D81E4807F0F4FB044668B10024204652
:10D9B000F8BD95F91030022B08D05BF0EFFA184A49
:10D9C000062154F01FFCF2E7002EF2D03A46314611
:10D9D00028467CF00FFF04460028E7D0114ED6F809
:10D9E000B42D06F648539A4203D003F214702DF07A
:10D9F00059F8D6F8B40D03689B6B98470A4B83F827
:10DA000030042846FFF7A8FD4FF0FF330749C6F85A
:10DA1000E43D28467CF048FDC9E700BF582C0020B3
:10DA200034BB0B08586C0020587C00204CBB0B0802
:10DA3000F8B505460E467BF00BFD104B93F98B7342
:10DA40000446CFB90E48BD212CF0C2FF38B10D4BB2
:10DA500032464FF4804128467BF056FC3C4608484D
:10DA6000BC212CF0B5FF38B1074B32464FF4804152
:10DA700028467BF049FC00242046F8BD584C002085
:10DA8000B480002060BB0B088CBB0B0800207047E3
:10DA9000014800F0E9BC00BF582C002003685B6817
:10DAA000184700000DF098B864F01ABB5CF0B6BEE1
:10DAB00025F0D4BA50F066BC07F0A2BC4EF01EBDF3
:10DAC0000AF05EBA02F040BE4DF0B4B813F0F4BFF5
:10DAD00060F01EBB5FF09CBF0CF076B946F078B8E2
:10DAE0000AF0CABF13F046BB66F0AEB85CF0B8BB34
:10DAF0005AF0C2BC06F0B0BE04F03ABA09F0C8BD94
:10DB00000AF0AEB90BF094BF0CF00CBA0AF0ECBD01
:10DB10000CF0B4B801F032B900F2845017F096B8A6
:10DB200007F0D8B990F8F432B02202FB030390F862
:10DB3000382393F8D13012B1012B28BF01231846A6
:10DB400070470000034808602C21117008221A60F9
:10DB5000704700BFD0BE0B0870B5044604F5985559
:10DB600000F5C04044301035FFF7F6FC0021284690
:10DB70000FF056FF802120460CF03EFC18B126F035
:10DB800061FE24F031FF04F50053D3EDDA7ADFEDC6
:10DB9000236A93EDDC7A67EEA67A04F58052FDEEF7
:10DBA000E77A02F25C51D1ED006AF8EEE77A02F50D
:10DBB000AB6267EEA67A03F61843FDEEE77A05F549
:10DBC000457017EE901A43F8041CD2ED007AF0EE7F
:10DBD000E77A67EE877A04F5B251C3ED007A08312F
:10DBE00029F004FE04F5A04694ED467AD6EDEB7AD2
:10DBF000E7EE007AC6EDEB7AB0EE670A27F046FB57
:10DC00004FF4001186EDEB0A20460CF0F5FB20B135
:10DC10002846BDE870400EF039BA70BD0000C84219
:10DC2000FFF79ABF10B500F580430446D3F8B40D52
:10DC300003689B6B984704F5A04393F8EB333BB91B
:10DC400030B104F532503030BDE8104080F088BF6C
:10DC500010BD0000FFF7E6BF38B54FF48011044651
:10DC60000CF0CAFB054620B9012120460CF0C4FB8C
:10DC70000546022120460CF0BFFB48B115B92046ED
:10DC800002F006FD04F5985010300EF0FDF801E0AA
:10DC9000002DF7D14FF4805120460CF0ADFB30B190
:10DCA00004F5BF404030BDE8384060F057BB38BD98
:10DCB000FFF7D2BF38B54FF4801104460CF09CFB3F
:10DCC0000121054620460CF097FB18B115B92046F6
:10DCD00002F0DEFC102120460CF08EFB60B12046E5
:10DCE00002F04AFD4FF4800120460CF085FB18B984
:10DCF00026F0A8FD24F06AFF202120460CF07CFBD2
:10DD000028B1204602F0AEFD204602F0C9FE4FF4D5
:10DD1000005120460CF070FB10B1204602F0A8FE26
:10DD2000802120460CF068FB28B126F08BFDBDE871
:10DD3000384024F07DBE38BDFFF7BCBF00F58043FE
:10DD400000F5BD40D3F8D81D1C307EF04BB9000063
:10DD5000FFF7F4BF10B5044617F068F890F92130CA
:10DD60008BB190F8403373B194F9A8355BB1064B91
:10DD70001B68DB6A93F89C302BB904F28450BDE831
:10DD8000104016F07BBD10BD542C0020FFF7E2BF01
:10DD90002DE9F843424B1B68DB6A93F89C3004463C
:10DDA000002B7BD000F5805898F81936002B75D0E1
:10DDB00007F0EEF9002871D004F5005604F500557F
:10DDC000383695F8861130460DF002FC002865D0F3
:10DDD00004F590773846FFF7A5FE02285ED994F83F
:10DDE00014244FF0B00909FB024292ED837AF1EE60
:10DDF000007AB4EEE77AF1EE10FA4FD495F8861176
:10DE000030460DF095FEB5F9543307EE903AB8EE72
:10DE1000E77AB4EEC07AF1EE10FA0CDD94F814341F
:10DE200009FB0343F8EE677A93ED837AF4EEC77A41
:10DE3000F1EE10FA32DCD8F80835D5F8142C002BA6
:10DE4000B8BF5B42934229DC08F20C53D3ED007A51
:10DE5000D5EDDB6A9FED136AF8EEE77A66EE866A27
:10DE6000F4EEE67AF1EE10FA18DC05F6184393EDBD
:10DE7000007A27EE067AF4EEC77AF1EE10FA0DD4A6
:10DE800094F81414B5F95623B02303FB01713046FE
:10DE900001F58271BDE8F8430DF084BABDE8F8835E
:10DEA000542C00200000C842FFF772BF2DE9F0415A
:10DEB00090F814342D4D00EB03132F68D3F8C48170
:10DEC00000F5907604463046FFF72CFE474514D007
:10DED000022814D904F58047C5F8008097F8DC3D86
:10DEE000012B15D817D104F5A045D5F8403FE3B96B
:10DEF000D5F8443FCBB905230BE0022810D804F530
:10DF0000804393F8DC2D5AB1052283F8DC2D07E01D
:10DF1000013B87F8DC3D04F5BA500C3010F07AFF75
:10DF20002046BDE8F04109F05BBD114B1B68D86A83
:10DF300003685B68984780460028ECD194F8141475
:10DF4000B02303FB0161DC31204605F0EBF8D5F886
:10DF5000243F0FCB05F6287605F6487586E80F00B6
:10DF600085E80F0087F8DC8DD5E700BF482C00203E
:10DF7000542C0020FFF79ABF10B500F5A04300F520
:10DF8000805493F8EB231AB1002384F819360AE081
:10DF9000D3F83834042B07D100F5BC40103081F0A1
:10DFA0007DF884F8190610BD0123EEE710B500F5E1
:10DFB000804400F59A43D4F8B41D4833994200F5E3
:10DFC000A04308D000F59B420C3291421CBF4FF099
:10DFD000FF32C3F8A423074AC3F89423064AC3F8C0
:10DFE0009823FFF7C9FFD4F8B40D0368BDE81040CB
:10DFF0001B6918470000C8420000C8C2FFF7D6BF1F
:10E00000F7B500F5A0460446D6F838348B420D46E5
:10E010003ED00B1F00F5BC47594207F1100759418C
:10E020003846019180F02AFF0199384680F026FF9A
:10E03000042D02D117486CF08BFCD6F83834012B34
:10E0400018D1032D16D104F5C04044307BF042F9BD
:10E0500040B1204607F09CF820B104F52E502C303A
:10E060006CF070FC2046C6F8385403B0BDE8F040B0
:10E0700002F064BC072DF5D1D6F8B4236423052142
:10E0800092FBF3F304F54F50034A54F0BBF8E9E771
:10E0900003B0F0BD0458002030BC0B0838B500F5C3
:10E0A00080450446D5F8B40D03689B6B984700285B
:10E0B0003FD004F5A04393F83024D2BBD5F8B41D6B
:10E0C00004F59A424832914235D193F8E4232AB9B3
:10E0D00001212046BDE83840FFF792BFB3F89A24EB
:10E0E000152A26D193F8141E11F001011FD1D3F87F
:10E0F0003824072A1BD093F98A3E0BB90421E8E79C
:10E1000020460AF03BFCDFED0F7AB4EEE70AF1EEB1
:10E1100010FAF3DB04F5BC40103080F0FFFE00285D
:10E12000ECD0094A062104F54F5054F06BF8072152
:10E13000CFE70321CDE704F59B430C339942F8D197
:10E1400038BD00BF0000B44254BC0B0838B5214CA8
:10E15000D4F8B42D04F648539A422DED028BB0EE5C
:10E16000408A03D00020BDEC028B38BD04F58055F9
:10E17000D5F83834042B23D194F8DD3D33B116495A
:10E18000A1F6DC202CF006FF0028ECD19FED137ADD
:10E19000F0EEC87AF4EEC77AF1EE10FA07D49FEDEC
:10E1A000100A28EE008ABDEEC88A85EDED8A0D487A
:10E1B00080F0B4FE0028D5D0002385F8E733D2E7FD
:10E1C000B5F89A14A4F5804006F0AAF90028D3D136
:10E1D000C8E700BF586C0020908B0020000000347E
:10E1E0000000C842688A002010B52DED028B00F5B2
:10E1F000A0430446D3F83824042A0BD104F07EF956
:10E200002046B0EE408A04F049FA38EE400ABDECF0
:10E21000028B10BD03F6747393ED000AF7E700005C
:10E220002DE9F0412DED028B00F58C658AB0044696
:10E23000284611F0A9FF04F59850002307A91030D3
:10E240000793089309930FF077FA002800F087806E
:10E250009DED090ADFED597A04F5A04595EDF17AB7
:10E2600020EE270ADFED567AA7EE270A04F5AA402A
:10E27000543004F5804685EDF10A65F0F9FE20463C
:10E28000FFF70CFFD6F8B40D03689B6B984795F821
:10E29000EB33002B5ED100285CD095F83034002B96
:10E2A00058D1D5F83834042B70D09FED468A2046DB
:10E2B00004F016FA04F5C04204F59A43C2F8FC00D3
:10E2C000D6F8B41D603399421CD195F8B83FCBB94C
:10E2D00004F50053B3F9E43B002B04DC3A49D1F8D0
:10E2E000A41BC9060ED5D5F8247FD5F82C1F7F684E
:10E2F0000A33C91B64277B438142ACBF5B181B18E0
:10E30000C2F8FC30D5F83834D2F8FC10D6F8E02D3D
:10E3100005912046049203930CF0D6FAB6F9EE6DFF
:10E3200007462046FFF760FFCDE9007604F5005070
:10E33000D0EDFC1A059905F2544504F53250F0EE83
:10E34000400ADDE9033295ED001AB0EE480A30309C
:10E3500080F0AAF80AB0BDEC028BBDE8F08104F5AC
:10E360009070FFF7DFFB02280AD994F81434B0222A
:10E3700002FB034393F8402212B193ED8B0A69E745
:10E38000284611F09BFDB1EE400A63E704F5BE4755
:10E3900004F5BE48383708F1480804F5BE41424646
:10E3A0002831384615F086FE00283FF47EAF4146FE
:10E3B000384615F013FFB0EE408A78E7CDCC4C3EDE
:10E3C000CDCC4C3F00000000584C0020FFF728BF88
:10E3D00000F5804200F59B43D2F8B42D04339A42F5
:10E3E0001FBF00F5A040D0F8CC330B60012008BF60
:10E3F0000020704710B500F5804200F59B43D2F82D
:10E40000B42D04339A420C4612D000F54050D0F897
:10E41000E80503681B69984707EE900A9FED057AA7
:10E42000F8EEE77A012067EE877AC4ED007A10BD36
:10E430000020FCE70AD7233C10B500F5804200F528
:10E440009B43D2F8B42D04339A420C460AD000F50F
:10E450004050D0F8E80503685B699847012084EDD7
:10E46000000A10BD0020FCE730B505460FC985B095
:10E470006C4684E80F0040F279322146284604F0C9
:10E48000E5FC0C4B03F55762D3F8B43D93420ED133
:10E490009DF8001011F0040102D1204615F006FC91
:10E4A0000548214604F08CFD012005B030BD002058
:10E4B000FBE700BF586C0020582C002000F580407E
:10E4C000D0F8B40D03689B6C1847000000F580403D
:10E4D000D0F8B40D0368DB6C1847000010B500F5E8
:10E4E000805303F5A36403F21453246814601B687B
:10E4F0000B6000F50050D0F8A43B9B0509D4D0ED8B
:10E50000FC6AD2ED007A9FED037AE6EEC77AC2ED9F
:10E51000007A10BD35FA8E3C38B50D4D04462946BB
:10E520000C480FF057F804F5804305F13C0183F8DF
:10E53000DD0D04F5985010300EF0E4FE04F5BE40F9
:10E54000D0ED1D7AF1EE677AC0ED1D7A38BD00BFBF
:10E55000908B0020683F002010B5044600F59070B5
:10E560001FF00EF82046BDE81040FFF7D5BF0000B1
:10E57000FFF7F2BF00F50050D0F8A43B194214BFDA
:10E58000012000207047000038B5054B1C68236847
:10E590000A461D68034B01462046A847002038BDA7
:10E5A000542C0020582C002070B52DED028B044611
:10E5B000036804F500559B6D9847D5F8A43B1B06EE
:10E5C00018D5B5F95433B5F95613CA1A0B4402EBF2
:10E5D000D27203EBD37352105B1000EE902A00EE60
:10E5E000103A04F59850F8EEE00AB8EEC00A103080
:10E5F0000EF046FC5A4BB5F886231A7004F5C04558
:10E600005EF026FB44355DF075FF00212846FEF7DD
:10E61000F5FF544E0123B0712846F3717AF050FE95
:10E6200028B928467BF054FFB0FA80F040093071D9
:10E63000042120460BF0E0FE20B104F5AA4074301E
:10E640004EF00EF828467AF03BFEE8B994F8143400
:10E6500004F5A04504EB031341F28832D3F8C461FA
:10E66000D5F8BC3FF31A93420ED904F59070FFF72A
:10E6700059FA022808D9C5F8BC6F204605F561652E
:10E6800004F0DEFC00232B60B4F9A4301BB9B4F80D
:10E69000A230A4F8A430B4F8A430DFED338A07EE3A
:10E6A000903AF8EEE77AB7EE008A88EE270AD4EDC2
:10E6B0002B7AF0EEE77AF4EEE87AF1EE10FA09D56B
:10E6C000B4F9A23007EE903AF8EEE77A88EE277AAE
:10E6D00084ED2B7AD4ED2B0A26F0DAFC20BB4EF029
:10E6E000D1FE40F27D124FF480114EF083FE4CF0CB
:10E6F00057FB4BF0BFFF04F53D502C30B0EE408A85
:10E7000073F0A8FE04F54350B0EE480A083073F0E9
:10E71000A1FEB0EE480ABDEC028B04F547503C3038
:10E72000BDE8704073F096BED4ED2B7A94ED460AA6
:10E73000F0EEE77AF4EEE87AF1EE10FA09D5B4F9E2
:10E74000A23007EE903AF8EEE77A88EE277A84ED69
:10E750002B7AD4ED2B0A26F09BFC0028BFD0C6E70D
:10E76000A0230020058E002000000034FFF71CBF0E
:10E7700070B500F5A046044696F9883E002B27DDCB
:10E7800006F006FD20BB04F5C045443528467BF065
:10E790009FFEE8B128467AF093FDC8B182F042FDB1
:10E7A000D6F8D433C01A96F9883E4FF47A725343A0
:10E7B00098420DD301221C212846FFF7E9F838B111
:10E7C00004F54F50034ABDE87040062153F01ABDCE
:10E7D00070BD00BF74BC0B0830B52DED028B044634
:10E7E00083B000F5985001A910300EF077FF002893
:10E7F00071D004F5A04595EDEF7ADDED017AB4EE28
:10E80000E77AF1EE10FA08D504F5C04044307AF00A
:10E8100061FD10B1019BC5F8BC3304F50054D4ED83
:10E82000EA6AB4F95433052BB8BF052307EE903AD2
:10E83000B4F9563307EE103AB8EEC77AF8EEE77A35
:10E8400037EE077A1820C6EE870AB6EE007AF4EEA5
:10E85000470AF1EE10FAC8BFF0EE470A9FED2D7A95
:10E8600067EE877A9FED2C7A86EEA71AF0EE007A93
:10E87000B4EE671AF1EE10FA48BFB0EE671ADDED9C
:10E88000017AF4EEC77AF1EE10FACCBF86EEA70A51
:10E89000B0EE410A26F00EFDB0EE408A1F480DF0A2
:10E8A00027FF90B91E484021FFF764FE68B11D4B59
:10E8B000D3F83834012B08D1F7EE007AB4EEE78AAA
:10E8C000F1EE10FA58BFB0EE678AB0EE480A03B016
:10E8D000BDEC028B30BD04F5C04044307AF0FAFC48
:10E8E000B7EE008A0028D9D046205DF053FCB4EE84
:10E8F000C80ADFED0D7AF1EE10FAD8BFB0EE480A83
:10E9000087EE800AA6F062FD2F209FED081ADFED4A
:10E91000080ABFE73333333F17B7D138683F0020C9
:10E92000582C0020587C0020000034428FC2D53F74
:10E930009A99193FF8B504465CF022F80368DB6841
:10E940009847054610B900252846F8BD204606F030
:10E95000AFFA04F580460746D6F8B40D03689B6B02
:10E96000984780B10E4BD3F8B40D03685B6B9847A2
:10E9700048B104F5005494F9FD33002BE3D0032B88
:10E98000E1D03D46E0E796F8C83D002BDCD004F529
:10E99000005494F9C053023D18BF0125D4E700BFCD
:10E9A000586C002073B500F5804202F6FC5393EDDD
:10E9B000000AD2F8B42D00F5994364339A422BD162
:10E9C00000F50053D3F8FC3BB3F90840003C18BFF6
:10E9D000012400F5A04300F53C5500F58050D3F824
:10E9E0004C64D0F8082593F848343435B61A5BB136
:10E9F0000A488DED010A4FF40061FFF7BBFD9DED64
:10EA0000010A80F00100C3B222463146284602B016
:10EA1000BDE870407CF00ABC0024DAE7582C0020E6
:10EA200010B5044605F070FE98B104F5A042D2F886
:10EA30004C3403F58C415031C2F84C1404F580512C
:10EA4000D1F808150029BEBFA3F58C43503BC2F88E
:10EA50004C342046FFF7A6FFBDE8104004205DF0CF
:10EA600085BB00002DE9F0412DED048B00F500562B
:10EA700096EDFC8ADFED388A28EE288A00F580487A
:10EA8000BDEEC88A00F5A04708F6FC5393ED009A46
:10EA9000D7F8503418EE102A1A4408EE102A05460A
:10EAA00046205DF077FBB8EEC88AD6EDE67AD8F856
:10EAB000B40DA0EE278A05F5994364339842FDEE24
:10EAC000C87A17EE904A44D1D6F8003CB3F90860F2
:10EAD000003E18BF012603685B699847D0B9D8F893
:10EAE000B40D03689B6B9847A0B905F5C043D3F8F4
:10EAF000F430022B0ED1284609F08EFD50B107F6F6
:10EB00006863D3ED007A67EEA87AFDEEE77A17EE38
:10EB1000903A1CB205F5425805F5805508F10C08ED
:10EB2000D5F80C35E41A97F848343BB10B484FF44C
:10EB30000061FFF71FFD80F00100C3B2B0EE490A8B
:10EB4000BDEC048B324621464046BDE8F0417CF0E6
:10EB5000A9B80026BFE700BF0000C842582C00201B
:10EB600010B504460BF0F4FF68B100B200EB4000B2
:10EB7000C0EB001300EE103AB8EEC00ABDE810403A
:10EB800013205DF0F3BA2046FFF76CFFF6E70000B4
:10EB900010B50E48FFF7CEFEB0B10D4C04205DF06D
:10EBA000F9FAD4F8FC0B5CF05BF904205DF0DEFAB6
:10EBB00013205DF0EFFAD4F8000C5CF051F9BDE8D9
:10EBC000104013205DF0D2BA10BD00BF582C0020B9
:10EBD000584C0020F8B52DED028B0446FFF7AAFE35
:10EBE000002800F0838004F5804704F59942D7F8A7
:10EBF000B43D7432934279D004F59A421C32934268
:10EC000074D004F59A42403293426FD004F59A4290
:10EC1000243293426AD004F59A422C32934265D052
:10EC200004F599426C32934260D004F50055F6EE3B
:10EC3000008AD5F8FC0B5BF0D3FFB4EEE80AF1EEE6
:10EC400010FA40DDB0EE087AFFEE007AE0EE077AC7
:10EC5000B0EE670AD5F8142C04F5A04607EE902A0A
:10EC6000D6F84C34B8EEE77A07EE903AF8EEE77A49
:10EC70005142E7EE007AFDEEE77A17EE900AC6F809
:10EC80004C0426F0B7FBC6F84C04D7F8B42D04F5B5
:10EC90009A4368339A4222D0D5F8000C5BF0A0FF6B
:10ECA000B4EEE80AF1EE10FAB0EE408A21DCFEEE96
:10ECB000007AB4EEE70AF1EE10FA22D5B0EE087A47
:10ECC000F7EE007A19E0FEEE007AB4EEE70AF1EE14
:10ECD00010FABFD5B0EE087AF7EE007AB6E725480D
:10ECE0004FF48051FFF746FC0028D5D0BDEC028BD5
:10ECF000F8BDB0EE087AFFEE007AE8EE077AB0EEE3
:10ED0000678A204605F000FD08B1B1EE488AD6F8C2
:10ED10005034D5EDDB6A9FED186A05F6184595ED80
:10ED2000007AB5EEC08A07EE903AF1EE10FACCBF49
:10ED300028EE268A27EE488AF8EEE77A66EE866A9B
:10ED4000E8EE067A27EE067AFDEEE77AFDEEE66A51
:10ED500017EE903ABDEEC77A16EE902A17EE101A0B
:10ED600017EE900AC6F8503426F044FBC6F850045B
:10ED7000BCE700BF582C00200000C84270B5044614
:10ED800004F5804582F04EFAD5F8C43DC31AB3F5B8
:10ED9000FA6F064603D9D5F8B40D06F099FE2E4B4E
:10EDA000C5F8C46DD3F8B40D026813689847002104
:10EDB000204609F0E3FDDFED297AB0EEC00AB4EE9B
:10EDC000E70AF1EE10FA45D504F5BE43D3ED1D7AFE
:10EDD000B1EE047AF0EEE77AF4EEC77AF1EE10FACB
:10EDE00038D504F58C6011F069F8F6EE007AB0EED3
:10EDF000C00AB4EEE70AF1EE10FA2BD504F5B855C7
:10EE000095ED057AF0EE087AB4EEE77AF1EE10FAB5
:10EE100005F114051ED504F53C5034307CF076FA2B
:10EE200004F542500C307BF0EDFF04F547502430E0
:10EE30007CF01AFF95ED007AF7EE007AB4EEE77AEF
:10EE4000F1EE10FA06D504F54D501830BDE87040CB
:10EE50007CF060BC70BD00BF586C00200000003426
:10EE600000F5005090F94B33012BC3BF00F54B6008
:10EE700090ED290ADFED047A9FED040AC8BF20EE69
:10EE8000270A46205DF072B90000C8420000000069
:10EE90002DE9F8432DED028B00F5804909F6FC536E
:10EEA000D3ED008A054609F0D9F98046D9F8B40DAA
:10EEB00003681B6A984705F54756243698B14F4CAE
:10EEC000D4F81034002B0EDD82F0ACF9D4F81034F5
:10EED000C01A40F6B733984205D8B4F90444304616
:10EEE0007CF0CEFE7AE005F5C04305F5005793F8B7
:10EEF000E93043B1B7F9DC33002B04DD05F54053AD
:10EF000093F9FA3103BBD9F8B43D05F59945643559
:10EF1000AB426DD00021B0EE680A30467CF048FC70
:10EF2000054604205DF036F92BB207EE903A97EDD6
:10EF3000E47AF8EEE77AE0EE077AFDEEE77A17EE8C
:10EF4000904A444424B2CAE72846012109F05AFBFA
:10EF50009FED2B7AB7F9DC33C0EE077A05F5A045B3
:10EF600005F58B6508EE103A55F80C3C9FED250A27
:10EF7000B8EEC88A28EE278A07EE903AF8EEE77ACC
:10EF800067EE807A9FED200A27EE800AA6F042F80D
:10EF9000B7F95433DFED1D7A95ED007A20EE270A9C
:10EFA00007EE903AF8EEE77A0021B4EEE77AF1EE58
:10EFB00010FA58BFF0EE477A80EE277A3046DFED40
:10EFC000147AB0EE480AA7EE270AF0EE680A7CF041
:10EFD0004BFDBDEEC00A10EE103A1CB2BDEC028B28
:10EFE00020460C49BDE8F84341F2941226F012BACB
:10EFF000B8F1000118BF01218DE700BF587C002047
:10F0000000A08C450AD7233C35FA8E3C0AE81C4107
:10F01000E02E65426CEEFFFF38B500F54053054623
:10F02000D3F8E8050368DB689847014605F54D50BD
:10F0300018307CF051FB04B22846FFF77BFC70B11E
:10F0400007EE904A05F50055B8EEE70AD5F8080C2A
:10F050005BF006FFBDEEC00A10EE103A1CB220466F
:10F060000349BDE8384041F2941226F0D3B900BFFD
:10F070006CEEFFFF38B590F81434B02202FB0303A6
:10F0800093ED837AF7EE007AB4EEE77AF1EE10FAB8
:10F09000044600F5A0451CD5002109F06FFCDFED0A
:10F0A000407AB0EEC00AB4EEE70AF1EE10FA10D5DD
:10F0B000D5F83834012B0CD0072B0AD0002385F863
:10F0C000A8330023C5F8AC332046BDE8384009F02A
:10F0D000C5B882F0A7F8D5F8B033C5F8B003C31AA5
:10F0E000B3F57A7F84BF002385F8A833204609F062
:10F0F000B5F8D5F83834012B07EE100A2DD0072BC0
:10F100002BD0B8EEC77ADFED276AC7EE267A04F572
:10F110000052B2F9A02300EE102AB8EEC00A27EE82
:10F12000800ADFED1F7AB0EEC07AB4EEE77AF1EE36
:10F1300010FA14D4002385F8A83395F8A83304F501
:10F140004D501830D3B97CF0AFF9BDE838401649BE
:10F1500000B241F2941226F05DB99FED140A95F8C1
:10F16000A823002AE9D10122934285F8A823E4D0FC
:10F17000072B1CBF0023C5F8AC33DEE795EDEB7A17
:10F18000DFED0B7A67EEC77A9FED0A7A67EE877A32
:10F19000FDEEE77A17EE901A7CF09EFAD5E700BFF5
:10F1A0000000003400A08C456CEEFFFF0000000062
:10F1B000E02E65420000C84270B52DED028B00F5CF
:10F1C000BC46103682B0054630467FF0D7FD044677
:10F1D000D8B905F50052D2F8FC3BB3F9083073B941
:10F1E00005F5BE43D3ED1D7A92EDE77AF0EEE77AAE
:10F1F000F4EEC77AF1EE10FA4CBF01240024304639
:10F200007FF0D0FD002808BF002430467FF0B6FD17
:10F2100028BB05F5A043D3F8A433013319D0F4B9C2
:10F220009FED1A8A2846FFF733FE07EE900AB8EEE4
:10F23000E70A8DED010AD4B915205CF097FF9DED2A
:10F24000010A1A2002B0BDEC028BBDE870405CF0F0
:10F250008DBF002CE4D02846FFF70CFF02E02846C3
:10F26000FFF7DAFE07EE900AB8EEE78ADAE71A202F
:10F270005DF01EFA9DED010A08B9B0EE480A1520AE
:10F280005CF074FFB0EE480ADBE700BF000000004E
:10F2900010B500F5005303F61842D3EDDB6ADFED3D
:10F2A000127A92ED007A9FED116A03F54B6366EED8
:10F2B000A76A27EE277AD3ED2A7A67EE867AFDEEE3
:10F2C000E66ABDEEC77AFDEEE77A044616EE902AAE
:10F2D00017EE101A17EE900A26F08CF804F5A044E9
:10F2E000C4F8500410BD00BF0000C842A00CB345D4
:10F2F00010B504460BF084F8031E2ADB04F5005118
:10F3000091F94B239A4224DD04F5A040D0F838440B
:10F31000022C1ED0D1EDE97ADFED0E6AD31A66EE2B
:10F32000E76A07EE102A07EE903AB8EEC77AF8EED1
:10F33000E77AD0F8503487EE876A07EE903AF8EE15
:10F34000E77AE6EE867AFDEEE77A17EE903AC0F8B5
:10F35000503410BD0000C842F8B52DED028B00F509
:10F36000A0459FED440AD5F84C349FED437A07EE53
:10F37000903AF8EEE77A044667EE807A9FED3F0A0E
:10F38000F0EEE76AF4EE476AF1EE10FAC8BFF0EE6D
:10F39000477A27EE800AA5F07DFC25F0ADFEB7EE9A
:10F3A000008AC8EE007A05F2544704F50056C7ED0E
:10F3B000007A96F97C3353B3204605F0A5F930BBAB
:10F3C000B6F95433012BB8BF012307EE903A05F587
:10F3D0008B62F8EEE77AD2ED006A86EEA77AB4EE99
:10F3E000C87AF1EE10FA15D840F6C4122449D5F8BF
:10F3F0004C0425F0FFFFC5F84C04D6F8142C40F659
:10F40000C4139A42D4BFC6F8142CC6F8143CBDEC01
:10F41000028BF8BDD7ED007AB4EEE77AF1EE10FA80
:10F42000F5D588EE070A20EE000AA5F01DFEDFEDF7
:10F43000157AD5F84C0420EE270ADFED137A20EE7A
:10F44000270A40F6C413FDEEC07A17EE904A9C429C
:10F45000B8BF1C462246614225F0CCFFC5F84C04DB
:10F46000D6F8143CA342D4BFC6F8143CC6F8144CDA
:10F47000CDE700BF0AD7233C0000AA4235FA8E3CF4
:10F480003CF6FFFFE02E65420000C84210B500F5D3
:10F4900040530446D3F8E80503681B68984704F511
:10F4A0000053D3F8142C514225F0A4FF04F5A043D7
:10F4B000C3F84C042046BDE81040FFF74DBF0000E4
:10F4C00070470000012070470820704701207047F6
:10F4D00070470000014B93F888037047584C002098
:10F4E000034B93F9980B003818BF0120704700BFF9
:10F4F000584C0020014B93F98A037047584C002068
:10F5000013B5064BD3F8B40D4B690468009308316A
:10F510000EC9646CA04702B010BD00BF586C00203B
:10F5200070470000002070477047000038B5254D37
:10F53000D5F8B40D03685B6898470F2834D80F28B6
:10F5400039D8DFE800F00836080808080808083845
:10F5500036363636363610241B4B93F8B92312B1A3
:10F5600093F8B8330BB944F01004184BD5F8B42D08
:10F570009A42A3F1080303D09A4218BF44F0100442
:10F58000134991F9FD13C1B19A4218D0032902D150
:10F59000104B9A4201D144F040040F4879F090FE9C
:10F5A00068B144F080040AE0182814BF012418242C
:10F5B000D2E71824D0E70124CEE79A42EDD144F0F7
:10F5C000010038BD586C0020585C0020DC79002018
:10F5D000584C0020A07900209C8C002008B50448DD
:10F5E00005F0D6FD00280CBF0120022008BD00BF99
:10F5F000582C0020F0B52DED028B8BB005460EF097
:10F6000089FA4FF48071D0F8047290ED828AD0F8B4
:10F610000C6204461448FEF7ADFF30B9134BDFED22
:10F62000147A93EDFC7AA7EE678A2D7C81F0FAFDBF
:10F63000D4F81823D4F81C33D4F81413089209937F
:10F6400027221C23CDE900320390079103AA1E2133
:10F65000284604978DED058A069653F007FE0BB0F9
:10F66000BDEC028BF0BD00BF582C0020584C002090
:10F6700035FA8E3C2DE9F0432DED068B414ED6F840
:10F68000B42D06F684539A428BB075D006F5805996
:10F69000A6F5805390F81080D3F8E875D9F84C346B
:10F6A0009FED399A07EE903AD9F85034B8EEE7AAB0
:10F6B00007EE903A3B6838469B68F8EEE79A984721
:10F6C00007EE900AF8EEE77A384667EE897A2AEE76
:10F6D00009AAFDEEE77A69EE899A17EE903A1DB213
:10F6E0003B681B69984707EE900AF8EEE77AD9ED78
:10F6F000F38A67EE897AA6F58040FDEEE77A06F692
:10F70000E85617EE903ADFED217AF4EEE78AF1EE53
:10F7100010FA58BFF0EE678A1CB202F045FE3B6853
:10F72000D6ED00AADFED1A7A5B6908EE100A3846BA
:10F730006AEEA7AA9847FCEEE88AB8EEC88A18EEE7
:10F74000903AB72228EE098AADF824301A23CDE981
:10F7500000323E2103AA40468DED03AACDED049A66
:10F760008DED058ACDED06AA8DED070AADF8205086
:10F77000ADF8224053F07AFD0BB0BDEC068BBDE82E
:10F78000F08300BF586C00200AD7233C00FF7F475E
:10F790000000C84208B502480AF032FE00B208BDB7
:10F7A000582C002055F024B837B50D46134840F2C8
:10F7B000EF2203F04BFB2C7814F004040AD06968A4
:10F7C00003220F4814F0AEF90C4803B0BDE83040F6
:10F7D00002F0FCBC01AA2146284614F077FA002862
:10F7E000F2D0DDED017A9FED077A67EE877A224647
:10F7F000FDEEE77A17EE901AE3E700BF582C0020E1
:10F80000A08B00200000C84210B5054C012384F8ED
:10F81000BB3355F02DFA002384F8BB3310BD00BF75
:10F82000585C002058F0C8BC2DE9F0412DED028B4A
:10F830004FF0000882B0CDE900281E4F9FED1E8AD0
:10F840000C461546B0EE480AB1F90220D7F8FC1B69
:10F850004FF47A73064658F097FF0123CDE9005321
:10F86000B4F90020D7F8001CB0EE480A30464FF437
:10F870007A7358F089FFB4F90420D7F8041C9FED7F
:10F880000F0A43463046CDE9005858F07DFFCDE9D8
:10F890000058B4F90620D7F8081CB0EE480A4FF417
:10F8A0007A73304658F070FF02B0BDEC028BBDE8B1
:10F8B000F08100BF584C00200000FA4400007A4458
:10F8C00038B5C5780B46352D044628BF3525352279
:10F8D00000211846A7F026FE2A4604F10C01BDE8D7
:10F8E0003840A7F0D5BD000010B5074B93F974253B
:10F8F00040F24D3440F24D13002A08BF1C4654F02C
:10F90000FFFF204310BD00BF587C002010B5044607
:10F9100014F00CFD204610BD10B50C4C002384F8EB
:10F92000E73355F09FFEA4F58052A4F52E73D2F86C
:10F93000B42D9A4208D194F860342BB904F25C409B
:10F94000BDE810402BF080BA10BD00BF587C0020ED
:10F9500013B5124C94F8861104F138000BF038FE00
:10F9600078B194F8861104F138000CF09FF840B19A
:10F9700094F8861104F1380002B0BDE810400CF094
:10F98000D7B80EF0C7F801A90DF0A8FE18B19DED8B
:10F99000010A02B010BD9FED020AFAE7584C0020A0
:10F9A0000000000008B51248D0F8B42D00F67C53D2
:10F9B0009A4216D0B0F9CC3DABB900F5805393F81C
:10F9C000712382B990F8C92D6AB993F8213463B9CB
:10F9D000A0F5804005F0DCFB00280CBF03200420CC
:10F9E00008BD0220FCE70520FAE70620F8E700BF83
:10F9F000586C002010B5224B03F68452D3F8B43D66
:10FA0000934290B0044638D000231E48029314F06D
:10FA100073F8014618B91B4802AA14F0B9F8247CFF
:10FA200081F000FC184BDDED027AD3F8502FD3F8AB
:10FA3000543F05930023F8EEE77A9FED147A07937D
:10FA4000089309930A930B930C930D930E934FF61F
:10FA5000F853ADF83C300023CDE9030267EE877A16
:10FA600096228DF83E303323CDE90032572103AA88
:10FA70002046CDED067A53F0F9FB10B010BD00BF63
:10FA8000586C0020A08B0020587C00200AD7233C13
:10FA900010B555F02FF9044688B90A48A0F58052F0
:10FAA000A0F52E73D2F8B42D80F8E7439A4206D120
:10FAB00090F860341BB900F25C402BF0C5F9204689
:10FAC00010BD00BF587C00200120704708B5034BD3
:10FAD000D3F8B40D03685B68984708BD586C0020E4
:10FAE00030B587B005460EF015F804462D7C81F040
:10FAF0008DFBD4F88422D4F8883204920593002137
:10FB00001023CD22CDE900320290039102AA42F6E1
:10FB10000C31284653F0AAFB07B030BD30B52DEDAF
:10FB2000028B89B005460DF0F5FF00F55A7393E896
:10FB3000070002AC84E80700DDED020A9DED030A30
:10FB40002D7CF1EE600AB1EE400AA5F0F5FA2046F0
:10FB5000B0EE408A28F030FADFED0B7A049B079371
:10FB600028EE278A0C230122CDE90032A82105AA1C
:10FB700028468DED058A8DED060A53F077FB09B016
:10FB8000BDEC028B30BD00BFE02E6542282938B5A0
:10FB9000054623D007D824292BD0272911D01B298B
:10FBA00008D1012413E0432937D008D84029F8D0E0
:10FBB000422928D02846BDE8384058F041BF532993
:10FBC000EEE7122152F050FD044610B90024204601
:10FBD00038BD297C13484BF083FCF8E7162152F01E
:10FBE00043FD04460028F1D0297C0E484BF052FD1D
:10FBF000EDE70C2152F038FD04460028E6D02846F7
:10FC0000FFF78CFFE3E7102152F02EFD0446002899
:10FC1000DCD02846FFF764FFD9E7017C02487FF07B
:10FC2000ABF8BEE7CC810020688A0020F0B52DED4E
:10FC3000028B05468DB01646B0EE408A0C46002970
:10FC400030D0007C53F0A8FA0746287C54F0A8F97D
:10FC500000F121039F4207D2287C0DB0BDEC028B3E
:10FC6000BDE8F04052F0EEBC63690893636A226914
:10FC7000CDF82530236AA069E1680792CDF82930D4
:10FC80006222212327680590CDE900320691287C65
:10FC90000397192303AAC2218DED048A8DF82460ED
:10FCA00053F0E4FA0DB0BDEC028BF0BD70B52E49F7
:10FCB000D1F8B42D01F684539A42044652D0A1F5EE
:10FCC0000055B5F82E34DE0708D5A1F5805393ED25
:10FCD000180A0122A1F6A471FFF7A8FFB5F82E3487
:10FCE000980708D52149022291ED6F0A204601F5B7
:10FCF000DC71FFF79BFFB5F82E34590708D51B4977
:10FD0000032291EDCC0A204601F54B71FFF78EFFDF
:10FD1000B5F82E341A0708D51449052291EDE30AE7
:10FD2000204601F56271FFF781FFB5F82E34DB063E
:10FD300018D50F4ED6F83834042B13D10DF0EAFE47
:10FD4000054606F561607FF047F895EDC70ADFEDDF
:10FD5000097A014620EE270A20460622BDE87040B7
:10FD6000FFF764BF70BD00BF586C0020585C0020D6
:10FD7000587C0020E02E654270B504460E461DF00A
:10FD80003DFC90F8F412B02303FB0101DC31204666
:10FD900003F0C8F9054698B13EB10DF0BBFE90F8EE
:10FDA0007C3243F0020380F87C3204F5804304F592
:10FDB0009A44D3F8B40D6034A04201D105F0D4FDCB
:10FDC000284670BD73B51646019104460DF0A2FE9B
:10FDD00001990DF0EDFA054698B13EB10DF09AFE8D
:10FDE00090F87C3243F0020380F87C3204F58043C3
:10FDF000D3F8B40D04F59A436033984201D105F06D
:10FE0000B3FD284602B070BD30B5054685B00C463E
:10FE1000D1E9040125F0B8FC40B1684613F07CFE3E
:10FE20006A462146284658F01FFC08B9022067E0C0
:10FE3000344840F24F32694603F008F8D4ED037AB3
:10FE4000F4EE677AF1EE10FA22D69FED2F7AF0EEFB
:10FE5000E77AF4EEC77AF1EE10FA54BF01220022DD
:10FE60009DF80030294962F3410368468DF800305F
:10FE700013F0BCFF0028D9D12548694668F008FE78
:10FE800040B94FF011F9052216214EF0C5FECDE71D
:10FE90000022E5E7D4ED017AFDEEE77A17EE903A1D
:10FEA000DB0706D41B4B03F55762D3F8B43D9342EE
:10FEB00025D11949134802220AF0B6F89DF800101E
:10FEC00011F0040102D1684613F0F0FE0D486946B6
:10FED00003F076F894ED020AB4EE400AF1EE10FA5F
:10FEE0000BD6B5EEC00AF1EE10FA06DD9DF8001053
:10FEF0000948C1F3400106F09BFD002000E004200A
:10FF000005B030BD582C002000000034908B00203C
:10FF1000484E0020586C0020C879002010B52DED07
:10FF2000028BD1ED017A91ED008AFCEEE77A8AB07E
:10FF3000CDED037A9DF80C1005AA044658F07EFB1F
:10FF4000C8B1DFED0E7A059B009368EE277A002298
:10FF5000FDEEE77A114617EE903A06A813F0FCFD85
:10FF600023682046D3F8CC3006A9984700200AB071
:10FF7000BDEC028B10BD0220F9E700BF0000C842B3
:10FF800037B5124DD5F8B40D03681B6A0C46984777
:10FF900040B9D5F8B42D05F648539A4202D0042052
:10FFA00003B030BDD4ED007AD4ED020A94ED010A1D
:10FFB0000748FCEEE77ACDED017A9DF8041003F0D6
:10FFC00051FE0028EBD00020EAE700BF586C00206B
:10FFD000582C002008B5D1ED007A9FED087A08482A
:10FFE000F0EEE77AF4EEC77AF1EE10FA54BF012191
:10FFF000002104F083FB002008BD00BF0000003496
:020000040801F1
:10000000582C002010B5D1ED007AFCEEE77A17EEFF
:10001000903A9CB2012C02D0022C06D084B911482F
:10002000214663F093FF002010BD0F4890F868351B
:100030005B0707D558F0B2FF0C4A052152F0E2F8F1
:100040000420F1E790F954351BB958F0A7FF084A8E
:10005000F3E7A0F5A04007F0C3FF002814BF00207D
:100060000420E1E7AC810020587C002048C20B0846
:1000700063C20B0838B58B8BC02B05460C4631D8B4
:10008000B12B0BD8112B00F09680142B00F096802A
:1000900021462846BDE8384059F0C4BDB23B0E2B7E
:1000A000F6D801A151F823F01701010891000108C9
:1000B00091000108910001089100010891000108D8
:1000C00091000108910001080D010108910001084B
:1000D000310101086D0101089100010821010108A9
:1000E00003010108D42B08D0B3F5967F49D0D02B5B
:1000F000CED1BDE83840FFF785BFBDE83840FFF7F7
:1001000069BF2146BDE83840FFF77EBE2146BDE805
:100110003840FFF703BF2146BDE83840FFF730BF46
:1001200094ED000A2848FEF711F8E8B100201CE021
:10013000264C94F8DD3DBBB12549A1F6DC202AF020
:1001400081FF88B104F58053012283F8952404F6D9
:1001500048510222A4F5804009F066FF0028E5D14D
:100160001C4B002283F89524042038BD174C94F8CA
:10017000DD3D002BF8D01649A1F6DC202AF0E6FE82
:10018000DFE7D1ED007A9FED147AF0EEE77AF4EE36
:10019000C77AF1EE10FA14D5D1ED017AF0EEE77AD4
:1001A000F4EEC77AF1EE10FA0BD50C49022206489C
:1001B00009F03AFFBAE70A490222F8E709490222A0
:1001C000F5E70220D1E700BF582C0020586C002032
:1001D000908B0020587C002000000034A079002083
:1001E000C0790020B879002070B5424B03F5576202
:1001F000D3F8B43D93428EB00C4679D1CD78272DFB
:1002000028BF27252722002104A8A7F08BF92A461A
:1002100004F10C0104A8A7F03BF9059B9DF83640BA
:100220000093069B0193E443079B0293E4B2089B6F
:1002300003938DF8364080F0F5FF14F0810F04F041
:100240008705064601D1802D11D1684626F032FE81
:10025000DFED297A294B20EE270ADFED297AC3F852
:10026000086420EE270ABDEEC00A83EDFF0A14F0F1
:10027000820F01D1802D13D1684626F035FEDFEDC7
:100280001E7A1E4B20EE270ADFED1D7AC3F80C64A0
:1002900020EE270ABDEEC00A10EE102AC3F8002493
:1002A00014F0840F01D1802D13D1684626F02CFE66
:1002B000DFED117A114B20EE270ADFED117AC3F83A
:1002C000106420EE270ABDEEC00A10EE102AC3F813
:1002D000042463060CD5DDED0C7A9FED097A074BFB
:1002E00067EE877A03F21442C2ED007AC3F818640D
:1002F0000EB070BD586C0020E02E6542587C002086
:100300000000C84230B5214C91B0084602A9FFF761
:10031000D7FAD4F8B42D04F557639A4233D19DF837
:100320003C30072B2FD104F58054DDED056AD4F85D
:100330004C3F9FED177A07EE903AF8EEE77AE6EE3B
:10034000C77AFDEEE77A17EE903AC4F84C3F58F0C2
:1003500025FED4F8242FD4F84C3F52689FED0D7A37
:100360009B1A07EE903AF8EEE77A054667EE877A31
:1003700017EE900AFCF7C8F8074ACDE900010621FC
:10038000284651F03FFF11B030BD00BF586C00202F
:100390000000C8420AD7233C7CC20B0810B51D4B95
:1003A00003F55762D3F8B43D9342044696B008462D
:1003B0000FD108A9FFF784FA9DF8541003AA20462C
:1003C00058F03CF938B958F0E9FD134A042151F0CE
:1003D00019FF16B010BDBDF8503023F004039BB2D6
:1003E000002BF6D0DDED0B7A9FED0C7A039B00938A
:1003F00067EE877A0022FDEEE77A114617EE903A13
:1004000004A813F0A9FB236804A9D3F8CC30204634
:100410009847DEE7586C002090C20B080000C842E5
:1004200030B48D7A4B7A43EA0523CD7A43EA05430B
:10043000562B04460A461BD008D8522B12D0542BF8
:1004400013D02046114630BC58F0C8BD03F180736C
:10045000863B23F07F43012BF3D8017C064830BC58
:100460004BF0E0B930BCFFF7BFBE30BCFFF74ABF6E
:1004700030BCFFF793BF00BFCC8100200020704745
:10048000C820704701207047002070470020704747
:1004900090F89C308B4286BF283150F82100002014
:1004A0007047000090F89C308B4286BF283150F88E
:1004B000210000207047000003207047014B93F893
:1004C00086037047584C002070B504464C4808F02D
:1004D0004FFA18B1E36A43F40003E362484808F0B6
:1004E00047FA88B146205BF055FEDFED467AB4EE60
:1004F000E70AF1EE10FA07D8236B43F400032363F5
:10050000636B43F400036363E36A43F4F843E36219
:100510003D4BD3F8B40D03685B6898470138172842
:1005200014D8DFE800F03A420C4442424242133A07
:100530003A3A3A3A3A13131313131313133A334A4A
:1005400092F8B8338BB392F8B9238AB3304B93F84F
:100550000C3E012B3DD0022B44D02E4B1D68DDB14B
:100560002D4E284696F8F21B47F014F8A0B1E36A26
:1005700043F48073E36296F92C341BB1236B43F48C
:100580008073236396F8F21B284647F03BF818B1B6
:10059000636B43F48073636370BDD4E90C2342F44E
:1005A000E04243F4E04322636363012300E000235D
:1005B000216B41F480622263626B42F4806060636D
:1005C000002BC3D041F4406142F440622163626376
:1005D000BCE7E36A43F48003E362236B43F48003E4
:1005E0002363BAE7E36A43F48003E362236B43F4D3
:1005F00080032363636B43F480036363ADE700BF51
:10060000582C0020000000B4586C0020585C0020DA
:10061000587C0020B88E0020584C002013B54FF4B1
:100620004470CDE9002113F079FE044628B1DDE9DC
:10063000002158F0F3FE024B2360204602B010BDAB
:1006400090C40B08002070470020704700207047BE
:100650000020704700F50F50283070470048704761
:1006600018EA0B0800F58040D0F8B40D03685B6809
:100670001847000000F5804300F59A40D3F8B43DD8
:1006800048301B1A58425841704700009B20704761
:1006900030B500F5A04303F58A6353F8042CDFED71
:1006A000296A07EE902AB8EEE77AD3ED007AF8EEE1
:1006B000E77A85B0044627EE267A67EEA67A00F53B
:1006C0009850002301A9103003938DED017ACDEDF0
:1006D000027A04F57F650BF0FFFB04F541521C32F2
:1006E000692128464DF0ACFB04F5465238326A21A8
:1006F00028464DF0A5FB04F5405393F9FA2132B991
:10070000D3ED7C7AF5EEC07AF1EE10FA06DD04F551
:100710004C522C326B2128464DF092FB04F54D547F
:10072000183420467AF0FAFF28B104F130026D2126
:1007300028464DF085FB0DF0EDF90CF035FF05B0C6
:1007400030BD00BF0AD7233C10B54FF480110446DA
:1007500009F052FE10B12046FFF79AFF4FF48001D6
:10076000204609F049FE28B124F06CF8BDE810409D
:1007700022F02CBA10BD000030B500F5985591B0AC
:1007800000231035029302A9002304460DF107024D
:1007900028468DF807300CF0A7FF03A928460BF078
:1007A000F7FF08B92D4B03933022002104A8A6F0CF
:1007B000B9FEA3238DF8103095238DF8113080F009
:1007C00039FD04F5A042CDF81300D2F84C34ADF851
:1007D0001B3004F58053D2F85024CDF81710462072
:1007E000D3F80815D3F80C35ADF81D10ADF81F205F
:1007F000ADF821305BF0CEFC10EE103A1520CDF8AC
:1008000023305BF0C7FC10EE103ACDF8273004F52A
:1008100032539FED137AD3ED357A67EE877A284607
:1008200017EE903ACDF82B30029BCDF82F309DF883
:1008300007308DF83330039B0D930DF05BF904F511
:1008400080433022D3F8F03D8DED0E0A04A904F563
:100850007F600F934DF030FC11B030BD2292CA7F03
:100860000000C84270B58EB03522044600216846AB
:10087000A6F058FEA3238DF8003095238DF80130A3
:1008800001238DF8023080F0D5FC04F5A04504F575
:100890004056D5F8CC33CDF80300D6F8E805CDF8AE
:1008A0000710CDF80B3003681B699847ADF80F00AF
:1008B000D6F8E80503689B689847ADF811001E4814
:1008C00001F072FDADF81300D6F8E80503685B6926
:1008D000984710EE103AD6F8E805CDF815300368C1
:1008E0009B69984710EE103ACDF8193004F5804313
:1008F00003F6E85135220968CDF81D10D5F8501FD0
:10090000CDF82110D5F8541FCDF82510D5F84C1F7F
:10091000CDF8291004F5C041D3F8E03DD1F8FC1022
:10092000CDF82D1004F57F606946CDF831304DF0DB
:10093000C3FB0EB070BD00BF582C002030B587B08F
:100940001622044600216846A6F0ECFDA3238DF88C
:10095000003095238DF8013002238DF8023080F0AD
:1009600069FC04F5A045CDF803002046CDF807103A
:1009700004F00EFC05F23C438DF80B001B6803935A
:10098000124B1B68D86A90F89C308DF810300368C1
:10099000DB69984795F821348DF812308DF81100F5
:1009A00023F050FF23F09EF8D5F838348DF813006B
:1009B0008DF81430162295F822348DF815306946DA
:1009C00004F57F604DF078FB07B030BD542C00205B
:1009D00010B58AB02722044600216846A6F0A2FD81
:1009E000A3238DF8003095238DF8013009238DF86D
:1009F000023080F01FFCCDF803000420CDF8071072
:100A00005BF0C8FB10EE103A1320CDF80B305BF012
:100A1000C1FB10EE103A4620CDF80F305BF0BAFB68
:100A200010EE103A1520CDF813305BF0B3FB10EE4A
:100A3000103A0320CDF817305BF0BCFB10EE103AF3
:100A40001A20CDF81B305BF0A5FB10EE103ACDF864
:100A50001F3004F59B437C3327221B68CDF82330DD
:100A6000694604F57F604DF027FB0AB010BD000019
:100A700013B5044600F57F6001904CF04FFE0198DD
:100A80004CF0E6FE04F58053019893F920310BB148
:100A90004CF086FF204602B0BDE81040FFF798BF3B
:100AA0007047000010B500F580430446D3F8B40D3C
:100AB00003685B68984704F50053014693F80823E0
:100AC00004F57F604DF0B8FC04F5985010300DF03F
:100AD0006DFA04F59070BDE810401BF0F9BD000000
:100AE0009FED020A002245F023B900BF0AD7233C3C
:100AF000184B70B5044640F8043B59F0C1FD164E42
:100B0000164B63605425601959F070FF66513035FB
:100B1000B5F5557FF7D104F555705BF02FFF04F262
:100B20007C75FF2384F88C3784F894370C49284669
:100B300045F00EFB0B4B1A6812B10B4880F040FBDE
:100B40001D6001232046094984F8C13745F000FBA8
:100B5000204670BDC8380020B0140C08C4140C081E
:100B6000E87C0D088498002088010C08AC040C086F
:100B70002DE9F04100F50E519AB00D2204310446E2
:100B80004BF084FE0022BF48BF4E272145F048F8B5
:100B9000042100205BF0CCFE132101205BF0C8FE95
:100BA000462102205BF0C4FE152103205BF0C0FE4D
:100BB0005BF02AFC45F0D2FCB44A138843F00403EE
:100BC00013804FF000080AAF002110223846A6F02B
:100BD000A9FC01238DF830303388ADF8283005A901
:100BE00073680B93384644F023FFC8B19DF9143065
:100BF000002B15DD59F0C4FE9DF81410036801396F
:100C00001B68C9B2984758B1051D284644F05AFEE2
:100C100030B9B368ADF8183006A9284646F03CF95B
:100C200008F10608B8F12A0F06F10C06CCD1984855
:100C300000220DF10B0144F02DFC06AD064620B359
:100C400044F040FE08BB934B0FCB85E80F0004A98E
:100C5000284644F0EDFE002840F03C814FF00408A7
:100C60008D4B0FCB87E80F0005A9384644F0E0FE16
:100C700028B105A844F026FE08B148F0010803A9F0
:100C800030468DF80C8046F0B5F8844B0FCB85E8E4
:100C90000F0003A9284644F0CBFE002846D009984F
:100CA000002204A944F0F6FB064600283ED044F09A
:100CB00009FE0546002839D19DF80C30013BDBB216
:100CC000032B96BF764A0346D35C8DF82830304616
:100CD000394646F08FF87348002205A944F0DAFB44
:100CE000064668F017F978B168F012F990F83020EC
:100CF00090F8281090F84830114490F840200A44A9
:100D0000D34214BF0125002586B130469DF90C80E1
:100D100044F0D8FD50B91DB1B8F1000518BF012548
:100D2000394630468DF8285046F064F804F51050E6
:100D30000022B7EE000A0121203044F0F9FF04F54B
:100D40000E500022B7EE000A02213C3044F0F0FFC2
:100D5000012304F500510093534A002338318E20BB
:100D600044F062FF94F9A4C9BCF1000F1AD14F4EB0
:100D70000FCE3D460FC50FCE0FC50FCE0FC596E85F
:100D80000F0085E80F0062460421384644F048FF12
:100D90009FED470A474845F07BFD4748B7EE000AFC
:100DA00045F076FD012504F50751444A00950023DE
:100DB000303140F2051044F037FF04F50F500221A6
:100DC0003030FFF78DFE04F50D5003211830FFF78A
:100DD00087FE04F50D5003212030FFF781FE04F556
:100DE0000F5003212C30FFF77BFE04F50F5002213A
:100DF0003430FFF775FE04F50D5002212C30FFF75B
:100E00006FFE04F50D5002213030FFF769FE04F546
:100E10000D5002212830FFF763FE04F5BC4010306E
:100E20007EF040F9264A1368D90709D42549156090
:100E300004F5065318330B6004F588530433CB6074
:100E400004F510501F4902223030012544F03EFFC6
:100E50001D4A0095002304F57F61FD2044F0E4FE67
:100E60001A4B1A68D20705D4194A1D6004F591542B
:100E7000143414601648012144F044FF1AB0BDE850
:100E8000F08100BFE8010C0858040C08948E002083
:100E9000AC010C0850B70B0860B70B0870B70B0813
:100EA000E4010C08B7010C08A4280C0880B70B0853
:100EB00000000000C4010C08D3010C081C780D08C8
:100EC0004C2C0020002200208CB90C08502C002053
:100ED0001822002004A844F0F5FC00283FF4BEAE20
:100EE0004FF00C08BCE600BF0020704700207047A0
:100EF00000207047002070470020704770470000B6
:100F0000002070470020704784B001A880E80E00E0
:100F100004B00020704700000020704770470000B8
:100F20001020704700487047D4100C0800487047E4
:100F3000E4100C0800207047704700000120704743
:100F40000120704700207047002343608360C36026
:100F500003614361002303767047000010B5044627
:100F6000FFF7F2FF0023637610BD0000027E531CE2
:100F7000DBB2042B037600EB820288BF002382EDF4
:100F8000010A88BF0376704710B50446FFF7EEFFED
:100F9000D4ED017A9FED107A94ED020A637E77EE2C
:100FA000877A042B77EE807A94ED030A94BF01339D
:100FB000052377EE807A94ED040A637677EE807AE3
:100FC000637E94ED050A77EE807A00EE103AB8EE73
:100FD000C00A87EE800A10BD0000000003F016BEB4
:100FE00003F038B803F082BA03F042B801F09ABCBB
:100FF00001F022B801F0C0B901F006BAFDF7B8BBA4
:10100000FDF74CB870B51F4B036000F54053044624
:10101000D3F87C051C4AC3F8C02308B113F08AF941
:101020001A4B236004F5805393F8D42F42B9D3F8B8
:10103000D05F2DB1284620F051FE284613F076F9F6
:1010400004F59050183077F097FB04F589505CF068
:1010500013FF04F6F44504F69446B54204D0183D57
:10106000284620F091FAF8E7094BC4F8C83804F68E
:10107000C41050F0B1F904F5136050F0ADF92046FA
:1010800070BD00BF10F80B0880D40C088CB20C089F
:10109000F87A0C0838B54C4B044640F8043B61F034
:1010A0003FF904F1100010F08BF904F1680049F0E9
:1010B0004FFB04F590701AF0C5FE04F58C600EF03D
:1010C000D3FE04F2845013F037F904F6C80021F07F
:1010D00069FE04F5476060F001FF04F5546046F0D6
:1010E0007FF904F57F604CF01BFF04F58850043055
:1010F00066F04AFE04F589505CF0A6FE04F58A50BD
:101100001C3011F0BDFE04F59050183077F020FB34
:1011100004F59150143049F0DDFE04F59450083088
:1011200062F0DCFA04F580530025284A83F8AC52BB
:1011300004F5955004F595530C331C30136041F0C1
:101140001FF904F59850294610300BF009F804F502
:10115000CB5071F085FB04F5F350043074F02AFB9A
:1011600004F5FB501C3076F04DFC04F5FF5077F091
:1011700083F804F5005038300AF02AF904F50650D7
:10118000183072F0E5F804F50750303067F098F940
:1011900004F50A50303077F077FE04F5005304F57B
:1011A0000C5083F808530A4D203077F08FFF2B68DE
:1011B00013B1084880F004F82046074944F0C8FFFE
:1011C0002C60204638BD00BF8CB20C08EC97002084
:1011D000F08E0020EC100C0894B10C082DE9F04FB3
:1011E0002DED028B04469FB0FFF754FFE54B2360C3
:1011F00004F510503030FFF77BFC04F52F503430ED
:1012000004F5005779F016FB04F50F530E33C7F8B9
:101210001C3C04F53150062387F8203C08305CF074
:1012200025FA04F5BC431033C7F8C83C0E934FF4BD
:101230000063C7F8CC3C5A2387F84C3D04F50D58A1
:1012400007F54B6304F5985608F10808CE4ADFED20
:10125000CF8AC7F8C48C1036C7F8C06CB7EE008AC6
:10126000C3F8602104F53A50C94AC3F86821C3F8AD
:10127000CC2183ED578AC3ED598A0C3050F0CCFB5A
:1012800004F53A5004F5325A183050F0C5FB4FF0CF
:101290000009C04BC7F8A83E0AF1300A87F8C09E83
:1012A0000AF5FC70FFF750FEBB4BBC49C7F8A83EDF
:1012B00087F8C19E504644F04BFFB94BC7F8C83E73
:1012C00007F6C8630022C7F8CC6EC7F8D0AE04F5A5
:1012D0003B555A63DA6304F53C50012387F80C3F11
:1012E0000835203012F018FC87F8309FAD492846A9
:1012F00044F02EFF04F53C504146343079F050FE66
:1013000004F5425041460C3079F0AEFA04F54750EE
:10131000414604F5405724307AF00CFA2C22494615
:1013200007F56270A6F0FEF804F54D509E4918309E
:1013300044F00EFF04F54F599C4BC7F8C03309F138
:1013400014007EF039FE04F5515309F1380B1C33BB
:1013500058460F9355F058F90F9B0BF1140B5B4552
:10136000F6D10723C7F880350023A7F884354FF45A
:10137000CB7012F0D9FFC7F87C0504F55650083041
:101380007EF01AFE04F557500C307EF015FE884BA7
:101390001A680AB9C3F80090864BC7F8C03304F541
:1013A00057504FF48051C7F8E8552C3010F00AF927
:1013B00004F559502C3042F0C9FB04F55A502C303A
:1013C00045F020FE04F55B5069F0C8FA04F5994039
:1013D00004F580455C3004F0A9FA774BC5F8DC3C95
:1013E00004F59940643004F0A1FA744BC5F8E43C6C
:1013F00004F599406C3004F099FA714BC5F8EC3C57
:1014000004F59940743004F091FA6E4BC5F8F43C41
:1014100005F60853002204F59A40DA609A605A6093
:1014200083ED008A1C3004F081FA674BC5F81C3D3F
:1014300004F59A40243004F079FA644BC5F8243D51
:1014400004F59A402C3004F071FA614BC5F82C3D3C
:1014500004F59A40403004F069FA5E4BC5F8403D0F
:1014600004F59A40483004F061FA5B4BC5F8483DFA
:1014700004F59A40603004F059FA584BC5F8603DC5
:1014800004F59A40683004F051FA554BC5F8683DB0
:1014900004F59A40703004F59A4904F047FA09F1CE
:1014A0007C09504BC5F8703D484604F03FFA4E4B5E
:1014B000C5F87C3D04F59B40043004F037FA4B4BF3
:1014C000C5F8843D04F59B400C3005F0D1FFFE23A8
:1014D00085F8C03D052385F8DC3D4FF0FF3B444BCC
:1014E000C5F8B49DC5F8B89DC5F8E4BD119305F6DF
:1014F000FC55404B85ED008A224604F5A0454FF48B
:101500000071009304F59C40394B10940FF036FAAB
:101510000023C5F8FC33C5F80034C5F80434C5F819
:101520000834C5F80C34C5F810340323C5F8383432
:1015300005F25443C5F8A4B3C5EDF08A83ED008AE3
:101540002D4BC5F87C342D4BC5F8843404F5A940E7
:101550002B4BC5F88C34C5F87844C5F88044C5F8E1
:101560008844203012F0D8FA04F5A9403C3012F03B
:10157000D3FA04F5A94004F5A849583012F0CCFA82
:1015800040E000BF10F80B08000080BF0000B4422C
:101590000000B4C258110C0868110C083CB90D08C1
:1015A000B0B60D0858B60D08F4B00D0880D40C087C
:1015B000389200206CC50B08141B0C08F81E0C0890
:1015C000E0200C0868190C081C1C0C08A01C0C0856
:1015D000881B0C08981A0C08181A0C08801E0C0896
:1015E000901D0C081C1D0C0890110C080C1E0C08FA
:1015F000DD0F010840C20B08E10F0108E50F0108EB
:10160000E90F010809F15C09754BC5F8EC34A5F840
:10161000F0B409F1980012F07FFA724B7249C5F8E4
:1016200050B54846C3F8009044F092FD4FF6FF7362
:10163000A5F8983404F5AA406C4B6D49A5F8B4B4EC
:101640005430186044F084FD04F5AA4074304AF028
:1016500011FD684BD7F8E8251294CDE91334664B99
:10166000CDE91534654BCDE91734654BCDE9193417
:10167000644BCDE91B34644B1D931EA911E9030093
:101680000CAB83E80300DDE91A010AAB83E8030031
:10169000DDE9180108AB83E80300DDE9160106ABBC
:1016A00083E80300DDE9140104AB83E80300DDE90E
:1016B000120102AB83E80300CDE900284946324617
:1016C00053460E9804F5BD487DF0F4FA08F11C0865
:1016D0004E4BC5F89C3E08F13C0012F01DFA4C49F7
:1016E000404644F035FD4B4B1F6817B14A487FF028
:1016F00067FDC3F8008006F51B76484BC5F89C3E95
:1017000004F5BE40C5F8246F85F8A07E85F8A57E57
:1017100085F8C97E283012F0FFF904F5BE40383054
:1017200012F0FAF904F5BE40483012F0F5F91C2227
:10173000394605F65870A5F0F5FE04F5C04804F5E5
:10174000BF4008F1440840305CF0CCFC04F5C046D2
:10175000404677F075FD324B32497364404644F0A1
:10176000F7FC314A3149116033467C334FF0140C99
:10177000B8B20CFB00120137127C002AF8D12C4AB7
:1017800010802C4A17680FB12B48B0E704F5C14010
:10179000136077F03FFD294BC6F88030284BC6F820
:1017A0009030642386F89430264BC6F8C83004F590
:1017B000C140254BC6F8CC302449103044F0C8FC59
:1017C000234BC6F8903020460123C6F8F07086F807
:1017D000F87085F8E4331FB0BDEC028BBDE8F08FE4
:1017E0000000FFFFD48D002054880C08F4970020DF
:1017F000DCEA0C08ED0F0108F10F0108F50F0108F4
:10180000F90F0108FD0F01080110010840110C0833
:10181000D4B40D0808A0002000110C08E8140C082E
:10182000E8BB0B08C0BB0B08A88E00205C060C08A8
:10183000A48E0020608E00201C110C0828BC0B0810
:1018400078110C08F0240C0848250C0800DC0C0862
:10185000C8260C0810B57EF0E9FF064C064B186050
:101860002046FFF7BBFC2046044A0549BDE810406E
:10187000A3F0EAB8582C0020542C0020B0F400202B
:10188000051001080069C0F3401070470F299DBF83
:10189000302303FB0100503000207047014B93F9C7
:1018A000CD037047584C0020014BD3F8080C70470B
:1018B000584C002008B503689B68984730B9044B22
:1018C00093F8CE0DB0FA80F0400908BD0020FCE787
:1018D000586C002008B5044806F0DAFD10B9034B37
:1018E00093F8C80D08BD00BF582C0020586C00208C
:1018F000022A10B50C4605D1BDE810400948352232
:1019000008F06CBC084BD3F8B40D03685B689847CB
:10191000A04205D159F034F8BDE8104058F0BABFE4
:1019200010BD00BF582C0020586C0020012910B5B4
:101930000C4614D0022907D0D1B90E4BC3F8F010D1
:1019400057F02CFB0C4A05E00A4BC3F8F01057F097
:1019500025FB0A4ABDE81040062150F053BC57F061
:101960001DFB074A062150F04DFC024BC3F8F04026
:1019700010BD00BF588C0020A7120C087C120C0868
:1019800090120C08012902D0022900D011B9024B93
:10199000C3F8F410704700BF588C0020622910B4BF
:1019A00000F3888047291ADC402900F0958008DC84
:1019B000162951DC032904DD4F4B01248C402340C0
:1019C00053B95DF8044B59F0ADBEA1F19604012363
:1019D000A3404A4C2342F4D05DF8044B7047A1F178
:1019E00048031A2BEDD801A454F823F0D9190108A3
:1019F000C3190108C3190108C3190108C319010853
:101A0000D9190108C3190108C3190108C31901082C
:101A1000C3190108C3190108C3190108C319010832
:101A2000C3190108CF1A0108CF1A0108CF1A0108FB
:101A3000D9190108C3190108CF1A0108D9190108D9
:101A4000C3190108C3190108D9190108D9190108D6
:101A5000C3190108D9190108A1F12703112BB0D826
:101A6000112BAED801A454F823F000BFD9190108F6
:101A7000C3190108C3190108C3190108D9190108BC
:101A8000C3190108C3190108C3190108C3190108C2
:101A9000C3190108C3190108C3190108D91901089C
:101AA000D9190108C3190108C3190108D919010876
:101AB000D9190108B02904DC952986DC6B2980D16D
:101AC0008AE7A1F1D003022B3FF67BAF84E75DF8F4
:101AD000044B002359F0F8BD094B012283F8EC2098
:101AE000A3F58043D3F8040C00283FF475AF5DF8EC
:101AF000044B642158F08ABF10004100A10080040B
:101B0000588C002038B50B46622B0446114600F372
:101B10009580472B13DC382B7ADC262B4CDC102BE2
:101B200000F0B680162B00F00781042B00F0C78070
:101B30000A4620461946BDE8384059F031BBA3F1AA
:101B400048021A2AF4D801A050F822F0991C010882
:101B5000311B0108311B0108311B0108311B010831
:101B6000C31C0108311B0108311B0108311B01088E
:101B7000311B0108311B0108311B0108311B010811
:101B8000311B0108CF1C01080F1D0108311B010882
:101B9000311D0108311B0108171D0108C91C01086E
:101BA000311B0108311B01087F1C0108451D01087C
:101BB000311B0108A71C0108A3F12702112AB7D87D
:101BC00001A050F822F000BF7F1C0108311B010862
:101BD000311B0108311B0108831C0108311B01085E
:101BE000311B0108311B0108311B0108311B0108A1
:101BF000311B0108311B0108B91C0108A11C010897
:101C0000311B0108311B0108B31C0108AD1C010880
:101C1000402B8DD1931E5942644C594184F8EB10EE
:101C200057F0BCF9624A94F8EB10624B002908BFE8
:101C30001346614A062150F0E5FA20E09B2B00F0A4
:101C40008E8007DC6B2B00F09480962B7FF470AFB6
:101C500007211EE0AD2B7AD00CDC9D2B7FF468AF02
:101C60000124002A00F08180022A5BD14F4B83F8C7
:101C7000EA4057E0A3F1D002022A3FF659AF01240F
:101C800050E08A1E4D4B5142514183F8C11DF6E789
:101C90000A21FFF72DFEF2E70A4601212046F8E768
:101CA0000A460421FAE70A460321F7E70A460C210F
:101CB000F4E70A460F21F1E70A460021EEE70B217F
:101CC000E7E70A460D21E9E70A460521E6E7374C32
:101CD000D1B102290DD1012384F8E830A4F50053D5
:101CE000D3F8B40D03685B6A984710B1344800F02C
:101CF000A5FD57F053F9334A94F8E810324B002908
:101D000008BF1346314A95E784F8E810E6E7204615
:101D1000FFF70CFEB3E7012431B1022902D12C4BAD
:101D200083F88441204638BD294B83F88411F9E7B4
:101D30002046FFF727FEA2E7022AA0D1204806F09E
:101D40004FF99CE758F01CFE58F0A4FD97E7022AD3
:101D500095D19FED200A1A48FCF7F8F98FE7022A7F
:101D60008DD1174806F0A4FA89E7104B83F8EA20D2
:101D7000D8E7022A14D1114DD5F8B40D0368DB6BF6
:101D80009847044628B10121A5F5804002F0B6FC31
:101D9000C8E757F003F9104A042150F033FA6EE710
:101DA0000748002102F0AAFC69E700BF588C002018
:101DB000BC120C08A3FA0B08C4120C08586C0020C3
:101DC000582C0020FFE50B08601F0C08D4120C08EB
:101DD000584C002000000000E7120C0810B5084C19
:101DE000D4F8B40D03689B6B984738B9D4F8B40D98
:101DF00004F68454001B18BF012010BD0220FCE72C
:101E0000586C002008B5022103205AF0DBFC0221A7
:101E100008465AF0D7FC012104205AF0D3FC0221D5
:101E200015205AF0CFFC132002215AF0CBFC1248A7
:101E300006F09EFDA8B1002146205AF0C3FC002107
:101E400049205AF0BFFC00214A205AF0BBFC002177
:101E500001205AF0B7FC0021BDE8084008465AF0BE
:101E6000B1BC012146205AF0ADFC012149205AF0B5
:101E7000A9FC0121E8E700BF582C002002490348D3
:101E8000052208F0D1B800BFA0790020582C00200E
:101E900038B5304B01241C7090F90A302B2B0CD133
:101EA0002D487DF0FDF82D4807F09CFEBDE8384038
:101EB0002B4801220921FBF76BBD284D9FED290A14
:101EC000D5ED460A642103205AF046FAD5ED460ABC
:101ED0009FED240A642102205AF03EFA9FED220A67
:101EE00003205AF043F99FED200A02205AF03EF9F0
:101EF0009FED1E0A04205AF039F99FED1C0A1520A7
:101F00005AF034F913209FED190A5AF02FF9284698
:101F100006F02EFDA0B1002146205AF081FC0021E0
:101F200049205AF07DFC00214A205AF079FC00211A
:101F300001205AF075FC002108465AF071FCB2E706
:101F4000214646205AF06CFC214649205AF068FC94
:101F50002146E9E798920020688A0020582C00204A
:101F60009C8C0020000000000000C84200A08C45AE
:101F700000F58040D0F8B40D03681B6C18470000D2
:101F800000F5005393EDFB7A00F5A040B5EEC07A62
:101F9000F1EE10FA5DBFD0F8243FDFED086AD3ED13
:101FA000017AD0F83C0F5FBFF8EEE77AE7EE267AC9
:101FB000FDEEE77A17EE900A704700BF0000C842B6
:101FC00000F5005090F82C0428B141F001010842BE
:101FD00014BF01200020704713B50346FFF7F0FF40
:101FE00058B103F5005191F8241CC90705D503F534
:101FF000315393ED000A02B010BD03F5A04422B99D
:1020000004F6747494ED000AF5E794F80C2E022A95
:10201000F6D103F5AA40012201A974304AF0B0F9C3
:102020000028EDD09DED010AE5E7000000F5A04392
:1020300093F8602FFFF7D0BF10B54B68516800F5DB
:10204000A0448B42D8BF0A46D4F8580FCCBF1A46DA
:10205000194623F0CFF9C4F8580F10BD10B5044647
:10206000564866F089FB10F0080217BF544BDFEDAD
:10207000557A93ED7F7AD3ED817A1FBF77EE877A19
:102080009FED517A012267EE877A10F0010317BFA6
:102090004B4B9FED4C7AD3ED816A93ED7E7A1CBF5A
:1020A00037EE667ADFED486A04F5005118BF27EE77
:1020B000267AD1EDFD6AF5EEC06A18BF0123F1EE74
:1020C00010FA3CDD3E4A9FED406AD2EDFD6A66EEB5
:1020D000866A0122F4EE676AF1EE10FA58BFF0EE5C
:1020E000667A04F5A04090F8601F69B393B1D0F808
:1020F000643F06EE903AF8EEE66AF4EEC76AF1EE57
:1021000010FA58BFF0EE476AFDEEE66A16EE903A16
:10211000C0F8643FBAB1D0F8643F07EE103AB8EEA9
:10212000C77AB4EEE77AF1EE10FAD8BFB0EE677A6C
:10213000BDEEC77A17EE103AC0F8643F03E0002AFC
:10214000CFD1002BCDD110BDD3B1D0F8243FD3EDEA
:10215000016AD0F8583FF8EEE66A76EE876A07EE35
:10216000103AB8EEC77AF4EEC76AF1EE10FAD8BFAB
:10217000B0EE667ABDEEC77A17EE103AC0F8583F57
:10218000002AE0D0D0F8243F93ED017AD0F8583FF0
:10219000B8EEC77A77EE277A07EE103AB8EEC77A2C
:1021A000F4EEC77AF1EE10FA58BFB0EE677ABDEEE2
:1021B000C77A17EE103AC0F8583FC4E7484E0020DF
:1021C000584C0020000000000000C84200F5A0406C
:1021D0000023C0F85C3F704773B5164605460023E0
:1021E0006A463046009311F085FD48B1DDED007A76
:1021F0009FED287A67EE877AFDEEE77A17EE900A70
:1022000005F5A044C4F85C0F33785B071CD594F83F
:10221000603FCBB105F5AA40012201A974304AF014
:10222000AFF888B1D4F8643FDDED016A9FED197A0B
:1022300007EE903AF8EEE77AE6EEC77AFDEEE77A37
:1022400017EE903AC4F85C3FD4F83834042B1FD012
:1022500005F50055B5F92624002A16DDD4F85C3FB3
:102260009FED0D7A83EAE371A1EBE37107EE901A1B
:10227000F8EEE77A67EE877A07EE102AB8EEC77AAB
:10228000F4EEC77AF1EE10FA02D50023C4F85C3FF1
:1022900002B070BD0000C8420AD7233C37B50B78A6
:1022A0005A0704460D461DD500F5AA40012201A992
:1022B00074304AF065F8A8B1D5ED017A2B78DFEDDE
:1022C0001C6AF8EEE77ADB0767EEA67A1BD59DED70
:1022D000017AB4EEE77AF1EE10FACCBF01200020CB
:1022E00003B030BD2B78D5ED017A13F0010FF8EE75
:1022F000E77A04F5A04411D104F63C7393ED007A1B
:10230000B8EEC77AE5E704F5A044D4F8243F93ED8E
:10231000017AB8EEC77AE7EE667AD8E7D4F8243FB8
:1023200093ED017AB8EEC77A77EE877AE4E700BFDB
:102330000AD7233C00F5005300F58042B3F9D633A9
:10234000D2F8B42D00EE103A00F59A4348339A4281
:10235000B8EEC00A0ED100F5A040D0F83834042BF6
:1023600002D090F8E5332BB100F56160D0ED007A32
:1023700030EE270A70470000014608B501F5A0417C
:10238000FFF7D8FF01F63C73D3ED007A9FED057A95
:10239000F8EEE77AE0EE477AFDEEE77A17EE900A7C
:1023A00008BD00BF0000C84237B500F5A04504468F
:1023B00095F8603FFBB100F5AA40012201A97430F5
:1023C00049F0DEFFB8B105F66472D2ED007A9FEDF8
:1023D0000D7A05F66873D3ED006AF8EEE77AE6EE5B
:1023E000877ADDED016AE6EEC77AFDEEE77A17EE51
:1023F000900A03B030BD2046FFF7BEFFD5F8583F26
:10240000181AF6E70000C842014608B5FFF792FF28
:1024100001F5BE40D0ED1D7A37EEC00ADFED047A3B
:1024200020EE270AFDEEC07A17EE900A08BD00BF25
:102430000000C8422DE9F04100F5BE4800F5BE4558
:1024400008F13808483504462946404611F0C6FED2
:1024500004F5BE4604F5A04728362A4631464046D4
:1024600087EDF30A11F0F0FDDFED220A87EDF40AA3
:10247000B7EE001A762022F01DFF04F5325383EDEB
:102480007D0A2046FBF70AFE04F58043D3F8B40D1D
:1024900003685B6898470B280BD006D80A280FD032
:1024A0000023C7F85C3FBDE8F0810E38C0B20128B8
:1024B000F6D829462046FFF7F1FE0028F0D011E0BB
:1024C00029462046FFF7EAFE30B90B484FF4804119
:1024D000FCF750F80028E3D12046FFF795FFB0F550
:1024E000FA6FE6DD2A4631462046BDE8F041FFF7A7
:1024F00073BE00BF00000000582C002010B52DED69
:10250000028B00F5A043DFED1F8AD3F84C2F93F820
:10251000483F07EE902ADA0758BF00F5AC52B8EEF4
:10252000E78A58BFD2ED007A28EE288A58BFF8EE25
:10253000E77A82B058BFA7EEE88A5B0704460FD55A
:1025400000F5AA40012201A9743049F019FF38B101
:102550009DED010A30EE480A02B0BDEC028B10BDC1
:102560002046FFF709FF04F5AC5393ED000A07EE90
:10257000900AB8EEC00AF8EEE77A28EEC00AA7EE95
:10258000A80AE7E70AD7233C38B52DED028B00F502
:10259000804200F59A43D2F8B42D24339A4204467F
:1025A0004DD100F58053D3F8105500F50053B3F921
:1025B0002434002B66DD04F5B85292ED057AF7EE6F
:1025C000007AB4EEE77AF1EE10FA5BD404F53352F8
:1025D000D2ED067AF6EE006A67EEA67A87EE871AE3
:1025E000B5EEC01AF1EE10FA4CD907EE905A9FEDF5
:1025F000288AB8EEE70A07EE903A04F5AA4004F5F7
:10260000A044F8EEE70A20EE080A743049F0C4FF4F
:10261000D4F85C3F9FED1F1ADFED1F0A002BBCBFF3
:1026200007EE903AF8EEE77A4FF42970B8BFA7EEBC
:10263000880ABDEC028BBDE8384022F03BBE05F0B5
:102640006DFBF8B904F54053D3F8E80503681B693E
:10265000984704F50053DFED100AB3F9243401EE76
:10266000103A04F5A04393EDF30AB8EEC11A0546FB
:1026700040F27F2022F01EFEBDEEC00A10EE103A9E
:102680001BB296E7BDEC028B9FED030A38BD00BF7D
:102690000AD7233C00007A440000000010B504462D
:1026A0007EF0C0FD04F50053D3F8382C801A41F2B7
:1026B000883290420FD802212046FFF781FC50B1AA
:1026C00004F5A044D4F83824042A04D103F62C439A
:1026D00093ED000A10BD9FED010AFBE7000000002A
:1026E00030B52DED028B00F5A045DFED298A95F878
:1026F000603F83B004467BB3D5F8643F9FED250A65
:1027000007EE903AF8EEE77A00F5AA4027EE800A45
:10271000012201A9743049F06BFEE8B12046FFF7B1
:1027200033FFDDED017A05F6687585ED000A37EEB9
:10273000800A20468DED010AFFF7B0FFDDED017A3A
:1027400030EE270A20EE280ABDEEC00A10EE100A6D
:1027500003B0BDEC028B30BDD5F8242FD5F8583F1F
:1027600052689B1A08EE103A2046FFF7E3FDB8EED8
:10277000C88A2046A0EE288AFFF790FFBDEEC88ADF
:10278000B8EEC88AA0EE288ABDEEC80ADEE700BF10
:102790000000C8420AD7233C10B500F58043044628
:1027A000D3F8B40D03685B6A984718B104F5C044C8
:1027B00094F8E80010BD000038B500F5A0440D46BF
:1027C000D4F8583F0B44C4F8583F94F8603F3BB1ED
:1027D000FFF7E2FF20B9D4F8641F2944C4F8641F4E
:1027E00038BD000030B500F50050D0F82024D307E4
:1027F0000FD4094B08201D785C688D4204D1224219
:1028000014BF0120002030BD013803F10803F2D1CC
:10281000F9E70120F7E700BF38150C0810B500F5FF
:1028200080430446D3F8B40D03685B6898470146BB
:102830002046BDE81040FFF7D5BF000037B500F5D2
:10284000A0440546D4F83C3FC4F8583F0023C4F8E0
:102850005C3FFFF7E3FFE0B105F5AA40012201A9C3
:10286000743049F08DFDA0B12846FFF795FF80B97F
:10287000DDED017A9FED097A67EE877A0123FDEE9F
:10288000E77A84F8603F17EE903AC4F8643F03B0EB
:1028900030BD002384F8603FF9E700BF0000C84264
:1028A00038B504460D46FFF7B9FF30B1032128467D
:1028B00011F0FCF980F00103D8B204F5A04484F8CB
:1028C000610F38BD73B500F5A0444A68C4F8582FAD
:1028D0000B780D46D90741BFD4F8243F5B689B189D
:1028E000C4F8583F94F8613F064623B100F5BE4155
:1028F0004831FFF7D5FF2B785B070FD506F5AA40C7
:10290000012201A9743049F03BFD38B1012384F85C
:10291000603F6B68C4F8643F02B070BD002384F868
:10292000603FF9E7F0B52DED028B044683B004F566
:10293000A0450E468DED010AFFF7C4FFDFED370A13
:102940009DED010A40F24310B7EE001A22F0B2FCEE
:10295000D5F85C3F5B4207EE903AF8EEE77A04F573
:10296000105767EE807A2046FDEEE77AB0EE408A97
:1029700017EE901AFFF720FFD7ED0A7AF5EEC07A2E
:10298000F1EE10FA07F1280743DDD5F85C3F002B84
:102990003FDD2046FFF708FD07EE900ADFED206AD5
:1029A000B8EEE77AD7ED007A67EEA67AB4EEE77A6A
:1029B000F1EE10FA2DD531462046FFF783FF04F5DE
:1029C000BE41324638312046FFF706FCD5F85C3F61
:1029D0005B4207EE903AF8EEE77A204667EE887A97
:1029E000FDEEE77A17EE901AFFF7E6FEB5EEC08A25
:1029F000F1EE10FA0DDDD5F85C3F07EE903AB8EE37
:102A0000E77AC7EE087AFDEEE77A17EE903AC5F856
:102A10005C3F03B0BDEC028BF0BD00BF00000000C6
:102A20000000C8C2F0B500F5A04487B094F8483F54
:102A300003F00503052B07460BD04AF023FD4FF4A6
:102A4000AE724FF480114AF0D5FC0025284607B03D
:102A5000F0BD1E486A46032111F038F90028F4D071
:102A60001B4801AA032111F031F905460028ECD0DA
:102A7000184BDFED190A93EDF40A40F26D10B7EE32
:102A8000001A22F017FC04F648730FCBB0EE401A80
:102A900002AEDFED111ADDED010A9DED000AB7EE81
:102AA000002A86E80F0022F037FBDFED0C7A20EEDB
:102AB000270A3046FDEEC07A032217EE901A11F075
:102AC00031F831463846FFF7FDFEBFE7808B002026
:102AD000A08B0020587C0020000000000000C842AD
:102AE000F7B50D4602210446FFF76AFA60B304F514
:102AF000A047D7F83834042B26D12046FFF78EFEA6
:102B000010B304F5AA46743604F5BE4101236A46A3
:102B10003831304649F01EFBB0B104F5BE41012307
:102B200001AA4831304649F015FB68B19DED017AA4
:102B3000DDED007A77EEC77A95ED007A37EE277AE9
:102B400085ED007AC7EDFC7A03B0F0BDF0B52DED50
:102B5000048B00F5005489B000F5546794F8F21B1B
:102B600003910546384644F00BFD03990646384666
:102B700044F018FD042E0399B0EE408A20D10023C2
:102B800005A88DED050A0693079324F001FF05F5CE
:102B9000B15005A9103022F01DFEDFED957A8DEDC4
:102BA000050AB4EEE71AF1EE10FACDED060A8DED46
:102BB000071A05DB05F5805393F88C35DE070CD436
:102BC00094F8243C002262F3000384F83C2C84F83F
:102BD000243C09B0BDEC048BF0BD94F8243C98076C
:102BE0005CBF43F0020384F8243C05F531565CBF1A
:102BF00004F6284383ED008A314686ED001A284604
:102C0000FFF76EFF94F83C3C092B00F2878004F636
:102C10004443D3ED000A9FED779AB0EE480A22F0C4
:102C200037FA00BB04F6284394F8F21BD3ED008A70
:102C3000384644F0D5FC07EE900A9FED6F7AF8EE27
:102C4000E77A78EEC88A67EE877AF0EEE88A67EE70
:102C5000897AF4EEE78AF1EE10FAC2BF94F83C3CB0
:102C6000013384F83C3C04F6444394F8F21BD3ED62
:102C7000008A384644F0B4FC07EE900AF8EEE77A92
:102C80009FED5E7A67EE897A78EEC88A67EE877A7A
:102C9000F0EEE88AF4EEE78AF1EE10FA02DD0023A6
:102CA00084F83C3C04F6444383ED008A94F8243CC9
:102CB000DA078ED5284605F5A047FFF71FFC96EDED
:102CC000008A97F8603F30EE488A002B4BD005F51C
:102CD000AA40012205A9743049F052FB002848D1CE
:102CE0007EF0A0FAD4F8382C41F28831821A8A4258
:102CF000034604F62C4204F5436141D982ED008A73
:102D0000284681ED008A0221FFF75AF918B107F52C
:102D10006167FA68BA60C4F8383C5AE794F8243C12
:102D200043F00103590784F8243CBBD405F5A042C5
:102D3000D2F83824042AB5D102212846FFF740F9F9
:102D40000028AFD043F0040384F8243C3068F9F73E
:102D5000DBFB05F54F57CDE90001294A062138462E
:102D60004FF050FA9EE72846FFF758FD0028AED1F5
:102D7000B6E796ED000A9DED058A38EE408AAFE78A
:102D80009FED1E0A92ED007ADFED1E7A28EE008A92
:102D9000A7EE278A82ED008AC4F8380CD1ED007ABC
:102DA00038EE678AF3EE0E7AB0EEC88AB4EEE78AA0
:102DB000F1EE10FA7FF70DAF94F8243C5B070BD5CA
:102DC0003068F9F7A1FB05F54F54CDE900010E4A33
:102DD000062120464FF016FA242205F53050002136
:102DE000104409B0BDEC048BBDE8F040A4F09ABBE0
:102DF000000000340AD7233CCDCC4C3DCDCC4C3E1A
:102E0000F8140C08CDCC4C3F15150C0838B52DED39
:102E1000028B0D460446FFF771FB002320462B7002
:102E2000B0EE408AFFF73AFC0221204638EE400A15
:102E3000FFF7C6F828B104F5005494F8240C00F00C
:102E40000100BDEC028B287038BD000070B50B7816
:102E500003F00503042B05460C46164615D105F56F
:102E6000A0454AF00FFBB2B24FF480114AF0C2FA0B
:102E7000D5F8242F636852689B1A13F5FA7FC8BFF0
:102E80006360237843F00103237070BDF8B500F54B
:102E9000805300F5A047D3F88065D7F8F453B542C6
:102EA000044619D00E4A1268D26A92F89C209AB150
:102EB00000F5BE41751B25224831FFF7C7FF07EE1D
:102EC000905AB8EEE70ADFED077A04F5325020EEAB
:102ED000270A30307BF076FCC7F8F463F8BD00BFFA
:102EE000542C00200AD7233CF8B500F5A044054631
:102EF00094F8E7C30F4604F62876BCF1000F53D0D0
:102F000004F648730FCB86E80F00012384F8E833FA
:102F100097E80F0004F6487686E80F00D4F8503F93
:102F200005F5BE46483693B9D4F8543F7BB9D4F87A
:102F3000403FD4F84C2FC4F8503FD4F8443FC4F875
:102F4000543F22B9D4F83C1F304610F0EBFD314617
:102F500028222846FFF77AFF94F8481F11F0040151
:102F600002D1304610F0A2FE05F5BE4105F5BE4087
:102F700032462831383011F09DF838B104F6287601
:102F800004F6387494E80F0086E80F00284604F031
:102F90005DFB2846FFF74EFA284604F087FE2846D8
:102FA000BDE8F840FEF7E4BF04F638730FCB86E8BF
:102FB0000F00012384F8E73384F8E8C3A8E7000092
:102FC000F8B500F500530446B3F97E33002B0E46E6
:102FD00033DB0B7813F0020F14BF4FF0FF330123E4
:102FE00004F5A04505F6287785F8003F05F6387307
:102FF0000FCB87E80F0096E80F0005F6487787E8C3
:103000000F0004F5BE41572248312046FFF71EFF4E
:103010002046FFF713FC2046FFF70CFA204604F089
:1030200045FE002385F8E833C5F8043F85F8ED3305
:103030002046BDE8F84004F009BB4FF0FF33CFE76E
:103040002DE9F043364B1B6885B00546D86AFAF780
:1030500079FA002861D105F5005393F9A03B5A1C79
:1030600054D0002B05F58C6711DD95F871242421CF
:1030700007EE903A01FB027292ED0B7AF8EEE77AD6
:10308000B0EEC77AB4EEE77AF1EE10FA3EDC05F561
:10309000805305F5985693F88C3513F0010406F12A
:1030A000100629D0C3F340089B0732D495F81414B6
:1030B00095F858444FF0B00909FB015191F8F131EE
:1030C0004CBB022B18D9684610F026FD69463046E5
:1030D0000AF080FA044678B195F8143409FB0353DA
:1030E0004246D3F80012684610F01CFD0AF012FDAB
:1030F00069460AF05DF9044638460CF089FF30460F
:103100000AF074F82846FBF707FA204605B0BDE838
:10311000F0830024F0E74446EEE70020F6E700BF26
:10312000542C002038B50C4B1B680546D86A0C4659
:10313000FAF708FA10B10024204638BD0AF0EAFC7C
:1031400021460AF035F904460028F4D005F5A840D8
:103150005C3025F00BFAEFE7542C0020F0B500F5B9
:10316000A045002385F8E73385F8E83305F6387382
:10317000044600EE101A0FCB87B005F6287686E8D5
:103180000F0002AE04F5BE42B8EEC00A3046174941
:10319000383244F03FF896E80F0005F6487787E8A4
:1031A0000F0004F5BE4140F257124831204601910C
:1031B000FFF74CFE01992046FFF772FB019920466C
:1031C000FFF780FB04F500532046B3F97E33002B54
:1031D000B4BF4FF0FF33012385F8003FFFF72AF912
:1031E000204607B0BDE8F04004F060BD0463002055
:1031F00010B50349044644F00DF8204610BD00BF49
:1032000004630020F8B500F5A04404F638730546C1
:103210000E460FCB04F6287787E80F0006F1080169
:103220002846FFF761FEB388D4F84C2F03EB8303E5
:1032300003EB83039B001BB2002BD8BF4FF4C87372
:10324000A4F8E233D4F8243F5968521AC4F8B423DE
:103250009A680A32C4F8502FDB680A33C4F8543F26
:103260000023C4F8C83384F8E43384F8F833C4F88E
:10327000B8330023C4F8AC334FF0FF33C4F8A433A1
:1032800095F8712405F58C63242101FB0233DB6A78
:10329000C4F8DC33F8BD000070B50E4608310546B1
:1032A000FFF722FEB38805F5A0444BB3642213FB5D
:1032B00002F3C4F8B433B4F9E233002BD8BF4FF4AF
:1032C0007A734FF0240205F53050D8BFA4F8E233EA
:1032D00000211044A4F026F904F6747305F5BC40EF
:1032E00093ED000A314610307BF0DAFDD4F8383423
:1032F000072B0CD128460421BDE87040FAF780BEA8
:10330000D4F8B433002BD6DC40F6B833D1E770BD27
:103310000B7A00F5A04013F0020F14BF4FF0FF33FB
:10332000012380F8003F70477FB501F1080305468F
:103330000E460FCB6C4684E80F0005F5BE413831D0
:10334000204610F053FD21462846FFF7CDFD3146BB
:103350002846FFF7DDFF04B070BD00007FB501F126
:10336000080304460E460FCB6D4685E80F0004F5B2
:10337000BE413831284610F039FD29462046FFF776
:10338000B3FD20463146FFF7C3FF337907EE903A8D
:10339000337E9B0748BF9FED0C7AF8EE677A04F501
:1033A000A04448BF67EE877A9FED087A67EE877A78
:1033B000FCEEE77A17EE903AC4F8F83E0123C4F821
:1033C000183F04B070BD00BF0000803B00A00C4758
:1033D0007FB501F1080304460E460FCB6D4685E824
:1033E0000F0004F5BE413831284610F0FFFC294695
:1033F0002046FFF779FD20463146FFF789FFB38865
:1034000004F5A0444FF47A725343C4F8103F0123EB
:10341000C4F8183F04B070BD2DE9F34100F5BE4576
:103420000446483500F5BE400E462830294610F0C7
:103430009DFC04F5A047C0B94FF0FF33C7F8A43393
:1034400006F10808404610F097FB032802463AD1DF
:10345000F168284610F066FBB388C7F8183F20468D
:1034600002B0BDE8F041FEF7B1BE1AF0C7F8FAF7B6
:1034700059FB012812D94FF0FF33C7F8A4331AF0D3
:10348000BDF890F8F432DFED150AB02202FB03001C
:1034900090ED3C0A284610F017FFD1E704F580585C
:1034A000D8F8100521F0DAFE08F5A263C7F8A403E6
:1034B000D3ED007A9FED0A0ADFED080AF8EEE77A0D
:1034C00027EE800AE6E701AA0021404610F060FBE3
:1034D0000028C1D001990022BBE700BF00007A4458
:1034E0000AD7233C7FB501F1080304460E460FCBF3
:1034F0006D4685E80F0004F5BE413831284610F0CE
:1035000075FC29462046FFF7EFFC20463146FFF7C1
:10351000FFFE04F5A0440023C4F8183F04B070BDBA
:1035200037B504460D467DF07DFEE060D5ED027AAC
:10353000F5EEC07AF1EE10FA15DD9FED127A67EE26
:10354000877AFCEEE77AC4ED027A55F027FDA2688F
:103550004FF47A73B2FBF3F30B4A062103B0BDE8D4
:1035600030404EF04FBE64F055FF0023009395F9B4
:103570000D2095F90E3095F90C1064F0E7FEA0606F
:10358000E3E700BF00007A4478150C082DE9F0410C
:103590002DED028B84B004460AF0BCFA09F00CFC55
:1035A00004F5805304F5A04593F808380BB90028BA
:1035B00074D0D5F8A433013370D1D5F8C833002BBB
:1035C00048D07DF02FFED5F8C833C01AB0F5FA6F99
:1035D00064D394F81424DFED5D7A9FED5D8A4FF09B
:1035E000B00808FB024292ED840A20EE270A21F07F
:1035F0004DFED5EDEB7A30EE670A21F047FEDFEDA8
:10360000557A20EE080A04F54F5720EE270A21F0DC
:10361000E5FDFDEEC07A17EE906AC5EDE97AD5EDCD
:10362000EB7A67EE887A17EE900AF8F76DFFCDE92E
:10363000020194F8143408FB0343D3F80C02F8F7A2
:1036400063FF454ACDE900013346062138464EF076
:10365000D9FD23E004F59070FAF764FA02281DD929
:1036600094F81434B02202FB034393ED837AF1EE15
:10367000047AB4EEE77AF1EE10FA0FDD374B1B68EF
:10368000D86A0368DB699847012803D07DF0CAFD3A
:10369000C5F8C803D5F8C833002B92D104F54053C0
:1036A000D5F8A413D3F8E8054A1C036845D01B6B72
:1036B00098472B4807F0BCFA20B104F5A8405C30CD
:1036C00027F0F0F92046FEF79FFED5F8B433834289
:1036D000064635DA07EE906A9FED227AF8EEE77A31
:1036E00004F54F5467EE877A05F6287617EE900AB0
:1036F000F8F70AFF1C4ACDE90001204606214EF0EA
:1037000081FD01244FF0FF33C5F8A43385F8E4436D
:1037100005F638730FCB05F6487786E80F0087E883
:103720000F00124864F0F2FF002385F8E7332046CB
:1037300004B0BDEC028BBDE8F0815B6B9847B8E745
:10374000074807F055FA0028C4D1F1E735FA8E3C56
:10375000E02E65420000C84288150C08542C002059
:10376000582C00200AD7233CAC150C08484E0020EA
:103770002DE9F04700F5A0462DED028B4FF0FF3309
:10378000C6F8A43306F648738C4607460FCBBCF840
:1037900004509CF8049088B004AC2D0A84E80F0013
:1037A00020D007F5BE4808F128082146404610F011
:1037B00015FD21464046B0EE408A10F0DFFBDFEDFC
:1037C000557AB4EEE78AF1EE10FA0BDBEBB200EEBD
:1037D000903ADFED517AF8EE600A20EE270A204693
:1037E00010F072FD07F5405A96F8E823DAF8E8057C
:1037F0009FED4A0A036807F5BE489B6A08F138083E
:1038000022B307F5BE4122462831984707F50052FA
:10381000B2F9AE33002B1CDD07EE903A96EDF37A49
:10382000F8EEE77AB4EEE77AF1EE10FA11DD07F57B
:10383000BE4122462831404610F03CFCF0B900253C
:10384000284608B0BDEC028BBDE8F0872246414611
:10385000DBE7B9F1000F1CD1002D3BD1B2F9AC333D
:10386000DAF8E805D6EDF00A00EE103A0368B8EE93
:10387000C00A1B6A9847B0EE408A0EE0002DDED1E8
:1038800006F6287406F6387696E80F0084E80F00EE
:10389000D6E707EE909AB8EE678A2146404610F0C8
:1038A0009DFCB4EEC08AF1EE10FA16DBB6F898343F
:1038B00003932146404610F091FCBCEEC00A039BE6
:1038C000174A8DED000A062107F54F504EF09AFC7D
:1038D0000125B5E79FED118ADFE707F5BE412246D6
:1038E0002831404610F0E6FB05460028A7D0B6F880
:1038F000983403932146404610F070FCBCEEC00A99
:10390000039B084A8DED000A062107F54F504EF043
:1039100079FC95E700000034E02E654200000000CD
:10392000C8150C08E6150C0870B500F5005500F533
:10393000A046B5F9B0130029ACBF01234FF0FF3307
:103940000029B8BF494286F8003F89B2044604F016
:10395000C9FAB5F9AC3396EDF37A002BCABF07EE7E
:10396000903ADFED0D7AF8EEE77AFCEEE77AF8EEC2
:10397000677AB4EEE77AF1EE10FA07D804F54F5003
:10398000064A06214EF03EFC012070BD204604F0A0
:10399000C5F90028F2D1F8E70000000004160C0871
:1039A0002DE9F04100F5BE4700F5BE452837483502
:1039B00004462946384610F0D9F904F5A04604F526
:1039C000405830B3D6F8A4134B1C22D0D8F8E805E1
:1039D00003681B6B9847D6F8183F012B47D0D6F8E1
:1039E000183F022B06D12046FEF7C6FCD6F84C3F06
:1039F000984243DD2046FEF7BFFCD6F84C3FC01A84
:103A00000028B8BF4042B0F5FA7FCCBF00200120AB
:103A100035E004F5BE402946383010F0DFFBDFED1D
:103A2000197AB4EEE70AF1EE10FA16D538462946AF
:103A300010F0A4FA9FED147ADFED140AF6EE007A86
:103A4000E0EE077A28469FED120AFDEEE77AF8EEDF
:103A5000E77A27EE800A10F037FCD8F8E8059FEDEA
:103A60000D0A03682A469B6A39469847B3E7204601
:103A7000FEF782FCD6F84C3F9842B0DB0120BDE84F
:103A8000F08100BF00004843A00CB34500009643FE
:103A90000AD7233C00000000F7B5374FD1ED026A8A
:103AA000D7F83C3F9FED357A07EE903AF8EEE77A8B
:103AB0000546D7EE876A0E46F5EEC06AF1EE10FABB
:103AC00008DD55F06BFA2E4A06214EF09BFB0120D3
:103AD00003B0F0BDD1ED037A97EDF16AF5EEC07A4F
:103AE000F1EE10FA13DDF4EEC67AF1EE10FA0ED50F
:103AF00055F054FA0446D7F8C403F8F705FD214AF7
:103B0000CDE90001062120464EF07CFBDFE7DFED2A
:103B10001E7A337CB4EEE76AF1EE10FA54BFB0EED1
:103B2000677AB0EE467A0BB90020D1E7B5EEC06AED
:103B3000F1EE10FA0CDC86EE876A03EB830307EEE6
:103B4000903AF8EEE77AF4EEC67AF1EE10FAEBD599
:103B50002C7C002CE8D17DF065FB6B69C01A337CAE
:103B60004FF47A7253439842DED901232B747DF0CF
:103B700059FB68612046ABE7587C00200AD7233CFC
:103B80001C160C082D160C080AD723BC38B50546A0
:103B900076F04AFE75F09EFB044640B97DF042FB8C
:103BA000EB68C01AAB68984284BFAC600124204621
:103BB00038BD000038B504460D467DF033FB04F5F2
:103BC000A0439FED077AC3F81C0FD5ED027A67EE8C
:103BD000877AFDEEE77A17EE902AC3F8182F38BDE2
:103BE00000007A4410B504467DF01CFB04F5A043A8
:103BF000D3F81C2F801AD3F8182F90424FF00000F2
:103C000084BFC3F8180F012010BD000000F5A043C9
:103C100093EDF37AD3F8182F22EAE27207EE902A96
:103C2000F8EEE77A0020B4EEE77AF1EE10FA44BF3E
:103C3000C3F8180F0120704710B500F5005300F5C8
:103C4000A040B3F97E33002BB4BF4FF0FF33012304
:103C500080F8003F00F6487400F638700FC884E81A
:103C60000F0010BD38B504462DED028BF0EE408AF2
:103C7000B0EE608A01B301295CD0B5EEC08AF1EEE6
:103C800010FA66DDDFED347AB4EEE78AF1EE10FA71
:103C90005FD8FCEEC87A04F54F5017EE903A2F4AE1
:103CA00006214EF0AFFAFDEEC87A04F5005417EE87
:103CB000903A84F84B333BE0F8EE000A21F0E8F943
:103CC00040B104F580444FF0FF33C4F8E43DBDEC4F
:103CD000028B38BD04F50053B3F9542307EE902A44
:103CE000F8EEE77AF4EEE87AF1EE10FAC5D8B3F917
:103CF000563307EE903AF8EEE77AF4EEE87AF1EE12
:103D000010FABADBDFED147A68EEA77A04F5804387
:103D1000FDEEE77A062117EE902AFCEEE87AC3F86A
:103D2000E42D04F54F5017EE903A0D4A4EF06AFA22
:103D30000120CCE7FCEEC07A0A4A17EE903A062141
:103D400000F54F5004F500544EF05CFAC4EDD88AEB
:103D5000EEE70020BBE700BF0000C84273160C0866
:103D60004C160C0860160C08D1F80D3000EE903A95
:103D7000D1F80930097A00EE103AFFF773BF00005E
:103D800070B58B88012B04460D4611D100F5907655
:103D90003046F9F7C7FE02280AD994F81414B02364
:103DA00003FB01612046DC31BDE87040FFF7BAB982
:103DB00009F0B0FE05F10801BDE8704009F0F8BA5D
:103DC000F0B500F5A0460027A04B86F8ED7389B04A
:103DD000044608460D4683F8617F24F0D9F940B3C4
:103DE000012386F8E43304F54053D3F8E80503686B
:103DF000DB6B984786F8EB73C6F8047F03A80FF0D7
:103E00008BFEB6F898144FF6FF73994208BF3946F7
:103E1000013104F5A84001AA89B25C3026F0C4F94A
:103E200028B1BDF80600A0F115035842584186F8A4
:103E3000E5036B885D2B00F0028132D81F2B29D857
:103E40000F2B01D800202AE0103B0F2BFAD801A23B
:103E500052F823F0473F01085D3F0108673F010822
:103E6000713F0108853F0108533F0108353F0108B4
:103E7000453E0108453E0108453E0108453E010812
:103E8000453E0108453E0108453E0108953F0108B1
:103E90007B3F0108532BD5D1012086F8EB0309B0F5
:103EA000F0BDBD2B18D8BB2B4BD8B22B7CD00CD877
:103EB000702B74D0722BC5D1D5ED027AFDEEE77A66
:103EC00017EE903AC6F8183F3BE0B32BBAD129461B
:103ED0002046FFF755FF34E0C33B9AB2112AB1D810
:103EE000112BAFD801A252F823F000BFE13F010827
:103EF000453E0108E13F0108453E0108453E0108F5
:103F0000453E0108E13F0108453E0108453E0108E4
:103F1000453E01081D400108453E0108453E010897
:103F2000453E0108453E0108B33F0108453E0108F2
:103F3000D13F0108002386F8213429462046FFF7A7
:103F400061F90120ABE705F108012046FEF7CCFF3F
:103F5000F7E729462046FFF79FF9F2E72946204672
:103F6000FFF7E2F9EDE729462046FFF7F7F9E8E722
:103F700029462046FFF72CFAE3E729462046FFF7BB
:103F8000B1FADEE704F59A4129226031204606F0B5
:103F90004BF8D6E729462046FFF73EFAD1E72946F7
:103FA0002046FFF707FECCE729462046FFF7DCFE58
:103FB000C7E7AB88012BC4D803F0010386F8E633CA
:103FC000AB88234A062104F54F504EF01BF9B8E7A1
:103FD000A988003918BF0121204600F08FFBB0E707
:103FE00004F5BF46EB6804F5C044403694F8391038
:103FF00073B92B6963B96B6953B930465AF0A0F8AD
:1040000004289ED194F8391030465AF0A3F898E766
:1040100005F1080230465AF0DBF992E704F5C04397
:1040200004F5BF4095ED041AD5ED020A95ED030A9B
:1040300093F83910002240305AF0AEF881E704F5C9
:104040009A4029464830FFF76BFA7AE7587C0020FF
:1040500084160C0800F5804200F59A43D2F8B42D7E
:1040600048339A4201D1FFF7ABBE012070470000F0
:1040700010B500F5804200F59A43D2F8B42D4833CC
:104080009A4204460DD100F59A410822603105F0AC
:10409000CBFF04F54F50034ABDE8104006214EF017
:1040A000B1B810BD94160C08F0B506468FB009AD36
:1040B00006F5A04428460F460FF02EFDB4F89834BC
:1040C0004FF6FF72934208BF0023013306F5A84064
:1040D00007AA99B25C3026F067F8A0B117B10023A7
:1040E000C4F8FC3E95E80F0001AE86E80F00D4F856
:1040F000543F009304F6487494E80E00034802F01D
:104100004BFD0FB0F0BD0120FBE700BFC0790020E0
:1041100070B5064606F5A045002103F0E3FED5F88C
:10412000044F7CB9304603F0F9FD10B90024204655
:1041300070BDD5F8FC3E012BF8DD7DF073F8C5F8B5
:10414000040FF4E7D5F8181F61B17DF06BF8D5F8CE
:10415000043FC01AD5F8103F9842E7D90023C5F8AC
:10416000183F01213046FFF79FFF04460028DDD0AD
:10417000044A062106F54F504EF044F8002385F816
:10418000ED33D4E7BC160C0870B50A468B88190AC3
:10419000137E0546DB0748BF01EB810105F5A0440E
:1041A00048BF4900002603F09DFE84F8ED632846D1
:1041B00003F0B4FD10B90024204670BDD4F8181FD8
:1041C00051B1D4F8FC3ED4F8F82E9342F3DD012B24
:1041D000F1DDC4F8186F01212846FFF765FF04469A
:1041E0000028E8D0034A062105F54F504EF00AF8A2
:1041F000E2E700BFD4160C0838B5054605F5A04423
:10420000898803F06FFED4F8183F73BBD4F8FC3EE6
:10421000002BB8BF5B42012B02DC0024204638BDD6
:1042200094F8012F94F8023F6AB9002BF5D0D4F826
:104230003C2F6423062192FBF3F305F54F500C4A03
:104240004DF0E0FF01E0002BF1D10121C4F8181F6F
:104250002846FFF729FF04460028DED0054A06213C
:1042600005F54F504DF0CEFFD8E70021F0E700BF35
:10427000EC160C080A170C082DE9F0474B881F2B89
:104280008AB004460A462FD80F2B06D8954A042137
:1042900004F54F504DF0B6FF87E0A3F110010F2950
:1042A000F4D801A050F821F0BB4301087D44010877
:1042B0008944010897440108B1440108C943010831
:1042C000AF4301088D4201088D4201088D4201086B
:1042D0008D4201088D4201088D4201088D4201087E
:1042E000BD440108A3440108702B00F0F5800CD8F0
:1042F000532B00F0E9805D2BC8D100F59A4048307F
:104300000AB0BDE8F047FFF741BCB32B08D8B12B8A
:104310004BD8722BBAD10AB0BDE8F047FFF776BC94
:10432000D42B3BD8BB2BB1D9A3F1BC02182AADD8F2
:1043300001A151F822F000BFAB430108AB430108D3
:104340008D4201088D4201088D4201088D4201080D
:104350008D420108AB4301088D420108AB430108BF
:104360008D4201088D4201088D420108AB430108CE
:104370008D4201088D4201088D420108AB430108BE
:10438000AB430108AB4301088D4201088D4201088F
:10439000AB4301088D420108AB430108DF2B04D079
:1043A00040F6B83293427FF471AF01202FE02046EF
:1043B0000AB0BDE8F047FFF7E9B8114620460AB059
:1043C000BDE8F047FFF7D4B904F5A04504F5BC46B5
:1043D000D5F8383404F5BE4704F5BE4804F5BE49A7
:1043E000072B06F1100607F1280708F1480809F124
:1043F00038090FD104F5A84430340194D5F8B4330A
:10440000009342464B46394630467AF00DFE0AB0DC
:10441000BDE8F08700230DF1270133488DF82730E0
:10442000FEF7F4FCD5EDFC7AD5EDF10A95EDF41A22
:10443000D5F8D4A3CDED060A30EE670A04F5C040E6
:1044400044308DED070A8DED051A74F039FF0546ED
:10445000204600F09DFE9DF827309DED051ADDED0C
:10446000060A9DED070ACDE90203CDE900A54B46FA
:104470004246394630467AF02DFDC8E720469188FD
:1044800003F030FD0020C2E7114620460AB0BDE827
:10449000F047FFF779BE20460AB0BDE8F047FFF7C6
:1044A00037BE114620460AB0BDE8F047FFF7A4BE6C
:1044B00020460AB0BDE8F047FFF736BA20460AB0FA
:1044C000BDE8F047FFF76CBA00F59A4048300AB0F3
:1044D000BDE8F047FFF7E0BA0AB0BDE8F047FFF7E4
:1044E00081BB00BF24170C08582C002070B500F5C4
:1044F000804200F59A43D2F8B42D48339A420546DB
:104500000E4602D00024204670BDFFF7B5FE0446DB
:104510000028F7D0318805F54F5052F057F8F2E7F0
:1045200021F04003152B04D0A1F15E0358425841FD
:104530007047012070470000102946D8DFE801F0DD
:10454000090D1115191D212529452D3135413939FF
:104550003D0000F59B400430704700F599405C3009
:10456000704700F599406430704700F599406C3011
:10457000704700F599407430704700F59A401C3040
:10458000704700F59A402430704700F59A402C306F
:10459000704700F59A404030704700F59A40483027
:1045A000704700F59A406030704700F59A406830D7
:1045B000704700F59A407030704700F59A407C30A3
:1045C000704700F59B400C3070470020704700009A
:1045D00000290DDB074890F8202CCBB29A4207D374
:1045E000D0F81C3C0122595CA0F5005005F0F6BD46
:1045F000704700BF584C00202DE9F34100F50053EF
:10460000044693F8F03B03F0010603F0020803F0C0
:1046100004075B0700F54F5535D01F4A0621284691
:104620004DF0F0FD26B104F53C50343076F00AFF31
:10463000B8F1000F04D004F542500C3076F07EFC47
:1046400027B104F54750243077F026FB04F5C04429
:10465000012384F8E930114A114B1249B8F1000FD7
:1046600008BF1A46002F08BF1946CDE900210E4A9F
:104670000621002E18BF134628460C4A4DF0C2FDF5
:1046800002B0BDE8F0810A4A0621284602B0BDE822
:10469000F0414DF0B7BD00BF51170C0846170C088C
:1046A00010F10C084D170C0840170C0862170C0885
:1046B00074170C0810B5044600F53C50343076F001
:1046C000EDFE04F542500C3076F064FC04F54750E2
:1046D000243077F01BFB04F5C04393F8E92052B176
:1046E000002283F8E92004F54F50034ABDE810404A
:1046F00006214DF087BD10BD94170C0809B1FFF7D6
:104700007BBFFFF7D7BF000000F580430A4AD3F80C
:10471000B41D91420DD093F8C13D43B900F59A42C2
:104720004832914203D100F5A04090F8E633184694
:1047300070470023FBE700BFDC79002010B504467A
:104740007CF070FD054BD3F8D43DC01A642804D822
:104750002046BDE8104056F08DB810BD586C0020C2
:1047600010B500F52F54D4ED087AF5EEC07AF1EECD
:1047700010FA8AB04FF0000304F1200445D90793E2
:104780000893099306AB019300F5985007AB00938B
:1047900003AA05AB04A9103008F090FE30B3DDED9C
:1047A000080A9DED070AA0F0FBFADDED090AA0F06A
:1047B000F7FAD4ED007A9DED047A77EEA76AB4EEAD
:1047C000E70AF1EE10FAF4EEC76AACBF0120002050
:1047D000F1EE10FA0CD802309DED037AF4EEC77AB0
:1047E000F1EE10FA0CD8003818BF01200AB010BD45
:1047F000F4EEC77AF1EE10FA9CBF0130C0B2EBE7DD
:10480000012894BF00200120F0E70020EEE700001F
:1048100010B5074B1A7A4AB901241C724AF044FCBD
:1048200022461121BDE810404AF0F6B910BD00BF84
:10483000588D002010B5074B1A7A4AB100241C721B
:104840004AF032FC22461121BDE810404AF0E4B99A
:1048500010BD00BF588D0020F0B5054685B005F5A8
:104860009856684610360FF057F96946304608F0FA
:1048700057FFA0B13248334C334F74F021FD40B1A3
:1048800005F52F53D3ED087AF5EEC07AF1EE10FA64
:1048900007D8002328462380FB73FFF7CBFF05B022
:1048A000F0BD2846FFF75CFF98B3637873BB2378AD
:1048B0000133DBB2082B237002D1304608F06AFEC8
:1048C0002378092B02D1304608F05CFE2378092BAF
:1048D0001CD94FF4857323804AF0E6FB0222102195
:1048E0004AF09AF97CF09EFC6368C01A47F2305394
:1048F000984208D9154A022105F54F504DF082FC27
:104900007CF090FC60602846FFF782FF6378FB73C1
:10491000C5E72678002EF9D0013E6378F6B22670FE
:10492000002BF3D0002EF1D166704AF0BDFB324669
:1049300010214AF071F92846FFF77CFFE6E700BF37
:104940009C8C0020588D0020058E0020A8170C0894
:1049500000F5A040D0F83834042B14BF90F864045C
:104960000120704773B500F580450192A5F8CC1D74
:1049700004467CF057FCC5F8D00DD5F8B40D03689B
:104980005B68984785F8CA0DD5F8B40D03685B6875
:1049900098470F28019A0BD80F2827D8DFE800F096
:1049A0001C261C1C1C1C1C1C1C264E260A260A0A23
:1049B00018281BD104F50056019296F9C033ABB10B
:1049C000D5F8B40D03685B68984785F8CA0D96F969
:1049D000C033019A022B27E01F4B93F8EA30F3B162
:1049E00004F59A411C31204605F01EFBD5F8B40DA4
:1049F00095F8CA6D03685B689847864204F54F5482
:104A000022D0D5F8B40D03689B689847134A034633
:104A10000421204602B0BDE870404DF0F3BB04F520
:104A2000005393F9C033022BDAD0042B0BBF04F5EB
:104A30009A4104F5994124315C31D4E72046FFF7CF
:104A400087FF0028D2D1B5E7054A0421204602B0ED
:104A5000BDE870404DF0D6BB588C0020B8170C084C
:104A6000DA170C08F0B5044604F5804685B00F4609
:104A7000154655F085FED6F8B40DA6F8CC7D036832
:104A80005B68984718281ED8DFE800F00D0D0D0D63
:104A90000D0D0D0D0D1D52680D0D57571D1D1D1DC2
:104AA0001D1D1D1D0D00314BD3F83824012A20D1C6
:104AB00004F5005393F8C133023B012B19D904F5D7
:104AC000405383F8BC23D6F8B40D294A294B052D51
:104AD00018BF1346026803939268904704F54F5439
:104AE0000090039B244A042120464DF08BFB05B027
:104AF000F0BD224B93F8EA303BB104F59A412A46C7
:104B00001C31204605F090FADDE704F5005393F9D7
:104B1000C133032B03D1204603F03EFAD3E7022B27
:104B2000EBD0042B15D104F59A412A464831E8E729
:104B30002046FFF70DFF0028C5D104F5005393F977
:104B4000C133032BE7D0022BD7D0042BEBD0012BA2
:104B5000B9D104F59A412A466031D2E704F50053F1
:104B600093F9C133042BAED1DDE700BF587C0020A0
:104B7000F0170C0827FC0B08F8170C08588C0020BD
:104B800070B5044600F54F56114A0421304604F52D
:104B900080454DF037FB0023A5F8CC3D04F50053CC
:104BA00093F80833032B12D195F8CA1D3022204602
:104BB00005F014FBD5F8B40D03689B689847054AC7
:104BC000034606213046BDE870404DF01BBB70BD6A
:104BD0000C180C0823180C0800F5405310B50022DF
:104BE0000529044683F8BC2300F54F500CBF054A45
:104BF000054A042104F580444DF004FB0023A4F889
:104C0000CC3D10BD3C180C084D180C0830B50B46B7
:104C100087B00446052A18D8DFE802F0172A0350A7
:104C2000175D00F5A043D3F83834042B20D02C4D69
:104C300095F8DD3DE3B12B49A1F6DC2025F086FE99
:104C400028B1294B012283F8642407B030BD2549DF
:104C5000A1F6DC2026F07AF950B104F59A4104223D
:104C60004831A5F5804007B0BDE8304005F0DCB91B
:104C700004F5A043D3F83834042BE6D004F50053F0
:104C800093F98B33022B0AD1154B93F8DD3D33B1E9
:104C90001449A1F6DC2025F059FE0028D1D104F5F5
:104CA0009A4104226031204605F0BEF904F50D500A
:104CB0000B3007B0BDE8304041F020BB0B4A11215A
:104CC00001A87BF013FB04F5BD4001AA01211C30B3
:104CD00077F0CEF8B9E707B0BDE8304003F05CB933
:104CE000586C0020908B0020587C002068180C081D
:104CF00070B52DED048B04467CF088FA4F4BB4F868
:104D0000BE101A884E4E8A4205464E4A06D0198079
:104D1000002330601370BDEC048B70BD33684A49CA
:104D2000C31A8B4276D90123137055F029FE55F032
:104D3000E1FC356055F024FE55F0DCFC04F54053F1
:104D400093F8BB3323B104F5BD401C3076F0E4FF8B
:104D500055F0F8FC0428DED955F012FD002120465C
:104D600003F03CFC00212046F0EE409A03F040FCAA
:104D700001212046B0EE409A03F000FE00212046BB
:104D8000B0EE408A03F03EFC04F5C0404430F0EE43
:104D9000408A74F09FFADFED2D7A0028B0EE690AA0
:104DA0004FF0040008BFB0EE678A57F0DFF9B0EEAD
:104DB000490A132057F0DAF9B0EE680A152057F0C7
:104DC000D5F904F5BD45B0EE680A1A2057F0CEF9C2
:104DD0001C354620B0EE480A57F0C8F9284677F04F
:104DE00029F808BB0121084657F0C2FC9FED170ABD
:104DF000022057F0BBF99FED150A032057F0B6F9D2
:104E0000204603F0D9FFBDEC048B2046BDE870407E
:104E100004F0E8BE1278002A3FF47DAF44F6206229
:104E200093427FF678AF80E72846FDF731F804F526
:104E3000A04393F9A63E2B2BD4D06CE7648D0020C1
:104E4000688D0020668D0020400D030000000000EA
:104E500000F5804200F59A43D2F8B42D48339A42C7
:104E600004D100F5A04090F86404E8B10F4B93F82A
:104E7000080303F58043A0F12702012A93F8F830D4
:104E80000FD92C2809D00A2809D0A0F131025042AC
:104E900050410A2B18BF002070470120F9E701207C
:104EA00070470A3B58425841704700BF584C002099
:104EB00008B500F5005393F8F02142B193F82C3275
:104EC0002BB1FFF7C5FF80F00100C0B208BD012083
:104ED000FCE700002DE9F04700F50055A64F95F8D6
:104EE0002C82044600F5C0408AB0443074F0E8F9E2
:104EF000D7F83834042B06464FD000284DD0B7F8E9
:104F00009A14A7F5A040FFF70BFB014620B197F8D4
:104F100060144B1E5942594104F50757DFF86CA243
:104F20003037384663F058FF9AF8F8300A2B81463C
:104F300003D1A6BB00238AF8F83095F8F031002B96
:104F400039D195F9F6318D4D012B03D0063BDBB2FB
:104F5000012B11D895F808330A2B0DD104F58046A2
:104F6000D6F8B40D03681B6A984728B1D6F8B81D67
:104F70002B22204605F058F89AF8F8300A2B04BF87
:104F800037238AF8F83095F808330A2B02D13723F3
:104F900085F808330AB0BDE8F0870121BCE740EA94
:104FA0000803DBB2002BC8D1AAF5C04000F0F0F82E
:104FB0000028BFD0C1E7002EECD004F5BC40103073
:104FC00079F0FEFE0028E5D12046FFF741FF0028DA
:104FD000E0D1B9F1000F00F0BF8069494A46384678
:104FE00063F0D2FA95F9F681B8F1010F07D040F3DA
:104FF0008780A8F10603DBB2012B00F281805FFA03
:1050000088F8B8F1010F4ED104F5804204F59A43B7
:10501000D2F8B42D48339A4209D104F5A04393F84D
:10502000643423B195F88B33013B012BB2D904F5DD
:105030009A410A226031204606AE04F0F5FF304660
:105040000EF06AFD95F9092292BBB8F1010F2FD03D
:1050500004F5A048B5F90A32D8F8241FDFED495A03
:10506000D1ED017A002BF8EEE77A52DD07EE103A27
:10507000F8EEC76AE6EEA57A3046FDEEE77A17EE5F
:10508000901A0EF04FFD00233846CDE9043363F04B
:105090003FFF04A964F09CFC002857D0049B0893B0
:1050A000059B099317E004F59A410A227031C2E783
:1050B0002046FCF765FF07EE900A6F4604F5BE42F6
:1050C000383221463846B8EEE70AFEF791F897E8FD
:1050D0000F0086E80F0095F9F631012B10D031460C
:1050E0002046FDF7DDFB31462046FDF769FF95F9C7
:1050F000F631072B04D104F54054012384F8BA3368
:1051000049F0D2FF4A4609210AB0BDE8F04749F00C
:1051100083BDD5ED7E6A95ED815A95ED7F7A35EEAA
:10512000076A36EEC57AB4EEC67AF1EE10FA89BF98
:1051300037EE067A95EDFB7A27EE257AF6EE006AD1
:1051400094BFE7EE257AE7EE267A95E7D8F8243F74
:105150009A680892DB68A4E7B8F1000F3FF41AAF31
:1051600095F82C32002B7FF415AF074A052104F582
:105170004F504DF047F8C3E7587C0020584C0020B2
:1051800074180C080000C8427D180C08588C0020C8
:1051900010B5044600F5C040443074F09BF804F5A7
:1051A000A04404F23C4494ED007A48B1DFED067A65
:1051B000B4EEE77AF1EE10FAACBF0120002010BD8A
:1051C000DFED027AF4E700BFCDCCCC3D6666663FEA
:1051D00000F58043D3F8B41D00F59B430C3399428E
:1051E00004D100F5A04393F830249AB900F59A430E
:1051F0004833994210D100F5A04393F830244AB1C6
:10520000D3F83824032A07D1B3F89A24A2F116035D
:105210005A425A41104670470022FBE72DE9F84FE9
:1052200000F5804200F59A43D2F8B42D48339A42F3
:10523000054600F5A04704D100F5005898F96433FD
:1052400033B90023C7F8243487F82134BDE8F88F38
:105250007BF0E8FFD7F8D843814634B1041B40F611
:10526000C3139C4294BF002401242846FFF790FFFB
:10527000834620B1002487F8204400263FE005F54E
:10528000C040443074F01CF882460028F2D005F586
:10529000BC461036304679F093FD002840D097F890
:1052A0002064C6BB44B305F5805141F27072D1F859
:1052B0000835002BB8BF5B42934206DCD1F80C35B1
:1052C000002BB8BF5B42934228DD05F5A94105F5E7
:1052D000BE40203138300EF081FFDFED467AC7F84E
:1052E0002494B4EEE70AF1EE10FA4FF000034CBF3D
:1052F00001260026C7F82834012387F8203405F555
:105300009070F8F70FFC022835D9002C46D1002305
:10531000C7F824349AE75C465E46EDE73446EBE78F
:10532000304679F035FD064638B1002CA5D04FF453
:10533000FA73C7F8283454469FE7D7F83834012B5E
:1053400003D0032B0FD03446D9E708F20443D3ED42
:10535000007AF5EEC07AF1EE10FAF4DD97F8303409
:10536000002BF0D1E3E72846FFF732FF0028EAD10F
:10537000002CDCD1C3E705F5005A0AF1380A98F889
:105380008611504606F09AFA0028C0D098F8861187
:10539000504606F08BFB0028B7D1B8E7D7F8243485
:1053A00013B9C7F8249451E7D7F82824A9EB0303CD
:1053B0009342FFF44BAF97F82134002B7FF446AFB4
:1053C000012287F8212498F86433DB0705D505F519
:1053D000C0400C214430F8F7DBFA05F54F502EB1F0
:1053E000054A0221BDE8F84F4CF00CBF034A314694
:1053F000F8E700BF0000964294180C08AA180C08A1
:105400002DE9F04F2DED028B054685B0002305F503
:10541000005803937BF006FFD8EDD87AF5EEC07AFA
:10542000F1EE10FAC4BF9FEDC07A67EE877A05F5FA
:10543000907BC8BFFCEEE77A07465846CCBF17EE14
:10544000906A9626F8F76EFB022840F2008195F8E4
:1054500014349FEDB67AB02202FB0353D3ED837A66
:1054600067EE877AFCEEE77A17EE903A9E428CBFA1
:1054700000260126B8F95433022BB8BF022307EEE9
:10548000903A05F59850B8EEE78A03A9F6EE087A47
:10549000103028EE278A08F021F9044640B1DDEDEE
:1054A000037AF4EEC87AF1EE10FAACBF01240024BE
:1054B0005846F8F737FB05F5C049012809F14409BA
:1054C00005F5A04A18D8484673F0FAFEA0B19CB979
:1054D0000AF23C4292ED007ADFED957AB4EEE77A7B
:1054E000F1EE10FA08DDDDED037AF4EEC87AF1EEA4
:1054F00010FAACBF01240024484673F0E1FE00908E
:10550000002800F0FE8095F8142405EB0212D2F872
:10551000C02172B158460192F8F704FB012800F24D
:105520009880019A41F28731BA1A8A428CBF0022D0
:105530000122DAF8D41301B11AB9002C40F08B80A3
:10554000344605F5804105F59A42D1F8B41D48323C
:1055500091421AD198F98C23002A40F084800022CD
:105560008AF82224DAF83824042A00F0AC80072ACA
:1055700000F0BD80032A08D12846FFF729FE20B19C
:1055800000248AF82144CAF8D8439AF8222402B1A8
:105590008CB907EE904A9FED677AF8EE677A0AF2C7
:1055A0003C4267EE877AD2ED006A9FED637AE6EEC1
:1055B000877AC2ED007A2846FFF7EAFD0446A8B1D3
:1055C0009AF84004CAF8D47308B9CAF8447405F5C7
:1055D000804105F59A42D1F8B41D4832914205D177
:1055E000DAF8D82302B108B9CAF8D8739AF868254E
:1055F0008AF8404464F3C3028AF868256DF0ACFF72
:1056000021466DF085FF4D4A28465471FFF706FE8E
:105610002846FBF793F934B198F80A231AB97BF0BE
:1056200001FEC8F80C0388F80A432846FFF7B0FDCE
:10563000002877D1484673F04DFE80F00100C0B2DB
:105640008AF8480405B0BDEC028BBDE8F08F002657
:1056500010E700226DE71FF0F5F81EF043FA00286E
:105660007FF46EAF6DE7524207EE902A05F6C8024E
:10567000F8EEE77A92EDDB7AF4EEC77AF1EE10FA03
:1056800013DD01228AF82224CAF82C740AF23C4263
:10569000DFED2B7A92ED007AB4EEE77AF1EE10FAB4
:1056A0007FF760AFC2ED007A5CE79AF82224002A07
:1056B0003FF458AFDAF82C2440F6B831BA1A8A42CF
:1056C0003FF64DAF4EE705F5BC40103079F060FB7A
:1056D00000283FF45AAF9AEDF17ADFED197AB4EE73
:1056E000E77AF1EE10FA7FF750AF009C4DE79AEDA4
:1056F000F17AFEEE007AB4EEE77AF1EE10FAF4D425
:1057000043E7DAF83824002C18BF3446012A07D0C2
:1057100005F5BC40103079F031FB00283FF435AF7F
:10572000002432E700208BE70000B4420000C842AA
:105730009A99993E9A99193E9A99593F058E002057
:10574000CDCC4C3E002070470020704701207047B0
:105750000020704701207047034BD3F83804431EE4
:1057600058425841704700BF587C002030B587B080
:1057700002A80EF0D1F9304879F000FB20B12F4992
:105780002F48FDF79FF81FE02B4879F001FBE8B1A7
:105790002C4C04F12405234604F11002A4F110015D
:1057A000A4F59470009579F019FBCDE90045A4F6B5
:1057B000387292EDF30A244904F11003A4F11002A7
:1057C000A4F5947079F0CCFA07B030BD1A4802A95C
:1057D00079F01CFB08B102A9D2E7194802F09EFA41
:1057E0000028CCD1194C94F8483F5B071DD4D4F85D
:1057F0005C3F002BC3D0114AA2F12001A2F110009E
:105800000EF058FC0028BAD1D4EDF47A0B490C48BC
:10581000B7EE000A30EE670AFDF784F80C4A084834
:1058200002F12001FCF708FCCEE7A4F5A040FDF74B
:10583000F9F80028C8D1DAE7688A0020A08B002098
:10584000582C0020908B00207C580020587C002091
:10585000808B002008B50A4890F8FD33013B012BEE
:1058600003D8A0F50050F9F7B5F90648F9F7D8F8CC
:105870000448F9F775F9BDE808400248F9F79CBCFF
:10588000584C0020582C0020124A904208B50ED0E7
:1058900002F1080188420AD002F11001884206D0C4
:1058A00002F13801884202D05C32904206D10A4BA4
:1058B00093F9B503B0FA80F0400908BD03681B6A8C
:1058C000984728B1054B93F8BA0380F00100F4E73C
:1058D0000120F2E73C790020584C0020585C002061
:1058E000104A904208B518D002F10801884214D03D
:1058F00002F11001884210D002F1380188420CD028
:105900005C32904209D003681B6A984738B1064B55
:1059100093F8BA0380F0010008BD0020FCE70120E5
:10592000FAE700BF3C790020585C0020024A026080
:10593000024A4260704700BFFC180C08683F002014
:1059400008B50368DB6D98470648D0F8B42D00F51C
:1059500054639A4205D0BDE80840A0F58040FEF7A8
:10596000A9BE08BD586C00202DE9F041474CA4F5B4
:105970002E73C11A4B42A4F500584FF000054B415D
:10598000002284F89053A4F8E65384F8EA53C4F84C
:10599000AC2384F8A85384F8215484F82254C4F822
:1059A0001054C4F80C54C4F80854C4F81854C4F87B
:1059B000BC2388F85C364368D3F8FC31A4F8E033A4
:1059C00004F6387306460FCB04F6287787E80F00F5
:1059D00084F8E95384F8F853C4F8045F7BF022FCA0
:1059E000A4F58057C7F8BC0D336830465B6998470B
:1059F0004FF0FF3384F8EC0384F8ED5388F8BC5380
:105A000084F8615F84F8EB53C7F8E43D33683046AF
:105A10009B6D98470546002835D0336830469B6B10
:105A2000984784F83004D8F8E8050368DB6B98479A
:105A3000A7F6A84075F06EFEA4F5A04002F03CFD6C
:105A4000A8F5616063F02EFA94F86434C3B1A4F54C
:105A5000A040FFF79DFB98B90D4873F03BFC78B967
:105A6000D7F8B40D03685B6B984748B953F096FAC2
:105A7000084A06214CF0C6FB04F25C4025F012F8FF
:105A80000548F8F70BFB2846BDE8F081587C00205C
:105A90009C8C0020BC180C08582C002070B50368A2
:105AA0001B6E0E4615469847044650B995F90030CE
:105AB0003BB90548054B00683246C06A29461CF0D0
:105AC000A7F8204670BD00BF542C0020E0180C0839
:105AD00010B50D4C204675F019FC04F5AC7075F04E
:105AE00091F904F52C7076F0BFF8084B03F5A0424D
:105AF000002182F8A81303F500530021C2F8AC136B
:105B0000012283F8802E10BD8C5B0020582C0020D1
:105B100008B52DED028B1520B0EE408A56F026FB1D
:105B2000B0EE480ABDEC028B1A20BDE8084056F0E2
:105B30001DBB000008B5084890F9B5330121A0F558
:105B4000005033B102F01AFFBDE80840462056F07D
:105B50000DBB02F03BFFF7E7584C002004207047D4
:105B60000048704772870D080048704772870D081B
:105B7000037A73B1D0ED037AFDEEE77A17EE903A2F
:105B8000084AC2F84C34437A3BB10369C2F8503436
:105B900070474368D3F8F831F2E74368D3F8FC3133
:105BA000F4E700BF587C002008B50023038100F112
:105BB0001401406807F0A8FD012008BD70B56E4EC5
:105BC0002DED048B06F59B4304460121304693EDF1
:105BD0001F9ADFED6A9A02F001FD0121B0EE408AC2
:105BE000304602F005FDC8EE297A06F500556068DA
:105BF000B5F9D83304F1140108EE903AF8EEE88ACA
:105C0000B5F9DA3368EEA78AC0EE297A08EE103AC1
:105C1000B8EEC88A28EE278A07F076FD95F9DE33BC
:105C200063B39FED577AF0EEE87AF4EEC77AF1EEBF
:105C300010FA23D5227A6368002A55D101222272F4
:105C40000022E26094ED037ADFED4E7AD3F8F8316A
:105C50004D4A4E4867EEC77A9FED4D7A67EE877AD8
:105C6000B0EE490AFDEEE77A17EE901A0B44C2F83F
:105C70004C340023012275F0D9FA08E00023434890
:105C80002372F0EE490AB0EE680A75F0CBFA0420F0
:105C900056F06CFA95F9DE3343B19FED397AF0EEA8
:105CA000C87AF4EEC77AF1EE10FA28D40023394806
:105CB0006372F0EE490AB0EE480A74F00DFF13204B
:105CC00056F054FAB5F9DC33002B03DD324E96F969
:105CD000FA3163BB28482021F8F74CFC002843D157
:105CE000254802F0BBFA42E0D3EDC56A96ED467A4C
:105CF000D4ED037AE6EE877AC4ED037AA2E7637AFD
:105D00002BB9012363726368D3F8FC3123611E4B06
:105D10002169C3F850146368D3F8FC010023091A01
:105D20001A461C48B0EE490A74F0BCFFC7E70121CF
:105D3000A6F5405002F066FC80EE297AB5F9DC3316
:105D4000002106F5F27007EE903AF8EEE77AF0EEF1
:105D5000490A27EE870A75F087FEBDEC048B2046C2
:105D6000BDE87040FFF7D4BE0348F9F791F807EE9D
:105D7000900AB8EEE70AF0E7582C002000A08C4506
:105D800000000034E02E6542587C00208C5B00202F
:105D90000000C842E45C0020585C00202DE9F04F70
:105DA0002DED0C8BDFF8A8A39FEDDEDA9FEDDE9AD8
:105DB00097B00AF59B4300F11405044601215046B3
:105DC00093ED1FBA02F00AFC01215046F0EE408A22
:105DD00002F00EFC01215046B0EE408A02F012FCA7
:105DE000DFEDD27A88EEA77A0AF5005601A8B6F957
:105DF000D8330AF5A04B0AEE903AF8EEEAAAB6F9C3
:105E0000DA33DFEDCB8A6AEE87AA88EE277A0AEECC
:105E1000103AB8EECAAAB6F9DC339FEDC68A2AEE6C
:105E200007AA80EE277A09EE903AF8EEE99A6AEE30
:105E30008D7A69EE879AF0EEEACAF4EEC8CACDED23
:105E4000017AB0EECACA6AEE0D7AF1EE10FAF0EEFF
:105E5000E9BAB4EEC8CACDED027A58BF4FF00109D5
:105E600069EE8D7A48BF4FF00009F1EE10FAF4EEBA
:105E7000C8BA9AED460ACDED037A54BF4FF0010837
:105E80004FF00008F1EE10FA54BF0127002721F06F
:105E900085FC01A9284620F0A1FF284621F090F8B2
:105EA000284621F007F820EE090A284620EE280AA5
:105EB000BDEEC00A10EE103ACBF84C3421F014F8C5
:105EC00020EE090A20EE280ADFED9B8ABDEEC00A0B
:105ED000CDED0D8A10EE103ACBF850340DF1280BB1
:105EE0004FF07E53594660680A93CDED0C8ACDED94
:105EF0000B8A07F009FC0021504602F03FFDB0EE8E
:105F0000C00AB4EEC80AF1EE10FA16D55046FFF7F3
:105F10003FF990B9F4EEC8CAF1EE10FA0DD5B4EE1F
:105F2000C8CAF1EE10FA08D5F4EEC8BAF1EE10FACC
:105F300044BF9BE80F0085E80F000AA821F0A4F8F1
:105F4000294612A88DED141A8DED120ACDED130A13
:105F5000CDED151A21F0AAF80DF1100A51460EA840
:105F60008DED101ACDED048ACDED058ACDED068AB2
:105F70008DED0E0ACDED0F0ACDED111A20F068FE61
:105F8000B6F9D833DFED6D7A01EE103AB6F9DA33AF
:105F900009EE103AB6F9DC3308EE903AB8EEC11AC1
:105FA000B8EEC99AF8EEE88A21EE271A29EE279A68
:105FB00068EEA78AF4EEC8CAF1EE10FA21EE0D1AC7
:105FC00029EE0D9A68EE8D8A07D594F82430DFED1E
:105FD0005A7A002B18BFB0EE671AB4EEC8CAF1EEB9
:105FE00010FA07D594F82530DFED537A002B18BF4F
:105FF000B0EE679AF4EEC8BAF1EE10FA07D594F84D
:106000002630DFED4D7A002B18BFF0EE678A9AE854
:1060100007000DF11C0B8BE80700F1EE410AC220CE
:106020009DED070A1FF046F9C3208DED070AB0EE7B
:10603000491AF1EE490A9DED080A1FF03BF9B0EE4E
:10604000681AF1EE680A8DED080AC4209DED090A70
:106050001FF030F9514658468DED090A21F034FB06
:1060600012A928468DED120ACDED130A8DED141AF2
:1060700006F6387620F0B2FE284620F0A1FFDDEDCE
:10608000076A96ED007A2E4B9FED270AC6EE877AB7
:106090005846DDED086ACDED077AD3ED247A86EE19
:1060A000A77ADDED096A8DED087A86EEA77A8DED87
:1060B000097A21F073FBB9F1000F01D0CDED07AAE9
:1060C000B8F1000F01D08DED08AA0FB1CDED099AFE
:1060D000F0EE4B0A9DED070A1A4875F0A3F804206C
:1060E00056F044F8F0EE4B0A9DED080A164874F09D
:1060F000F3FC132056F03AF80021F0EE4B0A9DED28
:10610000090A124875F0B0FC2046FFF701FD84F83B
:10611000249084F8258084F8267017B0BDEC0C8B91
:10612000BDE8F08F35FA8E3CE02E654200A08C452C
:106130000000C8420000003400000000CDCC4C3EFE
:10614000585C00208C5B0020E45C00203C5E00205A
:10615000582C002010B50446FFF7ECFC0B4B93F9CC
:10616000DE23022A0DD1B3F9DC23002A09DD03F571
:10617000805393F9FA3123B12046BDE81040FFF770
:106180000DBE2046BDE81040FFF718BD584C00205A
:106190000A2070470048704789230C080048704760
:1061A00089230C08012070470120704701207047A7
:1061B0000120704701207047034BD3F83804031FB8
:1061C00058425841704700BF587C0020F8B5194D1F
:1061D00005F638730FCB05F6287405F6487684E883
:1061E0000F0086E80F00002705F25C4085F8EC738D
:1061F00024F098FE104B1C68E66A336830465B68F2
:106200009847A8B196F84D3093B1E36A9B8F7BB164
:1062100052F0C4FEE36A094A9B8F06214BF0F2FF5D
:10622000E36A05F25C40998F24F068FCE36A9F877B
:106230000120F8BD587C0020542C0020CC190C08FB
:1062400010B50A4C94F86034012B0BD104F25C4079
:1062500021F012FFB4F89A34152B03D104F56160D4
:1062600078F06CFE0023C4F8D83310BD587C0020B1
:1062700008B507F04FFC90F87C32DB0704D5BDE889
:106280000840024824F0EABC08BD00BFB4800020EA
:1062900010B5304C94F86034012B0ED0A4F5287161
:1062A0000822A4F5A04003F0BFFE52F077FEBDE83F
:1062B0001040294A06214BF0A5BFB4F89A34162B9A
:1062C00005D0152B36D1D4F83834072B0AD1234802
:1062D00004F028FA214804F061FBBDE810401F4893
:1062E00004F080BAA4F5A040F9F7D0F8A4F5A040D6
:1062F000F8F7CEFFA4F54053D4F84C1493F91C24BE
:1063000064235A4304F5616078F074FDC4F84C04CA
:1063100004F5616078F0B0FE30B1BDE810409FED4B
:10632000100A462055F022BFA4F5A040BDE8104059
:10633000F8F796BD1E2B18BF4FF0FF33074818BF64
:10634000C4F8A433F9F7A2F80448F8F7A1FF03480A
:10635000ECE700BF587C0020E4190C08582C002002
:106360000000000010B5144BB3F89A34532B0446C8
:106370001ED102F0F7FE9FED110A462055F0F6FE01
:106380009FED0E0A492055F0F1FE9FED0C0A4A20C0
:1063900055F0ECFE462055F0C9FF492055F0C6FFE8
:1063A0004A2055F0C3FF2046BDE81040FFF790BBE0
:1063B000BDE81040FFF74EBA587C002000000000F6
:1063C00008207047004870477C1A0C080048704746
:1063D000881A0C080120704708B50248FEF70CF92E
:1063E000012008BD582C0020014800F059B900BF19
:1063F0007479002010B50446FFF72CFA2046BDE85A
:106400001040FFF797BB000001207047004870471D
:10641000FC1A0C0800487047041B0C080120704748
:106420000120704710B5054B03F6487403F6387326
:106430000FCB84E80F00012010BD00BF587C002066
:1064400008B50B4800F5A04200F500530321D3F82E
:10645000143C93FBF1F3C2F84C34F8F77DFF044889
:10646000F8F716FFBDE808400148F8F7F9BC00BF8F
:10647000582C00200720704700487047E4FD0B08A7
:1064800000487047781B0C080120704701207047B6
:10649000012070477047000008B5002303720361B4
:1064A0000248FCF7CBF9012008BD00BF582C0020A2
:1064B00010B5194CD4F8FC3BB3F9083023B9D4F823
:1064C000083CB3F90830F3B1002303720361D4F838
:1064D000FC0B54F045FB04F61443D3ED007A0F484F
:1064E000F8EEE77A27EE800ABDEEC00A10EE103A09
:1064F000C0F84C34A0F5A040F8F72EFFBDE81040DE
:10650000074801F029BB037A002BE0D0A4F5005026
:10651000F8F7BCFFF2E700BF584C0020587C002081
:10652000582C002070B54E4DDFED4E7A95F814349E
:106530009FED4D7A2DED048BB02606FB035393EDB2
:10654000848A9FED4A9A28EE278A05F5A853BDEE66
:10655000C88A93ED070AF8EEC87A044667EE897A8E
:1065600097EE870A1EF092FE237AF0EE408A002B07
:1065700062D105F50053D3F8FC3BB3F90830002B8A
:106580005AD1284601F06AFE002855D195F81434F6
:1065900095F8581406FB035393F8F12100294BD1C9
:1065A000012A49D993ED837AF0EE087AB4EEE77ABE
:1065B000F1EE10FA40DBDFED2E7AB0EEE80AB4EE31
:1065C000E70AF1EE10FA37D5236993B37AF02AFE81
:1065D0002369C01AB0F5FA7F32D8237A002B3CD059
:1065E000244DA5F1200696E80F0085E80F0094EDF4
:1065F000038AA5F110013046B8EEC88A0DF0EEFD11
:1066000028EE098ADFED1C0A284670EE200AB0EE5B
:10661000480A0DF059FE194B9FED190AD3F8E80509
:10662000BDEC048B03682A4631469B6ABDE8704086
:1066300018477AF0F7FD20612369002BCDD0C5E71C
:10664000104D84ED038A012323720023236105F199
:1066500010030FCB85E80F00BFE7BDEC048B70BDC6
:10666000582C00200000C84235FA8E3C0AD7233C43
:10667000DB0FC93FA08B002000007A44585C00204B
:1066800000000000808B0020052070470048704704
:10669000EC1B0C0800487047FC1B0C0801207047DD
:1066A00038B52DED028B4A4C9FED4A8AD4F8FC0B8D
:1066B00054F056FAD4F8143C07EE903AF8EEE77A24
:1066C00004F5405527EE800AA4F50050BDEEC00A3F
:1066D00010EE103AC5F84C34F8F73EFED4F8000C32
:1066E00054F03EFAB5EEC00AF1EE10FADABF04F645
:1066F0001843D3ED007AD4EDDB7A3748CBBF20EED8
:10670000270A20EE270A20EE080A28EE400ABDEEEE
:10671000C00A10EE103AC5F85034F8F7E9FD94EDD0
:10672000DB7AD5F8500404F6184327EE087AD3ED47
:10673000007A27EE888AFDEEC77A17EE902AFDEEE2
:10674000C87A17EE901A1EF055FEC5F8500422487C
:10675000FDF7DAFF20B1D5F850345B42C5F850346C
:106760001E4B93F8C83D63B194F9C033022B08D196
:10677000002301214620C5F84C34C5F8503456F0AA
:106780004FF854F0FDF85F2155F0A2F9E8B155F04B
:106790006FF9022819D195F8E933B3B904F20C4422
:1067A00095EDEF7AD4ED007AB4EEE77AF1EE10FAD7
:1067B0000BD5012385F8E933BDEC028B084A094863
:1067C000BDE8384004214BF01DBDBDEC028B38BD47
:1067D000584C00200000C842582C0020586C002063
:1067E000041C0C081860002010B50446FFF732F8AE
:1067F0002046BDE81040FFF79DB900000620704715
:1068000000487047801C0C0800487047901C0C081A
:106810000120704701207047012070470120704718
:106820007047000008B50248FCF708F8012008BDD1
:10683000582C002038B50F4C04F50055D5F8FC0B4A
:1068400054F08EF905F61442D2ED007AF8EEE77AAC
:1068500004F5A04327EE800A2046BDEEC00A10EEE4
:10686000102AC3F84C24F8F777FD2046BDE83840DD
:1068700001F072B9582C00200F2070470048704773
:10688000041D0C08004870470C1D0C0801207047BF
:106890000120704701207047012070470120704798
:1068A0007FB50B4D05F54053002283F8BA2305F55B
:1068B000BE43383306460FCB6C4684E80F000023F6
:1068C0002846B3602146FCF77BFB012004B070BD75
:1068D000582C002010B53C4CD4F80834002B2CDD8B
:1068E0007AF0A0FCD4F80834C01A40F6B7339842C6
:1068F00023D8A4F54053D4F8FC03D3F8142C514208
:106900001EF078FDC4F84C04A4F5A040F8F724FD6F
:10691000D4F80C34002B14DC2C48F8F7B9FC2C48C4
:1069200090F8BA3393B30121A0F5405002F026F855
:10693000BDE81040462055F019BC2448F8F7A6FDE4
:10694000E6E77AF06FFCD4F80C34C01A40F6B7339F
:106950009842E1D81F4BDFED206A93EDDB7AD4F843
:10696000000403F61843D3ED007A27EE267A67EE8B
:10697000A67ABDEEC77AFDEEE77A17EE102A17EE7B
:10698000901A1EF037FDC4F85004C8E7A0F58050F7
:1069900090F94B33012B04DCBDE810400B48F8F7AD
:1069A0005FBAD4F81834002BF6D07AF03BFCD4F858
:1069B0001834C01A40F6B7339842EDD804F21444A4
:1069C00094ED000AB4E700BF587C0020582C00204A
:1069D000585C0020584C00200000C842D0ED027ADC
:1069E0000348FCEEE77A17EE903A99B201F07ABAD2
:1069F000582C002084B010B503AC84E80E000B487E
:106A000021466F22FCF722FA9DF80C1011F00401C8
:106A100002D120460DF04AF904482146FCF7D0FA8D
:106A2000BDE81040012004B0704700BF582C002082
:106A3000B0EEC00AFDEEC07A38B54FF6FF720546DB
:106A40000C4617EE900A00211EF0D4FC07EE900AC7
:106A5000002CF8EEE77A054BC5ED027A14BF4FF033
:106A6000FF32012283F8002F38BD00BF587C002080
:106A7000FEF77CBE0C20704700487047801D0C0854
:106A80000048704761870D0801207047012070475A
:106A900001207047012070470120704708B50C485D
:106AA000FDF7CAF80A480B49FBF7FAFE0848F7F762
:106AB00041FF40B106484FF48051F7F75BFD10B13C
:106AC0000348FBF7BBFE024800F0C0FD012008BDF3
:106AD000582C0020A08B002008B50D48F8F7D6FCF4
:106AE0000B48F7F727FF50B109484FF48051F7F7EB
:106AF00041FD20B1BDE80840054801F02DB804482B
:106B0000F8F7C6FBBDE808400148F8F7A9B900BF8F
:106B1000582C002008B50A484FF48051F7F72AFD99
:106B200038B108480022D0F8581F00F648700CF021
:106B3000F9FFBDE808400248002101F0D3B900BFC9
:106B4000582C0020587C0020881A10B51EF07AFBC3
:106B5000104BD3F8FC2E0028B8BF4042002AB8BF23
:106B6000524248F6A041B2FBF1F24FF47A7102FBB7
:106B7000011188420CDC93F8482FD20606D503F6A3
:106B8000487403F638730FCB84E80F00012000E04F
:106B9000002010BD587C002084B070B52DED048B12
:106BA00086B00FAD85E80E004E4CDFED4F8A0646ED
:106BB000D4F8E80504F5005404F6147393ED000AC4
:106BC0000368B0EEC00A5B6A9847B4EEE80AF1EEDB
:106BD00010FAB0EE408A07DA012006B0BDEC048B53
:106BE000BDE8704004B07047404928460DF002FAF5
:106BF00002A8CDED030A8DED020A20F0C3FC04A823
:106C00008DED040AB0EE480ACDED050A20F0B4FB84
:106C100013A928468DED000ACDED010A0DF0EAF921
:106C200002A88DED020ACDED030A20F051FCB4EE6E
:106C3000E80AF1EE10FACFDBB4EEC08AF1EE10FAFA
:106C40009FED2B9ADFED2B8ADFED2B9A2BD802A834
:106C5000694620F081FB04A88DED040ACDED050AFC
:106C600020F0ECFB684620EE098A20F0E7FB94F95F
:106C7000003F07EE903AF8EEE77A28EE288AA7EE72
:106C8000A90A1EF003FB20EE090ABDEEC88A20EE19
:106C9000280A18EE101AFDEEC07A304617EE902A38
:106CA000FFF752FF99E738EE400A38EE088A80EE87
:106CB000080A9EF00DFA02A8B0EE408A20F0BEFB52
:106CC00094F9003FF0EE007AB0EE697AA8EE677AA8
:106CD00007EE903AF8EEE77AA7EE270A1EF0D6FA0A
:106CE000C0E700BF585C002000000034908B0020FB
:106CF000E02E65420000C842DB0FC93F10B50446D4
:106D00000848F7F717FE20B92046BDE81040FEF707
:106D10002DBD04484FF48051F7F72CFC0028F3D028
:106D200010BD00BF582C002000207047004870475D
:106D3000F41D0C0800487047FC1D0C08002070472B
:106D40000020704738B5154C05460021204601F05B
:106D500045FC042055F00AFA0021204601F048FCC9
:106D6000132055F003FA0021204601F04BFC284681
:106D7000FEF7CEFE2046012101F000FE462055F030
:106D8000F5F96B6804F5A044D3F8F831C4F84C3435
:106D90006B68D3F8FC31C4F8503438BD582C00204F
:106DA000FEF796BE0B20704700487047B7160C08D8
:106DB00000487047701E0C08012070470120704782
:106DC000012070470020704770B50B4E06F5A045B6
:106DD00005F638730FCB05F6287484E80F003046AB
:106DE000FBF7CEF801463046FCF7B8F9002385F8EA
:106DF000B83F012070BD00BF582C002038B5304886
:106E0000F8F744FB2E48F8F743FA2D48F8F728F82E
:106E10002B481021F7F7AEFBE0B12A4AD2F83C3FED
:106E2000D2F84C2F9342D4BF00230123254C94F871
:106E3000B82F72B973B304F638730FCB04F6287504
:106E400085E80F00A4F5A040FBF7F4FA012384F8CD
:106E5000B83F38BD1C4AB2F9E41B0029F9DD02F540
:106E600040529FED1A7AD2F83C3FD2F82C2F9B1A51
:106E700007EE903AF8EEE77A67EE877A07EE101A97
:106E8000B8EEC77AF4EEC77AF1EE10FACCBF012360
:106E90000023CBE7A4F54053642193F91C24D4F8D4
:106EA0004C0412FB01F2D3F8141C8A42A8BF0A4614
:106EB0005142C3F8142C1EF09DFAC4F84C04C8E7E4
:106EC000582C0020587C0020584C00200AD7233C26
:106ED00038B52B4DB5F9B03383EAE371A1EBE3711B
:106EE00089B205F5405431B1002BB4BF4FF0FF33E8
:106EF000012384F8003F234800F0F4FF94F8EA33BC
:106F0000F3B995F98B33022B1BD11F4D95F8DD3D5D
:106F10009BB11E49A1F6DC2024F018F868B10123CA
:106F200084F89534282205F64851A5F5804003F0F1
:106F30007BF828B9002384F89534012384F8EA33D8
:106F400038BD012B0CD10F4800F0E8FE40B10D48D0
:106F5000FBF72AFA0028B8BF4042B0F57A7FD4DBAD
:106F600095F98B33042BEBD1074D95F8DD3D002BC4
:106F7000E3D00649A1F6DC2024F064F8CEE700BF98
:106F8000584C0020582C0020586C0020908B00207A
:106F90000220704700487047E41E0C080048704704
:106FA00056870D08034B0022C3F84C24C3F8502425
:106FB000704700BF587C002038B5094D044628466C
:106FC000F7F72EFD2846F7F7CBFD2046F7F7E0FD53
:106FD0002846F8F7F1F82046BDE83840FEF7AABD8C
:106FE000582C00200D207047004870475C1F0C088B
:106FF00000487047641F0C0801207047012070474B
:10700000012070470023C37480F8243001207047AA
:107010000148002100F066BF582C0020F0B5B54CA7
:10702000D4F8442FD4F8403F2DED088B1343D4F807
:107030003C2F134389B005460FD1AF48F8F726FA25
:10704000AD48F8F725F99FEDAD0A462009B0BDEC33
:10705000088BBDE8F04055F089B806F05BFD90F86C
:107060007C32DB07E9D5B5F90830E97C09EE103A46
:10707000B5F9103008EE903AB8EEC99AF8EEE88A01
:10708000002940F0D7809FED9EAA29EE0ABA01227E
:10709000FDEECB7AA4F5A040C4EDED7AFAF79CFFA3
:1070A000686800F57F700790B0EE408A20F0C6F95E
:1070B000DFED947A20EE270A1EF066F80798F0EECE
:1070C000409A20F005FAA4F5A040F0EE40AAFEF7A1
:1070D0005FF8002879D104F6387696E80F0005F1BC
:1070E000140787E80F0096E80F0004F6287787E872
:1070F0000F0004F6487787E80F00D4F84C3F824829
:1071000007EE903AF8EEE77AF0EE680A77EE8B7ABF
:10711000B0EE690AFDEEE77A17EE903AC4F84C3FFC
:107120000DF0D2F8002384F8213495F9123072481A
:1071300003EB830303EB83039B000121A4F8E233F9
:10714000F6F75EFF94F83074002F73D16F4B9FED0C
:10715000707AB3F9543307EE903AF8EEE77A67EEB7
:10716000877AF4EEE7AAF1EE10FA63DD51F016FF2C
:10717000064619EE900AF5F7C7F9CDE9040118EEB5
:10718000900AF5F7C1F9CDE9020119EE100AF5F7F9
:10719000BBF9604ACDE90001062130464BF032F8D8
:1071A0007AF040F8C4F8A073C4F88C037AF03AF887
:1071B0000123C4F89C0329EE8A0AEB741EF00EF832
:1071C000BDEEC00A84EDE90A34E07AF02BF8D4F879
:1071D0004434C01A42F2107398427FF67CAFF0EE4E
:1071E000087AF4EEE7AAF1EE10FA7FF774AFBCEE7E
:1071F000C88A04F6487718EE103A9BB208EE103AA7
:10720000B8EEC88A04F63876B4EEC89AF1EE10FAF1
:1072100046D851F0C3FE404A06214AF0F3FF96E8F3
:107220000F0087E80F000123EB740321A4F5A040B1
:10723000F6F7E6FE304803F0FBFC28B12E480321A8
:10724000F6F7DEFE0023EB74D4F83834012B40F05F
:10725000B480D4F83C3FAA699FED29AA9B1A07EE97
:10726000903AD4F8A4330133F8EEE79A5CD0DFED1E
:107270002B7AE9EE0A7AF4EEE79AF1EE10FA0ADADE
:10728000274905F114000CF0A9FFF4EEC08AF1EED5
:1072900010FA00F2928018480321F6F7B1FE8CE054
:1072A00051F07CFE1F4A06214AF0ACFF96E80F0021
:1072B00005F1140C8CE80F0096E80F0087E80F002A
:1072C000D4F84C3F07EE903A39EE488AF8EEE77A68
:1072D000F0EE680AE8EE0A7A3846B0EE690AFDEE8A
:1072E000E77A17EE903AC4F84C3F0CF0EDFF01211D
:1072F000E9749BE7587C0020582C00200000000017
:107300000000C842E02E6542A08B0020584C0020AF
:107310009A99993EAD1F0C086C1F0C08000048C3D9
:10732000908B0020881F0C08B5F90A3007EE903AC0
:10733000F8EEE77A05F1140667EE8A7AF4EEE79A3A
:10734000F1EE10FA53DB434930460CF017FEDFED47
:10735000427AB6EE008AA0EE278A96E80F00BDEECC
:10736000C88A9FED3E0AB8EEC88A04F6487728EE30
:10737000008A87E80F00F0EE680A3948B0EE480A44
:107380000CF0A2FFD4F84C3F07EE903AF8EEE77A03
:1073900028EE0A0AE9EE0A7AFDEEE77A17EE903A4D
:1073A000C4F84C3F1DF01AFFBDEEC00A84EDE90A97
:1073B000D4F83834012B3FF45AAF2A4803F018FCB4
:1073C00018B128480321F6F71BFED4F83834012BF6
:1073D00017D1244803F0A6F9224803F0DFFA214828
:1073E00009B0BDEC088BBDE8F04003F0FBB91949CA
:1073F00030460CF0F3FEF4EEC08AF1EE10FAA2D99A
:10740000D6E795F824302BB9174861F07FF90123AE
:1074100085F824301348F8F739F81248F7F738FFA1
:107420001048F7F71DFD114890F8BC336BB10023ED
:1074300080F8BC3333220221A0F5405009B0BDECE6
:10744000088BBDE8F040FDF70DBB09B0BDEC088B23
:10745000F0BD00BF908B0020A00CB3450AD7233CA1
:10746000A08B0020582C0020484E0020585C0020A3
:1074700010B50446FEF75AFA2046054B40F8143B77
:107480000CF04AFB204603493EF062FE204610BD48
:1074900060200C08F81F0C08032070470048704754
:1074A000C4200C0800487047D0200C08F8B52A4DBD
:1074B00006460027A5F54050A5F8B873F7F74CFF2E
:1074C0007368A5F58052D3F8F811D2F8143C9942AC
:1074D00005F5005421DBC4F84C34736892EDDB7A77
:1074E000D3ED7F6A9FED1D6AF8EEE66A27EE067A15
:1074F000F4EEC76AF1EE10FA18DBBDEEC77A17EEAC
:10750000103A1748C4F85034FDF7FEF820B1D4F80B
:1075100050345B42C4F85034F8BD5B429942DADD26
:10752000012385F8B833C4F84C74D6E702F6184244
:10753000D2ED007A67EE867AF4EEE76AF1EE10FAA1
:1075400093BFFDEEE77A012385F8B93317EE903A41
:1075500088BF0023D5E700BF585C00200000C84268
:10756000582C002070B500212DED028B04463448C4
:10757000344D01F033F832480021F0EE408A01F03A
:1075800037F895F8B833B0EE408AD3B1B0EE680A58
:10759000042054F0EBFD95F8B93393B3B0EE480AEC
:1075A000132054F0E3FD2648002101F02BF820467B
:1075B000FEF7AEFABDEC028B2046BDE87040FEF748
:1075C000B9BA05F50056A5F54050F7F729FAD6F8EF
:1075D0004C34002B0CDCD6F84C34002BDBDA0420C6
:1075E00054F0D8FDB4EEE80AF1EE10FACED4D2E7AA
:1075F000042054F0CFFDB4EEE80AF1EE10FAEADD13
:10760000C4E7114D0E48F7F7ABFAD5F85034002B0C
:107610000CDCD5F85034002BC5DA132054F0BAFD39
:10762000B4EEC80AF1EE10FAB8D4BCE7132054F057
:10763000B1FDB4EEC80AF1EE10FAEADDAEE700BF24
:10764000582C0020585C0020587C002000F5A040F9
:107650000023C0F8FC3EC0F8F83E80F8013F80F8F7
:10766000023F704700F58043D3F8E43D002BCBBFC9
:1076700007EE903A00F50050B8EEE70ADFED037A26
:10768000DCBF90EDD60A20EE270A70470000C84202
:107690002DE9F0412DED028B00F5985784B09FED58
:1076A000C98A1037054603A938468DED038A06F0CE
:1076B00015F8B0B19FEDC47ADDED037A05F5A84366
:1076C00067EE877AD3ED166A9FEDC07AE6EE877A89
:1076D000F4EE487AF1EE10FA48BFF0EE487AC3EDC6
:1076E000167A2846F7F778F805F58044B0EE408A18
:1076F000F0EE000A9FEDB30A1DF0B4FE04F6FC5351
:10770000D3ED007A38EE678A05F50056E0EE087A88
:10771000C3ED007A94F8C83D002B40F09380D4F874
:10772000B42D05F59A4324339A4205D005F59A43C2
:107730002C339A4240F0868008212846F6F71AFF3B
:10774000804630B1D6EDD67A9FEDA17A67EE877A82
:1077500073E002212846F6F70DFF0146002855D0B8
:10776000D6F8043C1B8B2846414608EE103A01F03F
:1077700005F9D6F8040C4369B8EE488AB0EE401A11
:107780002BB3012B28D0DFED937AF0EE671A96ED3C
:10779000D60A9FED8F7AF4EEC17AF1EE10FA20EE60
:1077A000070A4FF0640124DBB6F8542312FB01F200
:1077B000B0EE672A07EE902AF0EE400AB8EEE70A2C
:1077C0001DF0AAFCBDEEC00A10EE103AECE0DFEDB1
:1077D000817AF1EE481ADAE78DED010A53F032F9B9
:1077E00007EE900ADFED7B1A9DED011AF8EEE77ABD
:1077F000CDE7B6F8563313FB01F300EE903AB0EE46
:10780000482AF8EEE00AF0EE671AD9E7B6F95423F1
:10781000B6F956339B1A07EE903A2846B8EEE78A37
:1078200001F0ACF8B6F85433642213FB02F307EE10
:10783000903AF8EEE77AE8EE007AFDEEE77A17EE96
:10784000903AB1E005F5A043D3F83834042B40F06A
:10785000A08005F5BC40103077F0DAFAC4F8E00DEE
:10786000D4F8B40D03689B6B984700285ED094F859
:10787000F43D002B5AD0D4F8B43D05F599455C355C
:10788000AB4253D0D4F8E03D9FED537A07EE903AE7
:10789000D4F8F03DF8EEE77A384627EE878A07EE0F
:1078A000903AF8EEE78A68EE878A06F023F9C8EE88
:1078B000807A04F6F8539DED037A77EE877AB6EE78
:1078C000007AB4EEE78AF1EE10FA4CBF77EEC87A90
:1078D000DFED407A77EE877A93ED007AFDEEE77A76
:1078E000F8EEE77AB4EEE77AF1EE10FA0ADD37EE59
:1078F000676ADFED3A6AB4EE666AF1EE10FA48BFE5
:10790000F0EE477A04F6F853C3ED007AD4F8E03D80
:10791000DFED2F6A07EE103AB8EEC77AA7EEA67A27
:10792000BDEEC77A17EE103AC4F8E03DD4F8B40DB6
:1079300003681B6B984740B1B4F9EC2D002AC2BF15
:10794000D4F8E03D9B18C4F8E03DB6F95623B6F9EB
:107950005413D4F8E00D64235A4359431DF04AFDF3
:10796000C4F8E00D06F54B63D6F8C00C93ED4A8AD7
:1079700006F0C0F8C8EE007A04F6E8549DED037AEC
:1079800077EEC77AC4ED007A04B0BDEC028BBDE897
:10799000F081D4F8B42D05F59A4370339A4206D19C
:1079A000D4F8E43D002B02DDC4F8E03D58E705F5CE
:1079B0009A4348339A427FF4C5AE2846FFF752FEF9
:1079C00000E700BFCDCCCC3DCDCC4C3ECDCC4C3F28
:1079D0000000C842000000000AD7233C9A99993F52
:1079E00030B500F5985587B0103500230446284679
:1079F00003930493059304F041FF002843D003A9A7
:107A0000284605F099FE00283DD004F5B15393EDCA
:107A1000047ADFED216A8DED017AB0EEC77AD3EDFD
:107A2000077AB4EEE67AF1EE10FACDED027A06D5D9
:107A3000F0EEE77AF4EEE67AF1EE10FA2AD401A835
:107A40001FF098FD03A901A81FF0DCFC04F500530A
:107A500093EDD87AB5EEC07AF1EE10FAC4BFDFED3F
:107A60000F7A27EEC00A04F58044C6BFA7EE270AA6
:107A70000123002384F8F43DCABFFDEEC07A002341
:107A800017EE903A04E004F58044002384F8F43DB6
:107A9000C4F8F03D07B030BD000000340000C8421B
:107AA0002DE9F0412DED028B00F5A04607EE901A6E
:107AB000D6F8043F00F5BE45B8EE678A044648355F
:107AC00000F54057BBBB00F58043D3F8B42D00F55B
:107AD0009A4348339A4204D000F59A4370339A424D
:107AE00029D196F8E83333B304F5BE40294638303F
:107AF0000CF074FBD7F8E8050368F0EE408A5B6A87
:107B0000B0EE480A9847F0EE087A60EE277AF4EE75
:107B1000E78AF1EE10FA0EDDBDEC028BD7F8E8052E
:107B20009FED0C0A036804F5BE412A469B6ABDE836
:107B3000F04128311847B0EE480ABDEC028BD7F867
:107B4000E80596F9002F03682946DB6ABDE8F04195
:107B5000184700BF0000000070B504462DED028BF1
:107B600004F5A04579F052FBD5F8703F474AC31A97
:107B70009342064672D907EE903AB8EE670ADFEDF7
:107B8000447A9FED441ADFED440A20EE270A40F2C2
:107B900095101DF08FFBC5F8706F04F50056DFEDF2
:107BA0003F7AD6F8003CB3F9083008EE103A96F95F
:107BB000B233B8EEC88AF0EE408A28EE278A0BB1BD
:107BC000B1EE488A9FED367ADFED367AB4EEC78A99
:107BD000F1EE10FA52DA05F66C73D3ED006AF4EEAA
:107BE000C76AF1EE10FAB4EEE78AACBF01230023B6
:107BF000F1EE10FA3FD905F66C7292ED007AB4EE10
:107C0000E77AF1EE10FA36D82046FAF717FE96F921
:107C1000B33300EE103A06F6D84306F54E66D6EDBD
:107C2000000A93ED001AB8EEC00A40F2A710F1EE78
:107C3000600A20EE080A1DF03DFB28EE800ADFED09
:107C40001A8A20EE280A2046FDEEC07A05F66C75E9
:107C500017EE901AFAF7B0FD85ED008A2046FAF784
:107C6000FDF92046F7F7FCF8BDEC028B2046BDE895
:107C70007040F7F70DBB002BC6D1C8E7B4EEE78A1A
:107C8000F1EE10FAC3D90023B5E700BF9F860100CB
:107C9000BD3786359A99193ECDCCCC3D5304693910
:107CA00000000034000000B40000C84270B5044673
:107CB00000F5A8404FF0FF315C3022F0CBFA431CB6
:107CC000054604F5A04603D1114BC6F8C03370BD7C
:107CD00004F5BE4104F5BE40483128300CF04EF9A1
:107CE0009FED0C7AF6EE007AE0EE077AFDEEE77A89
:107CF00017EE900A281A1DF0A5FA07EE900A9FEDDC
:107D0000067AF8EEE77A67EE877AC6EDF07ADEE774
:107D10000000B442A00CB3450AD7233C00F5405004
:107D2000D0F8E80503689B6B18470000F7B500F52D
:107D300040530546D3F8E80503681B699847074692
:107D40002846FFF7EBFF05F5A0440646D4F8FC0EE5
:107D5000002862D13EB1D4F83C3FC4F8083F3E4B06
:107D6000C4F80C3F0120C4F8F47E1DF06BFAD4F87F
:107D7000FC3E94F9002F00FB0230C4F8FC0E3EB329
:107D80000023019394F8603F002B4AD094F80C3EF6
:107D9000022B46D105F5AA40012201A9743044F016
:107DA000EFFA00283DD0D4F8643FDFED2C6A07EEEF
:107DB000903AB8EEE77ADDED017AE7EE667AB1EE59
:107DC000047AF0EEE77AF4EEC77AF1EE10FA33D4E3
:107DD00094F8013F002B3DD1D4F8FC3ED4F80C2F91
:107DE000002BB8BF5B42934234DBD4F83C1FD4F87D
:107DF000083FC4F8081FCB1A03F2F31340F2E63031
:107E0000834202F5D2328CBF0023012302F5F072C7
:107E100084F8023FC4F80C2F1CE0D4F8F43EF81AA2
:107E2000A1E7D4F8582FD4F83C3F9B1A03F2F31380
:107E300040F2E6329342CBD8012384F8013F00237D
:107E400084F8023FD4F8FC3E03F5D23303F5F07317
:107E5000C4F80C3F03B0F0BDE0A501000AD7233CF5
:107E60002DE9F04100F58048044698F8DD3DA3B3C4
:107E700000F5A045D5F8503F13B9D5F8543F63B38A
:107E800004F5BE4604F5BE47204638364837FAF7B3
:107E9000FDFF394630460CF0A1F904F5BE413A46E3
:107EA0002831304685EDF30A0CF0CEF8DFED0C0AF0
:107EB00085EDF40A7620B7EE001A1DF0FBF904F503
:107EC0003253204683ED7D0AFFF730FFD8F8B40D1A
:107ED0000368BDE8F041DB6A1847BDE8F08100BFE8
:107EE00000000000012938B5044600F5A04512D86D
:107EF00000F5005395F8482FB3F97E3383EAE37118
:107F0000A1EBE37189B2012998BF3C21920730D5DA
:107F1000FF2385F8003F07EE901AF8EE677A05F622
:107F20001473C3ED007A2046FFF7BAFDD5F8043F7D
:107F30002BBB2046FFF7F2FE40B995EDF47AF7EE41
:107F4000007AB4EEE77AF1EE10FA18DD79F06AF90A
:107F500004F58043C5F8040FD3F8B40D03681B6A19
:107F6000984760B104F54F500021BDE838404EF00D
:107F70002DBB002BB4BF4FF0FF330123C9E738BD41
:107F800010B500F5AA44543420465CF01DF8204694
:107F9000BDE810405CF088B810B500F5A043044679
:107FA00093F868359A0716D45B074FF002014CBF6F
:107FB000094A0A4A00F54F504AF024F904F5AA404C
:107FC00054305BF0D5FF04F52E500121BDE8104080
:107FD0002C3062F079BB10BD44210C085E210C08E6
:107FE00070B500F5A046054696F954459CB196F843
:107FF0006835C3F380045B0728D4B6F95A35002BE3
:108000000BDC2846FFF7C8FF05F52E5001212C3068
:1080100062F05AFB0124204670BD2146FAF706F8AB
:10802000B6F95A3507EE903AF8EEE77AB4EEE70A79
:10803000F1EE10FAE5D5D6F8D433002BE1D0044A9E
:10804000042105F54F504AF0DDF8E4E70024E2E7AB
:1080500074210C0808B52DED028B08EE901A30B390
:10806000F2B1B0F9083008EE103AB8EEC88AF8EE6E
:10807000E88A9FED100ADFED100A28EE800ADFED96
:108080000F8A4FF4D470B7EE001A1DF013F9C8EE42
:10809000280A1DF06BF820EE280ABDEC028B08BD03
:1080A00052F054FD07EE900AB8EEE78ADFE79FED45
:1080B000020AF2E70AD7233C0000000000A08C452A
:1080C00037B500F50054054694F9DF33002B52D044
:1080D00052F056FC52F04AFCC4F8FC0B52F050FC33
:1080E00052F030FCC4F8000C52F04AFC52F034FC60
:1080F000C4F8040C52F044FC52F038FC41F29411E4
:10810000C4F8080CD4F8FC0B52F084FCD4F8000C32
:1081100041F2941152F07EFCD4F8080C41F2941113
:1081200052F078FC284600F023FC48BBD4F8040C3D
:10813000642152F06BFC52F023FCD02153F0C8FCB8
:10814000C4F80C0C52F01CFCD22153F0C1FCC4F852
:10815000100C05F51E5004304921019054F046FAE8
:1081600001984A2154F042FA0198462103B0BDE833
:10817000304054F03BBA52F003FC52F0D9FBABE76D
:1081800005F5C043D4F8040C93F8EC30642173B1C6
:1081900052F03CFC6421462054F020F9642149202F
:1081A00054F01CF964214A2054F018F9C3E752F046
:1081B00031FCEFE710B500F500541E21D4F8FC0B9C
:1081C00052F02CFCD4F8000C1E2152F027FCD4F8FD
:1081D000080C1E2152F022FCD4F8040C1E21BDE82C
:1081E000104052F01BBC000007B500F0C1FB014677
:1081F00058B90190462054F013F80199492054F0E1
:108200000FF801994A2054F00BF80021042054F093
:10821000D9FA0021132054F0D5FA0021462054F059
:10822000D1FA0021492054F0CDFA00214A2054F01F
:10823000C9FA0021152003B05DF804EB54F0C2BA6E
:1082400010B5044654F004FD54F054F9204601F0F2
:10825000C9FCBDE8104054F003BC000038B500F57F
:108260000055044695F9DF330BB1002038BD0121DC
:10827000F6F780F990B104F58043D3F8B42D04F5F6
:108280009B4304339A4209D004F5994364339A42DC
:1082900004D004F5994374339A42E6D12046F6F7A8
:1082A00049FB0028E1D0D5F8083CB3F90800DDE728
:1082B00038B52DED028B00F5804393F8C83D002BB7
:1082C00040F0B7805C4A00F59B43D2F8B42D0433EC
:1082D0009A4200F54F5508D0584A0321BDEC028B55
:1082E0002846BDE8384049F08DBF00F500549FEDA9
:1082F000546AD4F8FC2BB2F90830002BB8BF5B42AB
:108300009BB207EE903A138B06EE903AF8EEE66ACF
:10831000F8EEE77A66EE866AF4EEE67AF1EE10FAA7
:1083200017DCD4F8002CB2F90830002BB8BF5B4240
:108330009BB207EE903A138B07EE103AB8EEC77A6D
:10834000F8EEE77A27EE067AF4EEC77AF1EE10FA45
:1083500001DD3C4AC1E700F5B15004301FF02CFEAE
:10836000DFED397A20EE270AF3EE0E7AB4EEE70A53
:10837000F1EE10FA01DD354AAFE7042054F0DAF9E6
:10838000132054F0D7F9152054F0D4F94D2054F0AF
:10839000D1F94E2054F0CEF94F2054F0CBF95020B3
:1083A00054F0C8F9152053F0F5FE9FED298AB0EE80
:1083B000C00AB4EEC80AF1EE10FA0BD5102054F042
:1083C000B9F9562054F0B6F9112054F0B3F95720FA
:1083D00054F0B0F9032053F0EDFEB0EEC00AB4EE55
:1083E000C80AF1EE10FA0FD5022053F0E3FEB0EE0A
:1083F000C00AB4EEC80AF1EE10FA05D5182054F000
:1084000099F9192054F096F9D4F8FC0B811D0C3021
:108410003EF05CFDD4F8000C811D0C303EF056FDA2
:10842000D4F8080C811D0C303EF050FD094A05219E
:1084300054E7BDEC028B38BD586C002088210C0835
:10844000CDCC4C3EA8210C08E02E6542D0210C0872
:1084500000000034EC210C0810B500F5005494F92C
:10846000B6339BB1D4F8040C52F0E6FAD4F8042CDD
:10847000B4F9B83330B1B2F906009842ACBF00206D
:10848000012010BDB2F906008342F7E70120F8E7AA
:1084900010B50446FFF7E0FF60B104F5804478F0C2
:1084A000C1FED4F8D43DC01AB0F57A7F94BF002045
:1084B000012010BD0120FCE770B50546FFF7E8FF7D
:1084C00005F5005408B3D4F8FC3B9A89DA80D4F857
:1084D000003C9A89DA80D4F8083C9A89DA80D4F88A
:1084E000FC3B00261E81D4F8003C1E81D4F8083CD9
:1084F0001E8105F58043D3F8B40DC3F8EC6D036815
:108500005B689847D4F8043C1E8105F5C0404430B0
:1085100070F0D6FE78B3002652F032FA437A13B9DF
:1085200052F02EFA837A94F9B623012A22D106B1A9
:1085300003B32846FFF7ACFF05F5804494F8CE3D21
:1085400030B30133DBB20A2B84F8CE3D0BD11F4B85
:108550001F4A042105F54F5049F054FE1D4A0123DE
:1085600084F8C83D937294F8CE3D0A2B02D90A23B1
:1085700084F8CE3D70BD2846FCF70AFE0028CAD11B
:1085800052F0FEF952F0C0F9061E18BF0126C3E7EB
:10859000002BEFD0013BDBB2032B88BF032384F811
:1085A000CE3D94F8CE3D012B08D105F54F500A4B36
:1085B000074ABDE87040042149F024BE002BD9D100
:1085C000044A84F8C83D9372D4E700BF83AC0D0819
:1085D000FC210C08058E0020DF230C0800F500505C
:1085E0000A4690F9E61BD0F8FC0BFFF733BD0000FC
:1085F00000F500500A4690F9E71BD0F8000CFFF791
:1086000029BD000000F500500A4690F9E81BD0F89B
:10861000080CFFF71FBD000010B54FF48061044641
:10862000F5F7A8FF04F5005328B1BDE81040D3F8D2
:10863000040C52F087BBBDE81040D3F8040C52F094
:108640008BBB00002DE9F04100F500530546D3F83F
:10865000083CB3F9088000F5C044B8F1000F02D11E
:10866000012384F8883005F5C0474437384670F058
:1086700027FE0646F8B9B8F57A6F2EDD78F0D2FD00
:10868000D4F88430804693B1C31A40F6B73293428F
:108690000FD905F5A045012231463846F5F752F9C4
:1086A000C4F8846084F88860C5F87C8301E0C4F86D
:1086B0008400BDE8F08118F57A6F0EDA78F0B2FD2B
:1086C000D4F884306BB1C01A40F6B7339842F0D971
:1086D000012200213846F5F75BF90023C4F8843005
:1086E000E7E7C4F88400E4E770B52DED028B04469B
:1086F00052F046F951F0FEFF30B9BDEC028B204636
:10870000BDE87040FFF7D8BE04F5804595F8C83D38
:108710001BB978F087FDC5F8D80D2046FFF79CFE01
:1087200018B178F07FFDC5F8D40D2046FFF7C4FEE0
:108730002046FCF7BDFB04F500560023C5F8EC3DD0
:1087400096F9BA3363B3D6F8043CB3F90830322B48
:1087500026DD28B3323B1BB207EE903A04F5985061
:10876000B8EEE78ADFED207A103028EE278A03F092
:10877000BFFF38B3B6F9563396EDD67A07EE903A86
:10878000F8EEE77A77EEC77A27EE888ADFED177A78
:1087900028EE278ABDEEC88A18EE103AA5F8EC3DFF
:1087A0002046FFF74FFFD5F8B40D03685B68984784
:1087B000BDEC028B014604F5C1401030BDE87040AD
:1087C00054F03ABE96F9493396F94B239B1A07EEBB
:1087D000903AF8EEE77A27EE888ABDEEC88A18EE5E
:1087E000103AA5F8EE3DDBE70AD7A33C0000C842EB
:1087F00070B500F500540546D4F8BC330BB9002021
:1088000041E094F94833002BF9DA00F58043D3F8BE
:10881000B40D03685B6898470138172832D801A364
:1088200053F820F0218901085D8901088588010835
:108830005389010849890108358901082B890108F4
:108840008588010885880108898801081789010839
:108850000D890108FF8701083F8901083F89010848
:1088600085880108858801088588010885880108B0
:1088700085880108858801088588010885880108A0
:1088800067890108012070BD05F5A045B5F89A6417
:10889000162EB4D0D4F8BC1311F0020301F001027B
:1088A00005D0A6F1150CDCF1000343EB0C0311F02D
:1088B000040043EA020303D0A6F11F0460426041B2
:1088C00043EA000211F0080007D01F2E1AD0A6F1CB
:1088D000110002288CBF0020012011F0100340EA93
:1088E000020005D0102E0FD0A6F152025342534180
:1088F000034311F4006014BF95F86414014643EA81
:108900000100C0E70120E8E70123F1E7D4F8BC0348
:10891000C0F34010B7E7D4F8BC03C0F38010B2E74F
:10892000D4F8BC03C0F3C010ADE7D4F8BC03C0F367
:108930000020A8E7D4F8BC03C0F34020A3E7D4F894
:10894000BC03C0F380209EE7D4F8BC03C0F3003022
:1089500099E7D4F8BC03C0F3403094E7D4F8BC03E3
:10896000C0F380308FE7D4F8BC03C0F3C0308AE78F
:1089700000F5005090F84803C009704738B5044628
:108980000D4651F0FDFF0368DB689847C8B104F558
:108990000053D3F8040C6DB152F0D8F807EE900AEA
:1089A000B8EEE70A04F5C04494F8EB300BB1B1EE31
:1089B000400A38BDB0F9083000EE103AB8EEC00AEF
:1089C000F0E79FED010AF4E70000000038B52DED57
:1089D000028B04460D4651F0D3FF0368DB689847CD
:1089E00000283FD0214BD3F8043C5B69012B07D012
:1089F000BDEC028B29462046BDE83840FFF7BEBFDC
:108A00004FF480612046F5F7B5FD0028F0D004F55D
:108A10000053DFED177AD3F8040C93F94B33028B34
:108A200008EE903A00EE102AF8EEE88AB8EEC08A16
:108A300068EEA78A52F094F8B6EE001AA0EE011A7A
:108A400004F5C044DFED0B0AB0EE680A1CF060FCD0
:108A500094F8EB3028EE000A0BB1B1EE400ABDEC01
:108A6000028B38BD9FED030AF9E700BF584C002088
:108A70000AD7233C0000000073B500F5A04504466A
:108A800095F80C3E022B00F5546612D100F5AA4071
:108A9000012201A9743043F073FC50B1019BC6F868
:108AA0009C3230463EF012FE2046FAF74FF802B0F4
:108AB00070BDD5F83834042B05D12046F9F71EFDDA
:108AC0008DED010AEAE705F674752B680193E5E779
:108AD00070B500F580460446D6F8B40D03689B6B6C
:108AE0000D46984748B9D4ED460A9FED1C0A64210B
:108AF0002846BDE8704053F02FBCD6F8B40D04F5FD
:108B00009A4104F500524831884292F84A3392F96A
:108B100014241FD104F5A04191F8E40350B94AB1DF
:108B2000D3B204F5A041D1F838140139012998BF16
:108B3000D3B207E091F98C0E60B1D1F83814042952
:108B400008D1C3B207EE903AD4ED460AB8EE670AF0
:108B50006421CDE7002AF5D0E3E700BF0000000064
:108B60002DE9F04100F58048044604F59B43D8F810
:108B7000B40D0433984203D100252846BDE8F081A6
:108B800003689B6B984750B104F5A04393F8685570
:108B900015F0010503D0012283F83024EDE704F538
:108BA000BC40103076F068FA054608B10125E4E7CC
:108BB00004F5A04696F83034002BDDD0D8F8B40D7B
:108BC00003689B6B984718B9002386F83034D4E7C4
:108BD00094F8143494F85874B02202FB034393F8C9
:108BE000F121B7BB012A0AD993ED837AF1EE047A19
:108BF000B4EEE77AF1EE10FAACBF01270027D8F8FF
:108C0000B42D04F59A4348339A4202D196F8E433DE
:108C100023B104F59B430C339A4240D104F5005331
:108C2000204693F90884FCF7B3FAA0B9204601F076
:108C300007FC0028BAD0002386F8303494F8712459
:108C400004F58C63242101FB0233DB6AC6F8DC33B4
:108C500093E72F46D3E778F0E5FAD6F844344FF49B
:108C6000FA62C01A642313FB082341F2883293424C
:108C700038BF13469842D9D92046F9F7C5FBB0F55D
:108C8000FA7FD3DD04F5805341F26E72D3F80C35D0
:108C900003F6B7339342C9D8002FC7D094E706F63E
:108CA0007473D3ED007AB2EE047AF0EEE77AF4EE64
:108CB000C77AF1EE10FA87DA002F3FF477AF04F5A8
:108CC0009850103003F014FD00283FF47DAF04F5F8
:108CD0000053184693F88611383002F029FFF1EE60
:108CE000047AB4EEE70AF1EE10FAFFF65FAF6BE735
:108CF000F8B52DED048B0446084616461D46BDF911
:108D0000287053F047FA04F500543046B0EE408A1C
:108D100053F040FAB4F9E423002AF0EE408A37DA3F
:108D2000C2F1640307EE903A9FED207AF8EEE77AFD
:108D300067EE877A60EE278AD4EDF87A9FED1C1AE9
:108D4000DFED1C0A38EEC80ABC2020EE270A1CF012
:108D5000B1FA38EE288AB0EE409A94EDF80A9FED09
:108D6000141ADFED140A28EE000ABD201CF0A2FA46
:108D70002846B0EE408AB0EE490A53F0F7F9B0EE5B
:108D8000480ABDEC048B3846BDE8F84053F0EEB914
:108D9000D2D002F1640307EE903A9FED047AF8EE28
:108DA000E77A67EE877A28EE278AC5E70AD7233C59
:108DB00000A08C4500A08CC500B52DED048B0420CF
:108DC00083B053F0E7F90320B0EE408A53F0F2F994
:108DD000DFED189A9FED181ADFED180A8DED011AD4
:108DE000F0EE408AB0EE480AA8EEA90ACF20CDEDF9
:108DF000000A1CF05FFAB0EE409AB0EE480A9DED12
:108E0000011ADDED000AA8EEE90AD0201CF052FAA2
:108E10001820B0EE408AB0EE490A53F0A7F9B0EE40
:108E2000480A192003B0BDEC048B5DF804EB53F045
:108E30009DB900BF0000344200A08C4500A08CC545
:108E4000F8B52DED088B00F5005600F5C04596F9F4
:108E5000CE3B13F0040F03F0010203F0020440F0D4
:108E6000F580D5F8F0707B1E5F425F41002A00F06C
:108E7000EF804D2053F08EF94E20F0EE409A53F0E3
:108E800089F9B0EE408AB6F9E633DFED87AA0AEE3B
:108E9000103A1520B8EECAAA53F07CF92AEE2AAA95
:108EA00020EE0AAA002C00F0DB80F0EE488AB0EE3B
:108EB000699AB5EEC0AAF1EE10FA40F3D6809FEDA4
:108EC0007B1ADFED7B0A38EE0A0A4FF480701CF043
:108ED000F1F99FED761ADFED760AB0EE408A40F2A6
:108EE000011038EECA0A1CF0E5F9F0EE408A96F956
:108EF000CF3B632B15DC07EE903A9FED6E7AF8EED0
:108F0000E77AB4EEC79A67EEAA7AF1EE10FAF4EEB9
:108F1000C78A98BF29EE279AF1EE10FA98BF68EE3B
:108F2000A78AD5F8F03096F9CC4B96F9CD6B022B89
:108F300000F0B48024B2002C01DC002E6EDD032092
:108F400053F038F9DFED5C7AB4EEE70AF1EE10FA8F
:108F5000B0EE40AA62DB002F00F0A2809FED571A0E
:108F6000DFED570A40F2271030EE000A1CF0A2F99C
:108F70009FED541ADFED520AB0EE40BA4FF49470F0
:108F80003AEE410A1CF096F970EE007AB0EE4BAA68
:108F900007EE104AF8EEC7AA9FED4BBA9FED431AB1
:108FA000DFED430A6AEEA7AAB0EE690A40F22B1081
:108FB000AAEE8B0A1CF07EF907EE906AF0EE409A5A
:108FC000B8EEE70A9FED391ADFED390A2AEE40AA1A
:108FD000B0EE490A4FF49670AAEE0B0A1CF06AF93B
:108FE000B0EE409AB0EE480A9FED301ADFED300A3D
:108FF00040F22D10AAEE8B0A1CF05CF9B0EE408A0C
:10900000B0EE680AAAEE0B0A4FF497709FED271A8C
:10901000DFED270A1CF04EF9F0EE408AB0EE690A47
:10902000102053F0A3F8B0EE490A562053F09EF8F2
:10903000B0EE480A112053F099F8B0EE680ABDEC82
:10904000088B5720BDE8F84053F090B801270DE792
:10905000042053F09FF8B0EE408AF1EE409A12E7F8
:10906000DFED178AB0EE689A23E79FED101ADFED67
:10907000100A39EECA0A4FF482701CF01BF99FEDFA
:109080000B1ADFED0B0AF0EE409A40F2051039EEB4
:109090000A0A1CF00FF9B0EE409A28E700244CE7CA
:1090A000F0EE407A74E700BF0AD7233C00A08C455D
:1090B00000A08CC5000000B4000000340000C842CD
:1090C00000000000000048426666E63E38B52DED1F
:1090D000028B00F500550446D5F8100CA0B304F53A
:1090E000804393F8C82D7ABB93F8CE3D63BB51F013
:1090F000F3FD07EE900AB8EE678A462095F94853CB
:1091000053F048F8002DF0EE408A20DA04F5BC4018
:10911000103075F033FEE8B99FED101ADFED100A3C
:1091200040F25110B1EE680A1CF0C4F8B4EE408A67
:10913000F1EE10FAC8BFB0EE480ABDEC028B6E200B
:10914000BDE8384053F012B89FED058AD5E79FED92
:10915000040AEBE79FED010AE8E700BF0000C84200
:109160000000000010B52DED028B4369002B4AD0A2
:10917000037C0BB101330374037C002B41D0182B0B
:109180001FD803EB4303C3EB03139B001CB2002364
:1091900007EE903AB8EEE78A0420B0EE480A52F0A3
:1091A000E5FF07EE904A1320B8EEE70A52F0DEFF23
:1091B000B0EE480ABDEC028B1520BDE8104052F01D
:1091C000D5BF4A2B02D8C3F13203DAE7632B01D8AB
:1091D000643BD6E77C2B08D8643B03EB4303C3EB2B
:1091E00003139B001BB20024D2E7AE2B02D8C3F1BD
:1091F0009603F2E7C72B01D8C83BEEE700230374C0
:10920000F1E71C46C4E7BDEC028B10BD10B59FED25
:109210001C7AD0ED017AF4EEC77A0023F1EE10FA51
:10922000044643722BDB90ED007AB4EEE77AF1EE60
:1092300010FA24D908F0B4F8217A07F005FDD4ED2E
:10924000010AF5EE007A60EEA77AB4EEE70AF1EED5
:1092500010FA14D494ED001A40F2A5101CF02AF86C
:10926000F7EE007AB4EEE70AF1EE10FA07D494EDC7
:10927000007AC7EE007A01236372C4ED037A10BD51
:1092800000000034437A7BB391F9003090ED037A0B
:1092900007EE903AF8EEE77A67EE877A9FED137A59
:1092A000F4EEC77AF1EE10FAD8BFF0EE477AFDEE91
:1092B000E77A17EE903A0B7092F9003090ED037A4E
:1092C00007EE903AF8EEE77A67EE877A9FED087A34
:1092D000F4EEC77AF1EE10FA58BFF0EE477AFDEEE1
:1092E000E77A17EE903A1370704700BF0000C8C2CB
:1092F0000000C842437AF0EE407A5BB190ED030A79
:109300009FED051ADFED050A27EE800A4FF4E6709F
:109310001BF0D0BF704700BF0000C8420000C8C2A9
:10932000F8B504460E46174677F07CFF054604F56F
:109330009C4007F013FE04F5A044D8B3462052F039
:1093400029FFDFED3E7AB4EEE70AF1EE10FA10DB0A
:1093500097F9002094F93134193A934209DAD4F894
:109360003424AA4205D0C4F83454013384F831348B
:1093700044E0462052F00EFFDFED317AB4EEE70A0A
:10938000F1EE10FA3AD896F90020002A36DAC2F146
:10939000FF2294F9323402F57F02E73293422DDA4C
:1093A000D4F83424AA4229D0C4F83454013384F8C0
:1093B000323423E0D4F83434EB1AB3F57A7F1DD37A
:1093C000462052F0E7FE94F9313407EE903AF8EE79
:1093D000E77AB4EEE70AF1EE10FA01DD002B22DCA9
:1093E000462052F0D7FE94F9323407EE903AF8EE68
:1093F000E77AB4EEE70AF1EE10FA18D497F9000014
:1094000094F931240021821A1CF004F8387096F97E
:109410000000002806DA94F93214002201441BF0FF
:10942000F9FF3070F8BDC4F83454013B9EE7002BBF
:10943000E4DDC4F83454013BB9E700BF0000003458
:10944000000000B410B52DED028B00F5005282B083
:1094500092F9483392F849238DF80630002B0446E0
:10946000B0EE408A8DF8072004DAFFF7C1F908B999
:109470008DF8060004F5A043D3F83824012A4CD017
:10948000072A4AD004F5BC40103075F077FC00285C
:1094900054D104F52F500DF106010DF107021030E3
:1094A000FFF7F0FE2046FFF73BFF9DF906309DF9E0
:1094B0000720DFED238A9342A8BF134607EE903AB8
:1094C00004F53254B8EEE70A303420EE280A20467C
:1094D0008DF8063074F04AFE9DF9073000EE103A20
:1094E000B8EEC00A204620EE280A74F049FE9DF925
:1094F000073001EE103A9DF9063000EE903AB8EED2
:10950000C11AF8EEE00A40F24D20B0EE480A1BF016
:10951000D1FE02B0BDEC028B10BDD3EDE57AFDEEBD
:10952000E77A17EE902AD3EDE67A8DF80720FDEE64
:10953000E77A17EE903A8DF80630AAE70023FAE7AB
:109540000AD7233C70B5044600F52F55103504F5B5
:1095500080462846FFF75AFED6F8B40D03685B6DC7
:10956000984740B1462052F015FE2846FFF7C2FE4C
:10957000462052F0FBFDD6F8B40D03681B6D9847EA
:1095800040B1462052F006FE2046FFF75BFF462022
:1095900052F0ECFD2046FFF7E3FA10B304F5005556
:1095A00095F9B43343B101212046FFF7E7F9BDE84F
:1095B0007040462052F0DABD04F5BC441034204619
:1095C00075F0DCFB50B1204675F060FD30B195F9C7
:1095D000483300EE103AB8EEC00AE8E79FED010A02
:1095E000E5E770BD0000000010B504462DED028BCC
:1095F000462052F0CFFD2046B0EE408AFBF7C8FD72
:1096000080BB04F5C04044306FF05AFE50B304F5FF
:10961000AB53D3ED028A1BF015F990F813339FED8D
:10962000137A0C2202FB0300D0ED627AE8EEC77ACF
:10963000F4EEC77AF1EE10FA0CDC04F5005494F95C
:109640004B3307EE903AF8EEE77AF4EEC87AF1EE93
:1096500010FA07D5BDEC028B0548BDE8104001218A
:1096600004F0CCBCBDEC028B10BD00BF0AE81C416D
:10967000683F00202DE9F04100F500550646D5F879
:109680000C3CA3BB002706F58048D8F8B40D03684E
:109690009B6B98470446002852D006F5985010302E
:1096A00003F026F880B308F55E63D3ED007A9FEDF2
:1096B0003F7AF8EEE77A67EE877AFDEEE77A17EE03
:1096C000903A1BB295F9FB230AB19A421FDA95F939
:1096D000F943FCB906F5A042D2F83834013B062B19
:1096E0002ED8DFE803F01E2D24602D2D1E0051F032
:1096F00047F90368DB6898470028C3D0D5F80C0CFD
:1097000051F0EAFA47B2BEE795F94B33DAE795F93B
:10971000FA43DFE724B29C42ACBF95F9F84300243A
:10972000D8E795F9FC33002B18BF1C4608E095F9E3
:10973000FC332BB13046FBF74BFD08B195F9FC43E8
:1097400087EAE773A3EBE773DBB2A342C8BF3C46EB
:1097500007EE904A0320B8EEE70A52F007FD07EE45
:10976000907A0220B8EEE70A52F000FD95F92D3408
:10977000D6ED460A00EE103A6421B8EEC00A032086
:1097800052F0EAFD95F92D34D6ED460A00EE103A76
:109790000220B8EEC00A642152F0DEFD3046BDE87A
:1097A000F041FFF709BB92F98B3EBCE70AD7233C97
:1097B00038B504462DED048B462052F0EBFC584B97
:1097C000DFED587A93F9993B08EE903AF8EEE88A83
:1097D000152068EEA78AB0EE408A52F0DBFC9FEDC0
:1097E000527A20EE280A04F5C045C0EE077A04F547
:1097F000BD401C30C5ED387A72F01CFB10B100235F
:10980000C5F8E030B5EEC08AF1EE10FA43D5204637
:10981000FFF7AEF800287ED02046FEF7E9FF0028CB
:1098200079D0D5ED387A9FED419A9FED411ADFED61
:10983000410AB0EE480AA7EE890A4FF43B701BF0CC
:1098400039FDD5ED387A9FED3A1ADFED3A0AF0EEA0
:10985000408A40F2ED20B0EE480AA7EEC90A1BF09C
:1098600029FDB0EE408A04F5C045443528466FF026
:1098700031FDD0BB284670F02BFE022827D10321F2
:10988000492052F0CDFFBDEC048B0321BDE83840E8
:109890004A2052F0C5BF3ED9D5ED387A9FED239AC4
:1098A0009FED251ADFED220AB0EE480AA7EE890ADD
:1098B00040F2F2201BF0FEFCD5ED387A9FED1E1A27
:1098C000DFED1B0AF0EE408A40F2F320C3E79FED84
:1098D000180A492052F04AFCBDEC048B9FED140A93
:1098E000BDE838404A2052F041BCB0EE680A492039
:1098F00052F03CFCB0EE480A4A2052F037FC2046B9
:109900004921FFF7E5F8BDEC048B20464A21BDE86C
:109910003840FFF7DDB89FED068AF0EE488AA2E7EF
:10992000584C00200AD7233C00A08C450000484238
:10993000000000000000C8C20000C842F8B52DEDCC
:10994000028B00F5A046044696F9893E002B32DDD5
:1099500000F5804200F59A43D2F8B42D48339A427C
:1099600029D196F9883E002B25DD00F5BC4010304A
:1099700075F076FAF8B104F5C04044306FF0A0FC01
:10998000C8B9124F9FED128A04463D682D190ED0BA
:10999000B5F9080052F010FA48B196F9893E012B4A
:1099A0000CD1B5F90800B0EE480A52F0DFFB1434D0
:1099B000B4F5A07FE9D1BDEC028BF8BD022BF6D146
:1099C000B5F90800032152F02BFFF0E7A092002028
:1099D0000000000037B500F5A043044693F890332B
:1099E0000BB39FED120A15204F2552F0BFFB204606
:1099F0000095502313221521FFF77AF9152052F014
:109A000057FE80B9284652F053FE60B99FED070A11
:109A10004E2052F0ABFB9FED050A4D2003B0BDE890
:109A2000304052F0A3BB03B030BD00BF00000000C7
:109A300070470000F8B52DED048B00F58044054615
:109A4000D4F8B40D03689B6B984738B9D4F8B42D9B
:109A500005F59A431C339A4240F0BE8005F5C0409C
:109A600044306FF037FC002800F0B6802846FBF742
:109A70008FFB002800F0B08005F5A046D6F84C34E6
:109A8000002BB8BF5B42B3F52F7F00F3A580D6F85B
:109A90005034002BB8BF5B42B3F52F7F00F39C809E
:109AA00077F0C0FBD6F8B03FC31AB3F5FA7F07468C
:109AB000C0F0928005F5B85393ED057AF2EE007A86
:109AC000B4EEE77AF1EE10FA00F1868006F58B63CA
:109AD00093ED007AB4EEE77AF1EE10FA7CD405F556
:109AE000405393ED1B8AD3ED728A05F51E5404345E
:109AF000B0EE480A0421204652F0AEFBB0EE680AF0
:109B00001321204652F0A8FB78EEC89A4D21B0EE02
:109B1000690A204652F0A0FB38EE289A4E21B0EE9A
:109B2000490A204652F098FBB0EE680A4F212046C1
:109B300052F092FBB0EE680A5021204652F08CFBA6
:109B400005F50055B0EE480A1821204652F084FB76
:109B5000B0EE480A1921204652F07EFB95F9CE3B23
:109B600003F00202DB075CBFF1EE489AB0EE489AC0
:109B70006AB3B0EE498AF0EE698AB0EE690A102144
:109B8000204652F069FBB0EE680A5621204652F09A
:109B900063FBB0EE490A1121204652F05DFBB0EEA6
:109BA000480A5721204652F057FBD6F8B43FC6F872
:109BB000B07FFB1A42F2107293420DD9C6F8B47FFF
:109BC000BDEC048B2046BDE8F84052F02BBF9FED62
:109BD000048AF0EE488AD0E7BDEC048BF8BD00BFE4
:109BE0000000000073B5044653F032F8054652F009
:109BF000C5FF2046FFF7DCFD4E23009313224D23C3
:109C000004212046FFF774F84F23152113220093F7
:109C100020465023FFF76CF82046FFF711F9204645
:109C2000FFF78CFE4FF400512046F4F7A3FC10B16F
:109C30002046FFF7CFFE04F50056D6F89C0B50B136
:109C400004F5804204F59B43D2F8B42D04339A42C4
:109C500001D152F065FA52F027FF52F07BF9284605
:109C600052F094FF96F9703B2BB1204602B0BDE84C
:109C70007040FFF7DFBE02B070BD000073B5044650
:109C800004F5BD4552F0E4FF1C3552F077FF28463D
:109C900072F0D0F804F5A046002866D1D6F8383422
:109CA000042B04D104F5BC40103075F093F8204625
:109CB000FFF748FC04F5804204F59B43D2F8B42D2D
:109CC000043304F5C0459A4205F1440523D02846E3
:109CD0006FF000FBF8B99FED310A462052F046FACA
:109CE0009FED2E0A492052F041FA9FED2C0A4A209E
:109CF00052F03CFA284670F0EBFB02280BD103210E
:109D0000462052F08DFD0321492052F089FD0321A8
:109D10004A2052F085FD2046FFF766FC2046FFF7FB
:109D2000A9FC2046FFF7D2F920464621FEF7D0FED7
:109D300028466FF0C5FA90B90190284670F0C8FB2C
:109D400068B102281AD10199462052F0D5FC019938
:109D5000492052F0D1FC01994A2052F0CDFC204616
:109D600002B0BDE87040FFF73DBF2846F8F790F815
:109D700096F9A63E2B2B91D002B070BD9FED070A3D
:109D8000462052F0F3F99FED050A492052F0EEF912
:109D90009FED020A4A2052F0E9F9E0E700000000D6
:109DA000F6F780BE0148FAF7A3BF00BF582C002089
:109DB00008B5044A0F2343F0B1F980F00100C0B2A6
:109DC00008BD00BF0C230C08F8B500F54057044649
:109DD000D7F8785577F026FA04F5804304F5005655
:109DE000B3F9CC1D8A1E92B2012A73D904F5A042A0
:109DF000D2F83824042A6DD0012993F8C81DD3F86D
:109E0000D42D08BFD3F8D02DB1B1821A07EE902A15
:109E100096EDF27ADFED416AF8EE677A27EE267A60
:109E2000F4EEC77AF1EE10FA06DD03220221204695
:109E3000BDE8F840FAF716BE96F9CC23032A1BD1E9
:109E4000D3F8B43D04F59A424832934265D1002DCF
:109E500063D0401B07EE900ADFED306AB8EE677AF8
:109E6000D6EDF27A67EEA67AB4EEE77AF1EE10FA62
:109E700053DD05220321DAE7012A4CD0022A4CD116
:109E80008DB1431B07EE103AD6EDF27ADFED236A6F
:109E9000B8EE477A67EEA67AB4EEE77AF1EE10FAFA
:109EA000E7DC022A39D197F85C34B3B3D7F86034D1
:109EB0009BB31B4B1B6883B3C01A07EE900A96ED49
:109EC000F27ADFED166AF8EE677A27EE267AF4EE7C
:109ED000C77ACBE796F9C023D6EDF27A032A18BFEA
:109EE000D6EDF17A03290FD1FCEEE77A4FF47A73BD
:109EF00017EE902A401B5A4390420ED2052120466D
:109F0000BDE8F840FAF768BE022906D193F8C83DCB
:109F10001BB90321F3E7002DB3D1F8BD00007A444B
:109F20001492002070B500F50056044696F9C0332F
:109F3000032B00F580450FD0B5F9CC3D63B900F592
:109F4000A043D3F83834042B17D095F8C83DA3B1FB
:109F500003220121FAF706FDB5F9CC3D012B0CD106
:109F600095F8C83D1BB196F9C033032B05D12046A7
:109F70000321BDE87040FAF703BE70BD70B500F66E
:109F8000C806044630461AF027FC034604F54F5035
:109F90005BB3174A04F598550121103548F032F9A2
:109FA000284602F04BFA04F58053032283F8242557
:109FB00040F20112A3F81826B4F9A4301BB9B4F882
:109FC000A230A4F8A430B4F8A41030461AF0A8FCCB
:109FD000284602F033FB8023C4F8743404F58C6007
:109FE0000121BDE8704006F0DFB9024AD2E700BFA8
:109FF00014220C0841220C0838B50B6805465B6832
:10A0000008460C469847074BD87023682046DB6803
:10A010009847014605F595501C30BDE8384038F0AA
:10A020005BBB00BF058E00202DE9F74F00F5804790
:10A030000446D7F8B43D8B420D4616460CD100F5C8
:10A04000005494F80833934240F0B3804FF0010974
:10A05000484603B0BDE8F08F0B6808465B69984737
:10A0600004F54F588146B0B143F00CFA40F20312A8
:10A070004FF4801143F0BEF9524A0621404648F0A1
:10A08000C1F81A2E1FBF504A137843F0040313700F
:10A090004FF00009DCE74D4B1B68DB6A93F89C30FE
:10A0A0005BB304F5005393F8F02132B3B3F80C22FC
:10A0B000D20722D593F82C32FBB12046FAF7C8FE1E
:10A0C000D8B1A6F12703DBB20A2B06D8012202FA87
:10A0D00003F340F2234213420FD12B6828469B68BA
:10A0E00098473B4A03460521404648F08BF8364ADC
:10A0F000137843F004031370AAE7022E2BD0D7F88D
:10A10000B4BDD7F8B83DC7F8B45D04F50059C7F839
:10A11000B8BD04F5C04A99F80823009328469AF878
:10A12000F8308AF8F82089F808630193FBF71CFCE3
:10A1300038BB284A0421404648F064F8009BC7F821
:10A14000B83DC7F8B4BD9AF8F83089F80833019BD8
:10A150008AF8F83095E72B6828465B6898470146EF
:10A160002046FFF725FE81460028C8D12B682846E7
:10A170009B689847184A03460521404648F042F834
:10A1800066E75846FBF7DCFBD7F8B40D03685B685D
:10A19000984799F80823014604F57F6044F04CF98C
:10A1A000D7F8B41D2046FFF727FF002140464FF0A7
:10A1B00011FD1A2E1FBF044A137843F002031370D7
:10A1C00044E700BF5C220C08248E0020542C0020A1
:10A1D00074220C08E0220C08A0220C0873B5054676
:10A1E0000A4801920E46FAF7A7F9019A044630B1DF
:10A1F0000146284602B0BDE87040FFF715BF28466B
:10A20000314642F0D1FE204602B070BD582C0020ED
:10A21000FFF7E4BF4FF40023F7B50446C0F8E03B76
:10A2200000F53C50343071F075F804F542500C30B4
:10A2300070F0ECFD50F0A4FB9922292151F08AFC2A
:10A2400050F09EFB50F044FB04F59450083059F058
:10A250002BFC04F595501C3038F022FA04F58043AD
:10A260002046D3F8B41DFFF7C7FE2046FDF7BCFF1C
:10A2700004F58C6006F0E0FA4FF480431921C4F82D
:10A28000EC3F04F554603DF0F3FC04F59C4006F00F
:10A2900021FC04F5895053F0FDFD04F5315004F51F
:10A2A0004F57083053F078FA38464CF0F3F904F57C
:10A2B0005B5060F055FF0AF0B9FD4FF48063036313
:10A2C0000AF0B4FD0BF02AFE04F50D5104F5005020
:10A2D0000831383004F5005501F0BEF88023C5F888
:10A2E00088310423C4F8A43104F5907011F03EFEC7
:10A2F0002046FDF75FFF04F5BF40403054F0BCFB43
:10A3000004F557502C3007F02FFF04F52E502C3059
:10A3100060F016FA324B33491E68B06A03684FF496
:10A320007A72DB6A984701203BF06CFB04F59A4196
:10A330001A227C312046FFF777FE2B4A0621384649
:10A3400047F060FF2046FFF719FE04F5A8405C3097
:10A350001FF014FB04F5A0434FF48072C3F850259E
:10A36000224B0093224B019302AB13E9060004F544
:10A370007F6043F079FE76F055FF04F54057C7F84B
:10A3800078052046FDF75CFFD5F8EC1B29B1706A13
:10A3900003680222D3F880309847706A154B1A6818
:10A3A000036892F8F113D3F8AC30984795F8D413BA
:10A3B0001A222046FFF712FF50F0E2FA50F06AFA34
:10A3C00097F971364BB104F559504FF0FF312C30ED
:10A3D00003B0BDE8F04039F0D1BB03B0F0BD00BF21
:10A3E000542C0020A59D0108FC220C08582C0020AC
:10A3F000A19D01084892002000F57F6044F07ABCDE
:10A4000010B52DED028B044682B0462051F0C2FEFD
